:100000000C94130F0C94440F0C94440F0C94440F55
:100010000C94440F0C94440F0C94440F0C94440F14
:100020000C94440F0C94440F0C94440F0C94440F04
:100030000C94440F0C94F5D90C94440F0C94440F79
:100040000C94440F0C94FF860C94440F0C94440FB2
:100050000C94440F0C94440F0C9464980C94DDD3CE
:100060000C94440F0C9475210C94440F0C94440F81
:100070000C94440F0C94440F0C94440F0C94440FB4
:100080000C94440F0C94440F0C94440F0C94440FA4
:100090000C94440F0C94440F0C94440F0C94F4D023
:1000A0000C94440F0C94440F0C94440F0C94440F84
:1000B0000C94440F0C94440F0C94440F0C94440F74
:1000C0000C94440F0C94440F0C94440F0C94440F64
:1000D0000C94440F0C94440F0C94440F0C94440F54
:1000E0000C94440FBE98CD98E998F89812992199EC
:1000F0003B993F9947990BD510D515D51FD529D5D3
:10010000A2D533D53BD543D54DD557D561D570D57F
:100110007AD5A2D584D58ED598D5C4D5C7D5B6D530
:10012000BAD5C0D5FED5CBD5CFD5D5D5D9D5DDD58A
:10013000E3D5E7D5EBD5FED5F1D5F5D5F9D5084A08
:10014000D73B3BCE016E84BCBFFDC12F3D6C7431EB
:100150009ABD56833DDA3D00C77F11BED9E4BB4C42
:100160003E916BAAAABE000000803F05A84CCDB20C
:10017000D44EB93836A9020C50B9918688083CA6ED
:10018000AAAA2ABE000000803F004D383420582023
:1001900059205A20450043616E6E6F7420656E745D
:1001A0006572207375626469723A20004D323400C2
:1001B0004D3233202573006175746F25692E6700F9
:1001C0006572726F722077726974696E6720746FDE
:1001D0002066696C65004E6F74205344207072690C
:1001E0006E74696E67002F005344207072696E74DC
:1001F000696E67206279746520002E0044656C6525
:1002000074696F6E206661696C65642C2046696C48
:10021000653A200046696C652064656C65746564A8
:100220003A002E006F70656E206661696C65642C03
:100230002046696C653A200057726974696E6720C0
:10024000746F2066696C653A20002E006F70656ED1
:10025000206661696C65642C2046696C653A2000F3
:100260002E006F70656E206661696C65642C204697
:10027000696C653A200046696C652073656C65633E
:10028000746564002053697A653A200046696C659C
:10029000206F70656E65643A20002E006F70656E89
:1002A000206661696C65642C2046696C653A2000A3
:1002B0004E6F772066726573682066696C653A20B8
:1002C000004E6F7720646F696E672066696C653ACF
:1002D00020002220706F73002220706172656E749E
:1002E0003A2200535542524F5554494E45204341FE
:1002F0004C4C207461726765743A2200747279699B
:100300006E6720746F2063616C6C207375622D675B
:10031000636F64652066696C657320776974682013
:10032000746F6F206D616E79206C6576656C732ECD
:10033000204D4158206C6576656C2069733A0053F6
:10034000442063617264206F6B006F70656E526F42
:100350006F74206661696C656400766F6C756D659D
:100360002E696E6974206661696C6564005344206F
:10037000696E6974206661696C006563686F3A0034
:100380004572726F723A0048617264636F646564AB
:100390002044656661756C742053657474696E677A
:1003A00073204C6F616465640053746F72656420E0
:1003B00073657474696E67732072657472696576AB
:1003C0006564002044002049002020204D33303156
:1003D0002050005049442073657474696E67733A05
:1003E00000205A0020590020204D3230362058007D
:1003F000486F6D65206F666673657420286D6D2982
:100400003A00204500205A00205800204200205485
:100410000020204D323035205300416476616E63F8
:100420006564207661726961626C65733A20533D40
:100430004D696E20666565647261746520286D6D16
:100440002F73292C20543D4D696E2074726176659E
:100450006C20666565647261746520286D6D2F730C
:10046000292C20423D6D696E696D756D207365673D
:100470006D656E742074696D6520286D73292C205C
:10048000583D6D6178696D756D205859206A6572A7
:100490006B20286D6D2F73292C20205A3D6D6178BB
:1004A000696D756D205A206A65726B20286D6D2FFD
:1004B00073292C2020453D6D6178696D756D20454F
:1004C000206A65726B20286D6D2F732900205400FF
:1004D00020204D323034205300416363656C6572D7
:1004E0006174696F6E3A20533D616363656C657238
:1004F0006174696F6E2C20543D726574726163740F
:1005000020616363656C65726174696F6E0020457C
:1005100000205A0020590020204D32303120580050
:100520004D6178696D756D20416363656C657261BD
:1005300074696F6E20286D6D2F7332293A00204543
:1005400000205A0020590020204D3230332058001E
:100550004D6178696D756D2066656564726174655D
:100560007320286D6D2F73293A00204500205A0012
:1005700020590020204D3932205800537465707383
:100580002070657220756E69743A005365747469E1
:100590006E67732053746F726564006563686F3AA9
:1005A0000053544F505045442E20005072696E74D1
:1005B00065722073746F7070656420647565207453
:1005C0006F206572726F72732E204669782074688E
:1005D00065206572726F7220616E6420757365208C
:1005E0004D39393920746F20726573746172742EBD
:1005F000202854656D706572617475726520697329
:100600002072657365742E205365742069742061AF
:10061000667465722072657374617274696E67299D
:10062000004B494C4C45442E20005072696E746555
:10063000722068616C7465642E206B696C6C28296B
:100640002063616C6C656421006F6B00526573659B
:100650006E643A20000A00207A3A200020793A207D
:100660000020783A2000426564002200556E6B6ECF
:100670006F776E20636F6D6D616E643A2022004368
:1006800068616E67652066696C616D656E74000AED
:1006900000207A6F66667365743A20000A00207A3B
:1006A00070726F62655F7A6F66667365743A200078
:1006B0007A5F6D696E3A2000795F6D696E3A20004D
:1006C000785F6D696E3A2000205A3A0020593A004E
:1006D00020436F756E7420583A200020453A002060
:1006E0005A3A0020593A00583A004649524D57416B
:1006F00052455F4E414D453A4D61726C696E2056D0
:10070000313B20537072696E7465722F6772626C30
:10071000206D617368757020666F722067656E3634
:10072000204649524D574152455F55524C3A6874E4
:100730007470733A2F2F6769746875622E636F6DDA
:100740002F4572696B5A616C6D2F4D61726C696EC9
:100750002F2050524F544F434F4C5F5645525349F0
:100760004F4E3A312E30204D414348494E455F545B
:100770005950453A524F424F5231504C55535632D0
:100780002045585452554445525F434F554E543AB4
:100790003120555549443A30303030303030302DEA
:1007A000303030302D303030302D303030302D3052
:1007B00030303030303030303030300A00524F423C
:1007C0004F5231504C55535632204F66662E0052D0
:1007D0004F424F5231504C5553563220726561642E
:1007E000792E0042656420646F6E652E0020423AC7
:1007F0000020453A00543A0042656420486561741F
:10080000696E672E0048656174696E6720646F6E5B
:10081000652E0020573A0020453A00543A004865BA
:100820006174696E672E2E2E002042403A002040EF
:100830003A00202F003A00205400202F0020423A96
:1008400000202F006F6B20543A002569206D696EDF
:100850002C2025692073656300456E642066696CF1
:1008600065206C69737400426567696E2066696C07
:1008700065206C697374004E6F206D6F76652E0075
:10088000526573756D696E67207072696E7400577A
:1008900061697420666F7220757365722E2E2E004A
:1008A0000A00205A3A200020593A200020583A20C5
:1008B0000042656400205A3A0020593A0020436FF4
:1008C000756E7420583A200020453A00205A3A00AC
:1008D00020593A00583A0020643A200020623A2019
:1008E0000045716E20636F656666696369656E7445
:1008F000733A20613A2000486F6D6520582F5920C7
:100900006265666F7265205A00486F6D6520582FCA
:1009100059206265666F7265205A00205A3A00209D
:10092000593A0020436F756E7420583A20002045D4
:100930003A00205A3A0020593A00583A005A20709A
:10094000726F6265206F75742E20626564005A2094
:1009500070726F6265206F75742E20626564004846
:100960006F6D6520582F59206265666F7265205A39
:1009700000486F6D6520582F59206265666F72655B
:10098000205A00536C6565702E2E2E002569206854
:100990006F757273202569206D696E7574657300BB
:1009A000446F6E65207072696E74696E6720666947
:1009B0006C650053544F505045442E2000507269CE
:1009C0006E7465722073746F7070656420647565F1
:1009D00020746F206572726F72732E2046697820C2
:1009E000746865206572726F7220616E6420757321
:1009F00065204D39393920746F20726573746172C6
:100A0000742E202854656D7065726174757265204E
:100A100069732072657365742E2053657420697440
:100A20002061667465722072657374617274696E98
:100A30006729006F6B004E6F204C696E65204E7504
:100A40006D626572207769746820636865636B7393
:100A5000756D2C204C617374204C696E653A2000D2
:100A60004E6F20436865636B73756D20776974689A
:100A7000206C696E65206E756D6265722C204C610C
:100A80007374204C696E653A2000636865636B730C
:100A9000756D206D69736D617463682C204C617392
:100AA00074204C696E653A20004C696E65204E7565
:100AB0006D626572206973206E6F74204C6173746F
:100AC000204C696E65204E756D6265722B312C204D
:100AD0004C617374204C696E653A20004D313130A1
:100AE00000446F6E6520736176696E672066696C7D
:100AF000652E006F6B004D3239002020506C616E06
:100B00006E657242756666657242797465733A20E5
:100B1000002046726565204D656D6F72793A200040
:100B20004A756C203131203230313600436F6D70A0
:100B3000696C65643A200028526F426F2033442C60
:100B40002052312B2053696E676C65204578747292
:100B5000756465722900207C20417574686F723A53
:100B600020004A756C20313120323031362031324C
:100B70003A35323A313000204C617374205570643C
:100B8000617465643A2000312E302E30004D617260
:100B90006C696E0020536F667477617265205265D0
:100BA00073657400205761746368646F67205265D1
:100BB000736574002042726F776E206F75742052D7
:100BC00065736574002045787465726E616C20529F
:100BD0006573657400506F7765725570007374614A
:100BE0007274002200656E717565696E672022005F
:100BF0002200656E717565696E67202200FFFFFF38
:100C00000000A0400000A0400000803F00007043B2
:100C100000007E4300007043000000000000000060
:100C2000000000000000704300007E43000070439D
:100C30000000000000000000000000006563686F15
:100C40003A004572726F723A0020746F6F206C6FB9
:100C50006E6720657874727573696F6E2070726547
:100C600076656E7465640020636F6C6420657874CB
:100C7000727573696F6E2070726576656E746564E7
:100C8000006563686F3A007C3C3E5E2B3D3F2F5B06
:100C90005D3B2C2A225C00656E6473746F70732058
:100CA0006869743A205A00205A3A00656E64737479
:100CB0006F7073206869743A20590020593A0065B2
:100CC0006E6473746F7073206869743A20580020E2
:100CD000583A00656E6473746F7073206869743A73
:100CE000200024F4D43050C38E20C2A24017828B3F
:100CF0007011127A910D816CD90AA861E108C75868
:100D00006607615143061E4B5D05C145A7041A41A4
:100D10001104093D9803713931034036DB02653314
:100D20009102D4305402802E1D02632CEE01752AEC
:100D3000C501B028A001102781018F2564012B2453
:100D40004B01E0223401AC211F018D200D01801FD9
:100D5000FC00841EED00971DDF00B81CD200E61BCE
:100D6000C600201BBC00641AB200B219A8000A1900
:100D7000A0006A189900D117910040178B00B51692
:100D8000840031167E00B31579003A157300C7143C
:100D90006F0058146A00EE13660088136300251371
:100DA0005E00C7125B006C12570015125400C1118F
:100DB000510070114F0021114B00D61049008D10C9
:100DC00047004610440002104200C00F4000800F50
:100DD0003E00420F3C00060F3B00CB0E3800930E46
:100DE00037005C0E3500270E3400F30D3200C10DC4
:100DF0003100900D3000600D2E00320D2D00050DDC
:100E00002C00D90C2B00AE0C2900850C29005C0CA1
:100E10002700350C27000E0C2600E80B2400C40B1D
:100E20002400A00B23007D0B23005A0B2100390B5B
:100E30002100180B2000F80A1F00D90A1E00BB0A67
:100E40001E009D0A1D00800A1D00630A1C00470A3F
:100E50001B002C0A1B00110A1A00F7091A00DD09F1
:100E60001900C4091900AB091900920917007B0980
:100E70001800630917004C091600360916002009EE
:100E800016000A091500F5081500E0081400CC0842
:100E90001400B8081400A4081400900813007D087A
:100EA00012006B081300580812004608120034089C
:100EB0001100230811001208110001081100F007A9
:100EC0001000E0071000D0071000C0071000B007A6
:100ED0000F00A107100091070E0083070F00740791
:100EE0000F0065070E0057070E0049070E003B076D
:100EF0000D002E070E0020070D0013070D0006073A
:100F00000D00F9060C00ED060D00E0060C00D406FD
:100F10000C00C8060C00BC060C00B0060C00A406B1
:100F20000B0099060C008D060B0082060B0077065D
:100F30000B006C060B0061060A0057060B004C06FE
:100F40000A0042060A0038060A002E060A00240695
:100F50000A001A060A001006090007060A00FD0525
:100F60000900F4050900EB050900E2050900D905AF
:100F70000900D0050900C7050900BE050900B5052F
:100F80000800AD050800A50509009C0508009405AA
:100F900008008C050800840508007C05080074051D
:100FA00008006C050700650508005D05070056058B
:100FB00008004E05070047050700400508003805F2
:100FC0000700310507002A050700230507001C0557
:100FD0000600160507000F050700080506000205B4
:100FE0000700FB040600F5040700EE040600E80411
:100FF0000600E2040700DB040600D5040600CF0467
:101000000600C9040600C3040600BD040600B704B8
:101010000600B1040500AC040600A6040600A00406
:1010200005009B04060095040500900406008A0450
:10103000050085040500800406007A040500750497
:101040000500700405006B040500660405006104DA
:1010500005005C04050057040500520405004D041A
:10106000050048040500430405003E0404003A045A
:10107000050035040500300404002C040500270495
:101080000400230405001E0404001A0404001604CE
:101090000500110404000D04040009040500040403
:1010A000040000040400FC030400F8030400F4033B
:1010B0000400F0030400EC030400E8030400E4036C
:1010C0000400E0030400DC030400D8030400D4039C
:1010D0000400D0030400CC030400C8030300C503CC
:1010E000030024F404D9201BC40C5C0E9804C4092A
:1010F0005F0265077101F405F900FB04B3004804C1
:101100008700C10369005803550003034500BE0270
:101110003A008402310053022A0029022500040209
:101120002000E4011C00C8011900AF01170098015C
:1011300014008401130071011000610110005101BD
:101140000E0043010D0036010B002B010B002001A6
:101150000B00150109000C01090003010800FB0048
:101160000800F3000800EB000700E4000600DE00C2
:101170000600D8000600D2000600CC000500C7001B
:101180000500C2000500BD000400B9000400B50060
:101190000400B1000400AD000400A9000400A50093
:1011A0000300A20003009F0004009B0003009800BE
:1011B00003009500020093000300900003008D00DF
:1011C00002008B00030088000200860002008400F9
:1011D0000300810002007F0002007D0002007B000E
:1011E000020079000200770001007600020074001E
:1011F000020072000100710002006F0002006D0029
:1012000001006C0002006A00010069000200670032
:101210000100660001006500010064000200620038
:10122000010061000100600001005F0002005D003C
:1012300001005C0001005B0001005A000100590040
:101240000100580001005700010056000100550040
:10125000010054000100530000005300010052003F
:10126000010051000100500001004F0001004E003C
:1012700000004E0001004D0001004C0001004B0039
:1012800000004B0001004A00010049000100480035
:101290000000480001004700010046000000460031
:1012A000010045000000450001004400010043002A
:1012B0000000430001004200000042000100410024
:1012C000000041000100400001003F0000003F001D
:1012D00001003E0000003E0001003D0000003D0016
:1012E00001003C0000003C0000003C0001003B000D
:1012F00000003B0001003A0000003A000100390004
:1013000000003900010038000000380000003800FB
:1013100001003700000037000100360000003600F1
:1013200000003600010035000000350000003500E7
:1013300001003400000034000000340001003300DC
:1013400000003300000033000100320000003200D2
:1013500000003200010031000000310000003100C7
:1013600001003000000030000000300001002F00BC
:1013700000002F0000002F0000002F0001002E00B1
:1013800000002E0000002E0001002D0000002D00A6
:1013900000002D0000002D0001002C0000002C009A
:1013A00000002C0000002C0001002B0000002B008E
:1013B00000002B0000002B0001002A0000002A0082
:1013C00000002A0000002A00010029000000290076
:1013D0000000290000002900000029000100280069
:1013E000000028000000280000002800000028005D
:1013F0000100270000002700000027000000270050
:101400000000270001002600000026000000260042
:101410000000260000002600010025000000250035
:101420000000250000002500000025000000250028
:10143000010024000000240000002400000024001B
:10144000000024000100230000002300000023000E
:101450000000230000002300000023000000230000
:1014600001002200000022000000220000002200F3
:1014700000002200000022000100210000002100E5
:1014800000002100000021000000210000002100D8
:1014900000002100010020000000200000002000CA
:1014A00000002000000020000000200000002000BC
:1014B0000000200001001F0000001F0000001F00AE
:1014C00000001F0000001F0000001F0000001F00A0
:1014D00001001E0000001E0000001E0000001E0093
:1014E00000006563686F3A004572723A204D4158BA
:1014F00054454D50204245440054656D70657261FD
:101500007475726520686561746564206265642025
:101510007377697463686564206F66662E204D4139
:101520005854454D50207472696767657265642030
:101530002121004572723A204D494E54454D5000CC
:101540003A204578747275646572207377697463A4
:10155000686564206F66662E204D494E54454D5097
:101560002074726967676572656420210045727234
:101570003A204D415854454D50003A2045787472F8
:1015800075646572207377697463686564206F663B
:10159000662E204D415854454D502074726967673E
:1015A000657265642021004572723A2054454D50A1
:1015B0002046414C4C204552524F5200457874729F
:1015C00075646572207377697463686564206F66FB
:1015D000662E2054656D7065726174757265206643
:1015E000656C6C20746F6F206D7563682064757214
:1015F000696E67207072696E742100202D20496E1B
:1016000076616C6964206578747275646572206EA9
:10161000756D626572202100504944204175746FD8
:1016200074756E652066696E697368656421205003
:10163000757420746865206C617374204B702C2065
:101640004B6920616E64204B6420636F6E7374611C
:101650006E74732066726F6D2061626F76652069AB
:101660006E746F20436F6E66696775726174696F1F
:101670006E2E6800504944204175746F74756E6514
:10168000206661696C6564212074696D656F75748D
:101690000020403A006F6B20543A006F6B20423AB2
:1016A00000504944204175746F74756E6520666101
:1016B000696C6564212054656D7065726174757222
:1016C0006520746F6F206869676800204B643A205A
:1016D00000204B693A2000204B703A200020436CD8
:1016E00061737369632050494420002054753A2087
:1016F00000204B753A2000206D61783A2000206D63
:10170000696E3A200020643A200020626961733AD1
:1017100020004572726F723A0070012C019001270F
:1017200001B0012201C0011D01F0011801100213D6
:101730000130020E016002090190020401C002FFA3
:10174000000003FA004003F5008003F000D003EB33
:10175000002004E6007004E100E004DC004005D74E
:1017600000C005D2004006CD00D006C8008007C3E7
:10177000003008BE00F008B900C009B400B00AAFDC
:1017800000B00BAA00D00CA500000EA000500F9BCB
:1017900000C01096005012910000148C00C01587F4
:1017A00000B0178200B0197D00D01B7800001E73B6
:1017B0000040206E0090226900F024640040275F02
:1017C0000090295A00E02B5500102E500020304B7D
:1017D0000010324600E033410090353C00103737AE
:1017E0000070383200A0392D00B03A2800A03B2309
:1017F00000603C1E00103D1900903D1400103E0F8B
:1018000000703E0A00C03E0500003F0000436172C8
:10181000642072656D6F766564004361726420694F
:101820006E736572746564002D2D3A2D2D002D2D7B
:101830002D005344002059000120000120004D36A6
:101840003030004368616E67652066696C616D6564
:101850006E7400466C6F7700466C6F770046616E61
:101860002073706565640046616E20737065656401
:101870000042656400426564004E6F7A7A6C6500D0
:101880004E6F7A7A6C6500537065656400537065BD
:101890006564004D61696E00580059005A00457832
:1018A000747275646572004578747275646572004F
:1018B0004D6F7665205A004D6F76652059004D6F4B
:1018C00076652058004D6F76652061786973004D0C
:1018D0006F766520302E316D6D004D6F766520314D
:1018E0006D6D004D6F76652031306D6D0050726505
:1018F00070617265004D6F76652061786973004D87
:1019000038300053776974636820706F7765722090
:101910006F6E004D38310053776974636820706FC3
:10192000776572206F666600436F6F6C646F776EC9
:1019300000507265686561742041425300507265C1
:101940006865617420504C4100473238004175741D
:101950006F20686F6D65004D3834004469736162B3
:101960006C65207374657070657273004D61696E8B
:101970000053746F7265206D656D6F7279004265FA
:101980006400426564004E6F7A7A6C65004E6F7A2F
:101990007A6C650046616E2073706565640046610F
:1019A0006E2073706565640054656D706572617456
:1019B0007572650053746F7265206D656D6F727915
:1019C0000042656400426564004E6F7A7A6C65007F
:1019D0004E6F7A7A6C650046616E2073706565643F
:1019E0000046616E2073706565640054656D7065B6
:1019F000726174757265005072656865617420412A
:101A0000425320636F6E6600507265686561742092
:101A1000504C4120636F6E66005049442D43005086
:101A200049442D43005049442D44005049442D441D
:101A3000005049442D49005049442D490050494423
:101A40002D50005049442D500020022046616374FF
:101A50000020022046616374002002204D6178005E
:101A60002002204D6178002002204D696E00200286
:101A7000204D696E004F6666004F6E20004F66660F
:101A8000004F6E20004175746F74656D7000466183
:101A90006E2073706565640046616E2073706565C5
:101AA000640042656400426564004E6F7A7A6C653A
:101AB000004E6F7A7A6C6500436F6E74726F6C00C3
:101AC0004573746570732F6D6D0045737465707325
:101AD0002F6D6D005A73746570732F6D6D005A739E
:101AE000746570732F6D6D005973746570732F6D0D
:101AF0006D005973746570732F6D6D005873746544
:101B000070732F6D6D005873746570732F6D6D0059
:101B1000412D7265747261637400412D7265747237
:101B200061637400416D6178206500416D617820CA
:101B30006500416D6178207A00416D6178207A00FE
:101B4000416D6178207900416D6178207900416DA7
:101B50006178207800416D61782078005654726178
:101B600076206D696E005654726176206D696E0044
:101B7000566D696E00566D696E00566D6178206510
:101B800000566D6178206500566D6178207A0056A8
:101B90006D6178207A00566D6178207900566D610C
:101BA00078207900566D6178207800566D61782034
:101BB000780056652D6A65726B0056652D6A6572F0
:101BC0006B00567A2D6A65726B00567A2D6A6572C3
:101BD0006B005678792D6A65726B005678792D6A9C
:101BE00065726B00416363656C00416363656C0003
:101BF0005A204F6666736574005A204F6666736597
:101C00007400436F6E74726F6C00526573746F7200
:101C100065206661696C73616665004C6F61642064
:101C20006D656D6F72790053746F7265206D656DAF
:101C30006F7279004D6F74696F6E0054656D7065D9
:101C4000726174757265004D61696E004D383420A3
:101C5000582059205A2045004D3234004D3233204F
:101C6000257300052E2E004D61696E004E6F2053C6
:101C7000442063617264005072696E742066726FF2
:101C80006D2053440053746F70207072696E74003D
:101C9000526573756D65207072696E740050617560
:101CA0007365207072696E7400436F6E74726F6C2E
:101CB00000507265706172650054756E6500496E02
:101CC000666F2073637265656E000A00207A3A20A1
:101CD0000020793A200020783A200000000A0B0208
:101CE000090C0D0E080703040100000000000000AD
:101CF00000000000000000000000000000000000E4
:101D000000000000000000121110000000000000A0
:101D100000000000000000000000000000000000C3
:101D200000010210202008081020401020408002EE
:101D30000102010804020101020408102040808011
:101D40004020100804020180040201804020100895
:101D5000040201080402010102040810204080016D
:101D6000020408102040800505050507050808083D
:101D700008020202020A0A0808040404040101011C
:101D80000101010101030303030303030304070724
:101D9000070C0C0C0C0C0C0C0C02020202060606C2
:101DA00006060606060B0B0B0B0B0B0B0B0000229B
:101DB00000250028002B002E003100340002010015
:101DC00000050108010B0100002100240027002A62
:101DD000002D003000330001010000040107010A5A
:101DE00001024E414E494E495459494E46CDCCCC44
:101DF0003D0AD7233C17B7D13877CC2B329595E6DF
:101E0000241FB14F0A000020410000C84200401CBE
:101E10004620BCBE4CCA1B0E5AAEC59D740006516E
:101E200068BCC8D00A5111241FBECFEFD1E2DEBF7B
:101E3000CDBF00E00CBF14E0A0E0B2E0E8E8FDECAC
:101E400001E00BBF02C007900D92A63CB107D9F785
:101E500023E1A6ECB4E001C01D92A634B207E1F77D
:101E60001EE1C4E2DEE100E006C022970109FE01A6
:101E70000BBF0E9454DFCE31D10780E00807A9F7DD
:101E80000E946ED60C94B3E60C940000FC01148200
:101E900017821382128288E594E0918380830895EB
:101EA00028E534E0FC01318320832781222319F0C7
:101EB00004960C94307D0895CF92DF92EF92FF92BA
:101EC0000F931F93CF93DF93EC018F96DFDFCE014B
:101ED000805B9F4FDBDF7E012FE6E20EF11C870166
:101EE0006E013BE5C31A3EEFD30AC801CFDF015EA6
:101EF0001F4F0C151D05C9F7FE01E955FE4F89E17D
:101F0000818314823596178ACE0186539E4FBEDF99
:101F1000FE01E558FD4F108211821282138238961D
:101F200010821182128213821A821B8218821982F5
:101F30006E0181E8C81A8DEFD80AF601108211826D
:101F400012821382F80111821082FE01E751FE4FC6
:101F5000108286E391E0F7019C01119221503040FC
:101F6000E1F7FE01E957FD4F81E080831EA61DA623
:101F70000E9427D468577C4E8F4F9F4FF601608395
:101F8000718382839383DF91CF911F910F91FF9093
:101F9000EF90DF90CF900895FC0120E03EE2DB015E
:101FA0004C91403241F0283011F430833196DB01FE
:101FB0004C91408331962F5F6F5F7F4F2B3079F7C5
:101FC000108208953F924F925F926F927F928F920C
:101FD0009F92AF92BF92CF92DF92EF92FF920F93B8
:101FE0001F93CF93DF93CDB7DEB7C758D1090FB694
:101FF000F894DEBF0FBECDBF8C016B017A01312C8E
:1020000084E0E80EF11C2801E1E14E0E511C58015C
:10201000F8E7AF1AFDEFBF0A480186E7881A8DEF8F
:10202000980A80E4682E712C6C0E7D1EE4E06E0E22
:10203000711CA201BE016F5F7F4FC7010E949A7B96
:1020400018160CF021C12C85322F3871303109F06F
:102050009CC0F501808191810197029708F495C099
:10206000BE016F5F7F4FCE0187589F4F95DFA096CF
:102070001FAEA097F6018081811107C067E173E070
:10208000CE01815A9F4F0E949EE3B601CE01815A34
:102090009F4F0E949EE3BE0167587F4FCE01815A39
:1020A0009F4F0E949EE367E173E0CE01815A9F4FEC
:1020B0000E949EE3CE01805C9F4FE8DE21E0AE01EE
:1020C00047585F4FB701C3010E94277F811139C074
:1020D000F50180819181892BA1F5EAE7F3E08491F4
:1020E000882341F09091C00095FFFCCF8093C600FB
:1020F0003196F5CFE9E1F3E08191882339F09091B1
:10210000C00095FFFCCF8093C600F6CF8091C00041
:1021100085FFFCCF8AE08093C600FE01E758FF4FA1
:102120008191882339F09091C00095FFFCCF809376
:10213000C600F6CF8091C00085FFFCCF8AE0809377
:10214000C6008BE1FE01EC5BFF4FDE01959601902E
:102150000D928A95E1F724968EAD9FAD24979CA3AE
:102160008BA388E594E09AA389A3AE014F5D5F4FEE
:10217000BE01615A7F4FC80125DFCE01819690DEF6
:10218000CE01805C9F4F8CDE54CF8981882309F477
:102190007BC0853E09F44DCF8E3209F44ACF8F358E
:1021A00009F447CFF8018189882331F08E3209F490
:1021B00040CF8F3509F43DCF23FD3BCF81E0303157
:1021C00009F080E0F80184A7811108C0898587346F
:1021D00009F02FCF8A858E3709F42BCF98012C5F19
:1021E0003F4FBE016F5F7F4FC901CA57DF4F288342
:1021F000C658D040C957DF4F3883C758D040CCDECF
:10220000F50180819181CA57DF4F2881C658D0409F
:10221000C957DF4F3881C758D0400097F1F4F60115
:102220008191882339F09091C00095FFFCCF809375
:10223000C600F6CFF9018191882339F09091C00052
:1022400095FFFCCF8093C600F6CF8091C00085FF3C
:10225000FCCF8AE08093C600ECCE8130910539F442
:10226000F40180819181019691838083E2CE02976F
:1022700009F0DFCE232D30E0F40180819181281711
:10228000390711F03394D5CEC957DF4F0FB6F89404
:10229000DEBF0FBECDBFDF91CF911F910F91FF9099
:1022A000EF90DF90CF90BF90AF909F908F907F90F6
:1022B0006F905F904F903F900895EF92FF920F9331
:1022C0001F93CF93DF93CDB7DEB76F970FB6F89418
:1022D000DEBF0FBECDBF8C01FC01E857FD4F118260
:1022E00010827C0183E3E80EF11C40E050E0BA016B
:1022F000C7010E944D7C8BE1F701DE01159601902C
:102300000D928A95E1F7F80181A992A99C838B83AC
:1023100088E594E09A838983AE014F5F5F4F6FE653
:1023200074E0C8014FDECE010196BADD6F960FB69C
:10233000F894DEBF0FBECDBFDF91CF911F910F91FB
:10234000FF90EF9008952BE1FB013496DC01149689
:1023500001900D922A95E1F7FB0122813381FC0166
:10236000338322830895EF92FF920F931F93CF93AD
:10237000DF93EC011B828EA9882321F0CE01C39646
:102380000E94307D7E0189E5E81A8EEFF80A45E368
:1023900060E0C7010E94B17781111FC0EAE7F3E056
:1023A0008491882341F09091C00095FFFCCF8093E9
:1023B000C6003196F5CFEDE6F3E08491882341F035
:1023C0009091C00095FFFCCF8093C6003196F5CF69
:1023D0008091C00085FFFCCF76C08E0104551E4F52
:1023E00041E0B701C8010E941A85811126C040E072
:1023F000B701C8010E941A8581111FC0E0E8F3E00F
:102400008491882341F09091C00095FFFCCF809388
:10241000C6003196F5CFEAE5F3E08491882341F0D8
:102420009091C00095FFFCCF8093C6003196F5CF08
:102430008091C00085FFFCCF46C0B801CE01C39695
:102440000E943E7A81111FC0E0E8F3E08491882366
:1024500041F09091C00095FFFCCF8093C60031966B
:10246000F5CFEAE4F3E08491882341F09091C00035
:1024700095FFFCCF8093C6003196F5CF8091C000C8
:1024800085FFFCCF20C081E08B83EAE7F3E08491F5
:10249000882341F09091C00095FFFCCF8093C60047
:1024A0003196F5CFEFE3F3E08491882341F09091EA
:1024B000C00095FFFCCF8093C6003196F5CF809188
:1024C000C00085FFFCCF8AE08093C6008E01015DCD
:1024D0001F4FB801CE01805B9F4F35DFC25BDF4FDE
:1024E00019830883DF91CF911F910F91FF90EF9097
:1024F0000895FC01128213820895FC012381222396
:1025000011F021E022830895FC0122812111128221
:102510000895AF92BF92CF92DF92EF92FF920F9306
:102520001F93CF93DF931F92CDB7DEB78C018FE25D
:10253000FB0181935F01D12C41E07801FBE5EF1AAB
:10254000FEEFFF0A9FE1C92E2D2D30E0F7018081BB
:10255000918128173907D8F4C29EC001C39E900DFF
:1025600011248D589F4FB501800F911F49830E9400
:10257000E579C50149815C010196F501208122239D
:1025800021F04D3810F44F5FF6CFD394DDCF47FDE7
:1025900011C0B501C80182539E4F0F90DF91CF91BA
:1025A0001F910F91FF90EF90DF90CF90BF90AF9071
:1025B0000C94E579F50110820F90DF91CF911F9176
:1025C0000F91FF90EF90DF90CF90BF90AF90089564
:1025D0002F923F924F925F926F927F928F929F9233
:1025E000AF92BF92CF92DF92EF92FF920F931F9321
:1025F000CF93DF93CDB7DEB7AC970FB6F894DEBFBD
:102600000FBECDBF8C016B01342EFC01838188236A
:1026100009F4D3C2EF52FE4F8081882309F4F8C039
:102620002111C4C07801F7E1EF1AFEEFFF0AF701AC
:102630008081882361F1E0E8F3E08491882341F010
:102640009091C00095FFFCCF8093C6003196F5CFE6
:10265000ECEFF2E08491882341F09091C00095FF67
:10266000FCCF8093C6003196F5CF4AE050E061E0A0
:1026700070E086EC94E00E94C2228091C00085FF49
:10268000FCCF8AE08093C6000E94303196C2EAE710
:10269000F3E08491882341F09091C00095FFFCCF36
:1026A0008093C6003196F5CFE3EEF2E08491882363
:1026B00041F09091C00095FFFCCF8093C600319609
:1026C000F5CFF6018191882339F09091C00095FFF4
:1026D000FCCF8093C600F6CFE8EDF2E0849188232A
:1026E00041F09091C00095FFFCCF8093C6003196D9
:1026F000F5CFF70180813DE8B32EB801B89E600D9B
:10270000711D112462517E4FC80103DFF7018081E2
:10271000F801B89EE00DF11D1124E251FE4F8191A8
:10272000882339F09091C00095FFFCCF8093C600BC
:10273000F6CFE2EDF2E08491882341F09091C00061
:1027400095FFFCCF8093C6003196F5CF5801FDE789
:10275000AF1AFDEFBF0AF50140815181628173819B
:102760002AE030E086EC94E00E94EE228091C000E6
:1027700085FFFCCF8AE08093C600F7012081F80135
:1027800084E0289FE00DF11D1124AF0146515E4FFA
:10279000F50180819181A281B381FA0180839183C7
:1027A000A283B3832F5FF70120832CC0EAE7F3E015
:1027B0008491882341F09091C00095FFFCCF8093D5
:1027C000C6003196F5CFE1ECF2E08491882341F028
:1027D0009091C00095FFFCCF8093C6003196F5CF55
:1027E000F6018191882339F09091C00095FFFCCFCC
:1027F0008093C600F6CF8091C00085FFFCCF8AE0B1
:102800008093C600C80182539E4F0E94307D30C025
:10281000F801E751FE4F1082EAE7F3E08491882344
:1028200041F09091C00095FFFCCF8093C600319697
:10283000F5CFE0EBF2E08491882341F09091C00065
:1028400095FFFCCF8093C6003196F5CFF6018191BC
:10285000882339F09091C00095FFFCCF8093C6008B
:10286000F6CF8091C00085FFFCCF8AE08093C60040
:10287000F8011282CE0101965C0108DB28019EE47A
:10288000490E511CC8018F96F20191838083F60195
:1028900080818F3209F084C06FE270E0C6010E942F
:1028A000A9E301967C012AE0222EE114F10409F447
:1028B0007DC06FE270E0C7010E94A9E34C01009760
:1028C00009F475C0E816F90608F071C03C016E18ED
:1028D0007F08A301B701CE0180960E94C9E3E0E220
:1028E000F0E0EC0FFD1FE60DF71D1082FE01B09623
:1028F0008191882339F09091C00095FFFCCF80939F
:10290000C600F6CF8091C00085FFFCCF2092C600A4
:10291000F201608171816115710519F06C5F7F4F63
:1029200002C060E070E021E0AE01405E5F4FCE018A
:1029300005960E94277F81112BC0ECE9F2E084917B
:10294000882341F09091C00095FFFCCF8093C60092
:102950003196F5CFFE01B0968191882339F09091A0
:10296000C00095FFFCCF8093C600F6CFEAE9F2E005
:102970008491882341F09091C00095FFFCCF809313
:10298000C6003196F5CF8091C00085FFFCCFEAC02C
:10299000F201B182A0827401FFEFEF1AFF0A85CF26
:1029A000C801805B9F4FF201918380837601C8014B
:1029B00082539E4F4C01F20160817181332009F4F2
:1029C00099C06115710519F06C5F7F4F02C060E01E
:1029D00070E021E0A701C4010E94277F882309F449
:1029E0005FC0F40181899289A389B489F801E5580F
:1029F000FD4F80839183A283B383ECE8F2E084915E
:102A0000D801A558BD4F882349F09091C00095FF8B
:102A1000FCCF8093C60031968491F5CFF701819168
:102A2000882339F09091C00095FFFCCF8093C600B9
:102A3000F6CFE4E8F2E08491882341F09091C00061
:102A400095FFFCCF8093C6003196F5CF4D915D91F7
:102A50006D917C912AE030E086EC94E00E94EE22B9
:102A60008091C00085FFFCCF8AE08093C600F8010A
:102A7000ED57FD4F1082118212821382E6E7F2E0D9
:102A80008491882341F09091C00095FFFCCF809302
:102A9000C6003196F5CF8091C00085FFFCCF85C080
:102AA000E2E6F2E08491882341F09091C00095FF26
:102AB000FCCF8093C6003196F5CFF7018191882332
:102AC00039F09091C00095FFFCCF8093C600F6CFFF
:102AD000E0E6F2E08491882341F09091C00095FFF8
:102AE000FCCF8093C6003196F5CF8091C00085FF62
:102AF000FCCF38C06115710519F06C5F7F4F02C0C3
:102B000060E070E026E5A701C4010E94277F8111E3
:102B10002DC0ECE4F2E08491882341F09091C00054
:102B200095FFFCCF8093C6003196F5CFF7018191D8
:102B3000882339F09091C00095FFFCCF8093C600A8
:102B4000F6CFEAE4F2E08491882341F09091C0004E
:102B500095FFFCCF8093C6003196F5CF8091C000E1
:102B600085FFFCCF8AE08093C60025C081E0F80194
:102B70008083E8E3F2E08491882341F09091C000E3
:102B800095FFFCCF8093C6003196F5CFF601819179
:102B9000882339F09091C00095FFFCCF8093C60048
:102BA000F6CF8091C00085FFFCCF8AE08093C600FD
:102BB000C7010E94B0AAC50173D9AC960FB6F894AC
:102BC000DEBF0FBECDBFDF91CF911F910F91FF9060
:102BD000EF90DF90CF90BF90AF909F908F907F90BD
:102BE0006F905F904F903F902F90089521E0FC01EF
:102BF000218340E0EDCC3F924F925F926F927F92A3
:102C00008F929F92AF92BF92CF92DF92EF92FF92FC
:102C10000F931F93CF93DF93CDB7DEB7AC970FB66B
:102C2000F894DEBF0FBECDBF7C015B01FC01838148
:102C3000882309F400C1C70182539E4F0E94307D52
:102C4000F7011282CE0101966C0120D927019EE482
:102C5000490E511CC7018F96F20191838083F501C3
:102C600080818F3209F084C06FE270E0C5010E945C
:102C7000A9E38C010F5F1F4F4AE0342E01151105A7
:102C800009F47CC06FE270E0C8010E94A9E34C0126
:102C9000009709F474C00817190708F070C03C01C8
:102CA000601A710AA301B801CE0180960E94C9E39F
:102CB000E0E2F0E0EC0FFD1FE60DF71D1082FE01D3
:102CC000B0968191882339F09091C00095FFFCCF98
:102CD0008093C600F6CF8091C00085FFFCCF309274
:102CE000C600F201608171816115710519F06C5F98
:102CF0007F4F02C060E070E021E0AE01405E5F4FB8
:102D0000CE0105960E94277F81112BC0E4E2F2E0FC
:102D10008491882341F09091C00095FFFCCF80936F
:102D2000C6003196F5CFFE01B0968191882339F027
:102D30009091C00095FFFCCF8093C600F6CFE2E2F1
:102D4000F2E08491882341F09091C00095FFFCCF80
:102D50008093C6003196F5CF8091C00085FFFCCFEF
:102D600065C0F201D182C08284010F5F1F4F86CF00
:102D7000C701805B9F4FF201918380838501F2013F
:102D800080819181009711F0049602C080E090E06C
:102D9000B8010E94FD7F882301F1E4E1F2E0849113
:102DA000882341F09091C00095FFFCCF8093C6002E
:102DB0003196F5CFF8018191882339F09091C000C8
:102DC00095FFFCCF8093C600F6CFF701ED57FD4F7E
:102DD00010821182128213822CC0ECEFF1E08491F8
:102DE000882341F09091C00095FFFCCF8093C600EE
:102DF0003196F5CFF8018191882339F09091C00088
:102E000095FFFCCF8093C600F6CFEAEFF1E0849106
:102E1000882341F09091C00095FFFCCF8093C600BD
:102E20003196F5CF8091C00085FFFCCF8AE080937A
:102E3000C600C60135D8AC960FB6F894DEBF0FBEFB
:102E4000CDBFDF91CF911F910F91FF90EF90DF9059
:102E5000CF90BF90AF909F908F907F906F905F903A
:102E60004F903F900895CF93DF93EC018B8188239F
:102E7000C1F1E8EEF1E08491882341F09091C00027
:102E800095FFFCCF8093C6003196F5CFFE01ED573C
:102E9000FD4F40815181628173812AE030E086ECF0
:102EA00094E00E94EE22E6EEF1E08491882341F066
:102EB0009091C00095FFFCCF8093C6003196F5CF6E
:102EC000C558DD4F488159816A817B812AE030E015
:102ED00086EC94E00E94EE228091C00085FFFCCF3A
:102EE00011C0E6EDF1E08491882341F09091C0009B
:102EF00095FFFCCF8093C6003196F5CF8091C0003E
:102F000085FFFCCF8AE08093C600DF91CF910895C2
:102F1000AF92BF92CF92DF92EF92FF920F931F93E7
:102F2000CF93DF935C01EB01FB0101900020E9F7F7
:102F30008F0101501109061B170B6C01F2E3CF1A28
:102F4000FEEFDF0AF60110826EE470E0CE010E940F
:102F5000A9E37C01009729F4F8013197EC0FFD1FDC
:102F60000DC060E270E00E94A9E3EC0121966AE2E4
:102F700070E0C7010E94A9E3FC0131978DE08183D5
:102F80008AE082831382BE01C50186539E4F0E9450
:102F9000C381F6018081882309F1E0E8F3E08491A0
:102FA000882341F09091C00095FFFCCF8093C6002C
:102FB0003196F5CFE0ECF1E08491882341F09091D7
:102FC000C00095FFFCCF8093C6003196F5CF80916D
:102FD000C00085FFFCCF8AE08093C600DF91CF91CF
:102FE0001F910F91FF90EF90DF90CF90BF90AF9027
:102FF00008952F923F924F925F926F927F928F929D
:103000009F92AF92BF92CF92DF92EF92FF920F9377
:103010001F93CF93DF93CDB7DEB7CC55D1090FB651
:10302000F894DEBF0FBECDBF8C0189579D4F5C0168
:10303000662339F0F5011082F801838181111DC0EA
:1030400015C0FC018081882309F4ADC0F801E15866
:10305000FD4FC080D180E280F3800E9427D4C61645
:10306000D706E806F90608F49EC0E4CFC8017BD96C
:10307000F8018381882309F496C0F80186A58F930F
:1030800085A58F9387EB91E09F938F937E01FFE35C
:10309000EF0EF11CFF92EF920E94D8E30F900F9079
:1030A0000F900F900F900F90B12CF701019000201E
:1030B000E9F73197EE19FF09BE1684F46701CB0CCE
:1030C000D11CB7FCDA94F6018081992787FD909591
:1030D0000E942FE3F6018083B394E7CF4801F3E326
:1030E0008F0E911C40E050E0BA01C4010E944D7C5B
:1030F000512CCE0101966C0150EB652E51E0752EDE
:103100005E0191E2A90EB11C40E050E0B601C4019D
:103110000E949A7B1816DCF5412CF60101900020E4
:10312000E9F73197EC19FD094E1674F41601240CD9
:10313000311C47FC3A94F101808190E00E942FE31A
:10314000F10180834394E9CF8A858E37E9F245E027
:1031500050E0B701C6010E94BBE3892BA9F6FF929C
:10316000EF927F926F92BF92AF920E94D8E3C50117
:103170000E946A278CEA91E00E94DD270F900F9051
:103180000F900F900F900F9055245394BDCF511076
:1031900004C08FEF9FEFF80104C0F80185A596A544
:1031A000019696A785A7C45ADF4F0FB6F894DEBFE5
:1031B0000FBECDBFDF91CF911F910F91FF90EF9088
:1031C000DF90CF90BF90AF909F908F907F906F9047
:1031D0005F904F903F902F9008950F931F93CF9340
:1031E000DF93EC018C0102531E4FC8010E94E67C64
:1031F000C8010E94307D18821982DF91CF911F9102
:103200000F910895EF92FF920F931F93CF93DF9347
:10321000CDB7DEB76F970FB6F894DEBF0FBECDBF48
:103220008C017C018EE4E80EF11CC801805B9F4F8D
:10323000F70191838083E65CFD4F22E030E031832B
:103240002083329670E07183608340E050E0BA01E1
:1032500004960E944D7CF701808191812BE1FC0155
:103260003496DE01159601900D922A95E1F7FC0146
:10327000828193819C838B8388E594E09A83898300
:10328000AE014F5F5F4F6FE674E0C8010E94E20F2E
:10329000CE0101960E94500F6F960FB6F894DEBFD4
:1032A0000FBECDBFDF91CF911F910F91FF90EF9097
:1032B0000895CF92DF92EF92FF920F931F93CF93D7
:1032C000DF93CDB7DEB76F970FB6F894DEBF0FBEB2
:1032D000CDBF8C016C012EE4C20ED11C805B9F4FD0
:1032E000F60191838083E65CFD4F21E030E031837D
:1032F00020837801F6E7EF1AFDEFFF0AF70111824C
:10330000108240E050E0BA0104960E944D7CF60124
:10331000808191812BE1FC013496DE0115960190AC
:103320000D922A95E1F7FC01828193819C838B8326
:1033300088E594E09A838983AE014F5F5F4F6FE623
:1033400074E0C8010E94E20FCE0101960E94500F66
:10335000F701808191816F960FB6F894DEBF0FBEA2
:10336000CDBFDF91CF911F910F91FF90EF90DF9034
:10337000CF900895AF92BF92CF92DF92EF92FF92DB
:103380000F931F93CF93DF93CDB7DEB76F970FB631
:10339000F894DEBF0FBECDBF8C017B01CE0101963C
:1033A0000E94460FF801E95AFF4F808168018111A0
:1033B00004C02FE2C20ED11C03C080E5C80ED11C90
:1033C00021E0A701B6016C5F7F4FCE0105960E94F8
:1033D000277F81112DC0EAE7F3E08491882341F033
:1033E0009091C00095FFFCCF8093C6003196F5CF39
:1033F000E6E9F1E08491882341F09091C00095FFC7
:10340000FCCF8093C6003196F5CFF70181918823D8
:1034100039F09091C00095FFFCCF8093C600F6CFA5
:103420008091C00085FFFCCF8AE08093C60036C043
:10343000F801EB55FE4F808191818A30910530F57E
:103440009C012F5F3F4F318320832FE1289F700124
:10345000299FF00C11242FE6E20EF11CE00EF11E64
:103460005C01B701C7014F960E94A31181E0A81A21
:10347000B1082FE1E21AF1088FEFA816B80689F714
:10348000B601C80181599F4F0E94A311BE016F5F11
:103490007F4FC801805B9F4F0E94A311CE01019610
:1034A0000E94500F6F960FB6F894DEBF0FBECDBFCF
:1034B000DF91CF911F910F91FF90EF90DF90CF9010
:1034C000BF90AF900895EF92FF920F931F93CF9309
:1034D000DF93EC01CB55DE4F288139812115310571
:1034E000F9F021503109398328838C0101591F4F8C
:1034F000B801805B9F4F0E94A311C80100E010E05B
:103500007C012FE1E20EF11C28813981021713079B
:1035100038F40F5F1F4FB7010E94A311C701F0CF0E
:10352000DF91CF911F910F91FF90EF900895EF924F
:10353000FF920F931F93CF93DF93EC010E94038EB2
:103540008E0107511E4FF80180819E0122533E4F8C
:1035500079018823A1F1C9010E94307DF8018081A1
:1035600081508083BE01FDE88F9F600D711D112485
:1035700062517E4F21E041E0CE012AD8F8018081DE
:10358000FE0124E0829FE00DF11D1124E651FE4F63
:103590004081518162817381FE01ED57FD4F40836F
:1035A000518362837383C7010E944D7CCE01DF91FA
:1035B000CF911F910F91FF90EF900C947D120E947C
:1035C000918EC7010E94307D1A828AE891E00E94A4
:1035D000DD278091BE0E8823F9F01092BE0EC091B7
:1035E0002207D0E0CC0FDD1FC551DE4E6881798106
:1035F000882777FD8095982F0E94D1DB20913D028E
:1036000030913E0240913F02509140020E9432DDD3
:10361000181614F419821882DF91CF911F910F911F
:10362000FF90EF900895EF92FF920F931F93CF9327
:10363000DF931F92CDB7DEB78C017B01460FF701F8
:1036400061917F01F8018081918149830E94FCE5AD
:10365000F8018081918101969183808349814E1187
:10366000EECF0F90DF91CF911F910F91FF90EF90D0
:103670000895EF92FF920F931F93CF93DF931F92C2
:10368000CDB7DEB78C017B01460FF80180819181B7
:1036900049830E94F4E5F70181937F01F80180815D
:1036A000918101969183808349814E11EECF0F90D5
:1036B000DF91CF911F910F91FF90EF9008950F939D
:1036C0001F93CF93DF93CDB7DEB72C970FB6F89447
:1036D000DEBF0FBECDBF80E390E3A0E3B0E08D83FB
:1036E0009E83AF83B88704E610E01C870B8744E015
:1036F000BE016B5F7F4FCE010B9695DF40E16FE11E
:103700007FE0CE010B968FDF40E16FE27FE0CE01DC
:103710000B9689DF40E16FE07FE0CE010B9683DFFF
:1037200044E067E07FE0CE010B967DDF44E063E09C
:103730007FE0CE010B9677DF44E06BE07FE0CE01C7
:103740000B9671DF44E063EF7EE0CE010B966BDFFA
:1037500044E06FE37FE0CE010B9665DF44E06FEF5E
:103760007EE0CE010B965FDF44E06BEF7EE0CE01A2
:103770000B9659DF44E067EF7EE0CE010B9653DFF6
:103780004CE066E377E0CE010B964DDF42E06BE460
:1037900072E1CE010B9647DF42E069E472E1CE01AF
:1037A0000B9641DF42E067E472E1CE010B963BDF0E
:1037B00042E065E472E1CE010B9635DF42E063E45E
:1037C00072E1CE010B962FDF42E061E472E1CE019F
:1037D0000B9629DF44E063E277E0CE010B9623DF0E
:1037E00044E060E872E0CE010B961DDF44E06CE738
:1037F00072E0CE010B9617DF44E068E772E0CE017D
:103800000B9611DF80E290E09A87898742E0BE0143
:10381000675F7F4FCE010B9606DF86E591E3A0E35D
:10382000B0E089839A83AB83BC831C870B8744E019
:10383000BE016F5F7F4FCE010B96F5DEEBE9F5E041
:103840008491882341F09091C00095FFFCCF809334
:10385000C6003196F5CFEBE8F5E08491882341F07E
:103860009091C00095FFFCCF8093C6003196F5CFB4
:103870008091C00085FFFCCF8AE08093C6002C9623
:103880000FB6F894DEBF0FBECDBFDF91CF911F9171
:103890000F910895CF93DF93CBE9D5E0FE0184919A
:1038A000882341F09091C00095FFFCCF8093C60023
:1038B0003196F5CFEBE7F5E08491882341F09091C4
:1038C000C00095FFFCCF8093C6003196F5CF809164
:1038D000C00085FFFCCF8AE08093C600FE01849182
:1038E000EBE9F5E0882349F09091C00095FFFCCF0B
:1038F0008093C60031968491F5CF40911F0F50916F
:10390000200F6091210F7091220F83E795E00E94B4
:103910002B274091230F5091240F6091250F709118
:10392000260F80E795E00E942B274091270F5091AA
:10393000280F6091290F70912A0F8DE695E00E9463
:103940002B2740912B0F50912C0F60912D0F7091D0
:103950002E0F8AE695E00E942B278091C00085FFFC
:10396000FCCF8AE08093C600FE018491EBE9F5E08C
:10397000882349F09091C00095FFFCCF8093C6004A
:1039800031968491F5CFE0E5F5E08491882341F00C
:103990009091C00095FFFCCF8093C6003196F5CF83
:1039A0008091C00085FFFCCF8AE08093C600FE01B5
:1039B0008491EBE9F5E0882349F09091C00095FFF0
:1039C000FCCF8093C60031968491F5CF40912F0FA4
:1039D0005091300F6091310F7091320F87E495E074
:1039E0000E942B274091330F5091340F6091350F77
:1039F0007091360F84E495E00E942B274091370F99
:103A00005091380F6091390F70913A0F81E495E031
:103A10000E942B2740913B0F50913C0F60913D0F2E
:103A200070913E0F8EE395E00E942B278091C0009D
:103A300085FFFCCF8AE08093C600FE018491EBE90C
:103A4000F5E0882349F09091C00095FFFCCF80936A
:103A5000C60031968491F5CFE0E2F5E084918823A9
:103A600041F09091C00095FFFCCF8093C600319645
:103A7000F5CF8091C00085FFFCCF8AE08093C6001F
:103A8000FE018491EBE9F5E0882349F09091C000B4
:103A900095FFFCCF8093C60031968491F5CF40917D
:103AA0000F0F5091100F6091110F7091120F87E15D
:103AB00095E00E943C274091130F5091140F6091A4
:103AC000150F7091160F84E195E00E943C274091FC
:103AD000170F5091180F6091190F70911A0F81E113
:103AE00095E00E943C2740911B0F50911C0F609164
:103AF0001D0F70911E0F8EE095E00E943C27809173
:103B0000C00085FFFCCF8AE08093C600FE0184914F
:103B1000EBE9F5E0882349F09091C00095FFFCCFD8
:103B20008093C60031968491F5CFE9EDF4E084915D
:103B3000882341F09091C00095FFFCCF8093C60090
:103B40003196F5CF8091C00085FFFCCF8AE080934D
:103B5000C600FE018491EBE9F5E0882349F09091DD
:103B6000C00095FFFCCF8093C60031968491F5CFBD
:103B70004091070F5091080F6091090F70910A0F43
:103B800080ED94E00E942B274091030F5091040F89
:103B90006091050F7091060F8DEC94E00E942B2729
:103BA0008091C00085FFFCCF8AE08093C600FE01B3
:103BB0008491EBE9F5E0882349F09091C00095FFEE
:103BC000FCCF8093C60031968491F5CFEAE1F4E012
:103BD0008491882341F09091C00095FFFCCF8093A1
:103BE000C6003196F5CF8091C00085FFFCCF8AE0FA
:103BF0008093C600FE018491EBE9F5E0882349F04B
:103C00009091C00095FFFCCF8093C60031968491BF
:103C1000F5CF40910B0F50910C0F60910D0F7091EB
:103C20000E0F81E194E00E942B274091F30E5091FA
:103C3000F40E6091F50E7091F60E8EE094E00E9405
:103C40002B2740913F0F5091400F6091410F709191
:103C5000420F8BE094E00E943C274091FF0E509170
:103C6000000F6091010F7091020F88E094E00E94B4
:103C70002B274091FB0E5091FC0E6091FD0E709130
:103C8000FE0E85E094E00E942B274091F70E5091A4
:103C9000F80E6091F90E7091FA0E82E094E00E94A5
:103CA0002B278091C00085FFFCCF8AE08093C6005F
:103CB000FE018491EBE9F5E0882349F09091C00082
:103CC00095FFFCCF8093C60031968491F5CFE0EF4D
:103CD000F3E08491882341F09091C00095FFFCCFE0
:103CE0008093C6003196F5CF8091C00085FFFCCF50
:103CF0008AE08093C600FE018491EBE9F5E0882319
:103D000049F09091C00095FFFCCF8093C60031969A
:103D10008491F5CF4091360750913707609138076D
:103D20007091390787EE93E00E942B2740913A0764
:103D300050913B0760913C0770913D0784EE93E002
:103D40000E942B2740913E0750913F07609140070A
:103D50007091410781EE93E00E942B278091C00073
:103D600085FFFCCF8AE08093C600FE018491EBE9D9
:103D7000F5E0882349F09091C00095FFFCCF809337
:103D8000C60031968491F5CFE3EDF3E0849188236A
:103D900041F09091C00095FFFCCF8093C600319612
:103DA000F5CF8091C00085FFFCCF8AE08093C600EC
:103DB000FE01C491EBE9F5E0CC2349F08091C0000D
:103DC00085FFFCCFC093C6003196C491F5CF4091DA
:103DD000800250918102609182027091830289EC8D
:103DE00093E00E942B2760917C0270917D0280916C
:103DF0007E0290917F020E94CA99AB01BC0186ECC1
:103E000093E00E942B276091780270917902809153
:103E10007A0290917B020E94D699AB01BC0183EC9F
:103E200093E00E942B278091C00085FFFCCF8AE0A1
:103E30008093C600DF91CF910895AF92BF92CF9249
:103E4000DF92EF92FF920F931F93CF93DF93CDB743
:103E5000DEB7E0970FB6F894DEBF0FBECDBF80E1AE
:103E6000E7EAF2E0DE01919601900D928A95E1F782
:103E700080E1E7EBF2E0DE01519601900D928A9528
:103E8000E1F780E1E7ECF2E0DE01119601900D929E
:103E90008A95E1F76E0181E2C80ED11C8FE1E82E10
:103EA0008FE0F82E8E010F5E1F4F6FE27FE0AE01B4
:103EB0004F5F5F4F9FE0A92E9FE0B92E20E030E0DA
:103EC000F60181919191A191B1916F01F7018193D7
:103ED0009193A193B1937F01F80181919191A19167
:103EE000B1918F01FB0181939193A193B193BF0194
:103EF000FA0181919191A191B191AF01F501819365
:103F00009193A193B1935F012F5F3F4F243031050F
:103F1000B9F60E94FA6480E090E8A2EAB4E48093E3
:103F2000070F9093080FA093090FB0930A0F80E03A
:103F300090E8ABE3B5E48093030F9093040FA09354
:103F4000050FB093060F10920B0F10920C0F1092EA
:103F50000D0F10920E0F80E29EE4A0E0B0E080937F
:103F60003F0F9093400FA093410FB093420F1092D8
:103F7000F30E1092F40E1092F50E1092F60E80E0F1
:103F800090E0A8E8B1E48093FF0E9093000FA09317
:103F9000010FB093020F8DEC9CECACECBEE3809370
:103FA000FB0E9093FC0EA093FD0EB093FE0E80E0EE
:103FB00090E0A0EAB0E48093F70E9093F80EA093FF
:103FC000F90EB093FA0E10923E0710923F0710922E
:103FD00040071092410710923A0710923B07109247
:103FE0003C0710923D071092360710923707109247
:103FF00038071092390782ED90E090934C1280932D
:104000004B1287E390E090934A12809349128FEF0E
:1040100090E090934812809347122BEE30E030935B
:1040200046122093451220E530E03093441220934D
:104030004312909342128093411286E696E6A6E6DA
:10404000BFEB8093230790932407A0932507B09399
:1040500026078AE999E9A1EBB1E480938002909365
:104060008102A0938202B093830261E77DE38AE834
:104070009FE30E94C49960937C0270937D028093B9
:104080007E0290937F0260E070E084EE92E40E94F2
:10409000D099609378027093790280937A0290931A
:1040A0007B020E94449080E090E0A0E8BFE3809310
:1040B000740290937502A0937602B0937702EBE9B5
:1040C000F5E08491882341F09091C00095FFFCCFEA
:1040D0008093C6003196F5CFE7E8F3E0849188231A
:1040E00041F09091C00095FFFCCF8093C6003196BF
:1040F000F5CF8091C00085FFFCCF8AE08093C60099
:10410000E0960FB6F894DEBF0FBECDBFDF91CF9122
:104110001F910F91FF90EF90DF90CF90BF90AF90E5
:104120000895CF93DF93CDB7DEB72C970FB6F894F1
:10413000DEBF0FBECDBF84E690E09C878B8786E50F
:1041400091E3A0E3B0E089839A83AB83BC8344E02E
:10415000BE016B5F7F4FCE010B968BDA43E050E0E0
:10416000BE016B5F7F4FCE0101960E94BBE3892B9E
:1041700009F0B1C040E16FE17FE0CE010B9679DA42
:1041800040E16FE27FE0CE010B9673DA40E16FE031
:104190007FE0CE010B966DDA0E94FA6444E067E09E
:1041A0007FE0CE010B9665DA44E063E07FE0CE016C
:1041B0000B965FDA44E06BE07FE0CE010B9659DAB4
:1041C00044E063EF7EE0CE010B9653DA44E06FE308
:1041D0007FE0CE010B964DDA44E06FEF7EE0CE013A
:1041E0000B9647DA44E06BEF7EE0CE010B9641DAA6
:1041F00044E067EF7EE0CE010B963BDA4CE066E3ED
:1042000077E0CE010B9635DA42E06BE472E1CE0145
:104210000B962FDA42E069E472E1CE010B9629DABF
:1042200042E067E472E1CE010B9623DA42E065E4F6
:1042300072E1CE010B961DDA42E063E472E1CE0139
:104240000B9617DA42E061E472E1CE010B9611DAC7
:1042500044E063E277E0CE010B960BDA44E060E8DD
:1042600072E0CE010B9605DA44E06CE772E0CE0115
:104270000B96FFD944E068E772E0CE010B96F9D9BE
:1042800042E0BE01675F7F4FCE010B96F2D90E94DC
:104290004490EBE9F5E08491882341F09091C000CF
:1042A00095FFFCCF8093C6003196F5CFE9EAF3E0A5
:1042B0008491882341F09091C00095FFFCCF8093BA
:1042C000C6003196F5CF8091C00085FFFCCF8AE013
:1042D0008093C60001C0B1DD2C960FB6F894DEBF06
:1042E0000FBECDBFDF91CF9108951F920F920FB6F1
:1042F0000F9211240BB60F922F933F934F935F931E
:104300006F938F939F93EF93FF936091C6002091DB
:10431000470530914805C90101968F77992740914B
:10432000490550914A058417950741F0F901E95371
:10433000FB4F60839093480580934705FF91EF9171
:104340009F918F916F915F914F913F912F910F901E
:104350000BBE0F900FBE0F901F9018959A01AB01E6
:10436000211581EE38074105510549F182E080931E
:10437000C00060E079E08DE390E00E9422DF2150F0
:10438000310941095109CA01B90122E030E040E098
:1043900050E00E9422DF3093C5002093C40080913A
:1043A000C10080618093C1008091C10088608093CA
:1043B000C1008091C10080688093C100089510926F
:1043C000C00020E130E0E7CF2091490530914A0557
:1043D00080914705909148058217930771F0F90184
:1043E000E953FB4F80812F5F3F4F2F773327309367
:1043F0004A052093490590E008958FEF9FEF0895B7
:104400008091490590914A0590934805809347050E
:1044100008954F925F926F927F928F929F92AF9288
:10442000BF92CF92DF92EF92FF920F931F93CF93A1
:10443000DF93CDB7DEB7A0970FB6F894DEBF0FBEFF
:10444000CDBF5C014115510561057105E9F420E01E
:1044500030E040E350E060E070E0A0960FB6F894E2
:10446000DEBF0FBECDBFDF91CF911F910F91FF90A7
:10447000EF90DF90CF90BF90AF909F908F907F9004
:104480006F905F904F905BC08E010F5F1F4FC12CEC
:10449000D12C76014801422E512C612C712C8FEFCA
:1044A000C81AD80AE80AF80ACB01BA01A301920196
:1044B0000E9400DFCA01F80161938F01A901BC01CC
:1044C000411551056105710551F7F1E0CF1AD10889
:1044D000E108F108F401EC0DFD1D80818A3010F433
:1044E00040E301C047E3480F552747FD5095652F2E
:1044F000752F20E030E0C50122D081E0C81AD10834
:10450000E108F108EFEFCE16DE06EE06FE0611F723
:10451000A0960FB6F894DEBF0FBECDBFDF91CF914E
:104520001F910F91FF90EF90DF90CF90BF90AF90D1
:104530009F908F907F906F905F904F90089521157E
:10454000310539F48091C00085FFFCCF4093C6004F
:1045500008952A30310509F41CC05BCFCF93DF9357
:10456000EC0120E030E04DE050E060E070E0E7DF9B
:1045700020E030E04AE050E060E070E0CE01DF9102
:10458000CF91DDCF9A01AB01662757FD6095762F5D
:10459000D6CFCF92DF92EF92FF92CF93DF93EC01D1
:1045A0006A017B0177FF0FC020E030E04DE250E070
:1045B00060E070E0C4DFF094E094D094C094C11C3B
:1045C000D11CE11CF11C2AE0B701A601CE01DF914C
:1045D000CF91FF90EF90DF90CF901BCF2115310549
:1045E00039F48091C00085FFFCCF4093C600089548
:1045F00010CF9A01462F50E060E070E0EFCFCF93EC
:10460000DF93EC019A01AB0160E070E0E7DFCE01DF
:10461000DF91CF91A3CF8F929F92AF92BF92CF9213
:10462000DF92EF92FF921F93CF93DF93EC016A0129
:104630007B01122F20E030E0A901C701B6010E94E2
:104640002FDB87FF0CC020E030E04DE250E060E05F
:1046500070E0CE0174DFF7FAF094F7F8F094B12C23
:1046600060E070E080E09FE3B11641F020E030E0D0
:1046700040E251E40E9436DBB394F6CF9B01AC01DB
:10468000C701B6010E9456DA6B017C010E94A3DBD0
:104690004B015C010E94CFDB9B01AC01C701B6015D
:1046A0000E9455DA6B017C012AE0B501A401CE011C
:1046B000B0DE112361F0EBEAF4E08191882339F058
:1046C0009091C00095FFFCCF8093C600F6CF1123D8
:1046D00019F120E030E040E251E4C701B6010E9448
:1046E00004DE6B017C010E949EDB4B01AA2497FC37
:1046F000A094BA2CB501A401CE014BDFC501B401D1
:104700000E94D1DB9B01AC01C701B6010E9455DAC2
:104710006B017C011150DBCFDF91CF911F91FF9096
:10472000EF90DF90CF90BF90AF909F908F900895C3
:1047300072CFFC0165917591859194910895809156
:104740000B0290910C02A0910D02B0910E02809389
:10475000FC069093FD06A093FE06B093FF068091A1
:10476000230290912402909353078093520784E68A
:1047700090E090932402809323020E9427D46093B8
:104780005B0570935C0580935D0590935E0581E009
:104790000C94F68680E00E94F6868091FC0690914B
:1047A000FD06A091FE06B091FF0680930B02909348
:1047B0000C02A0930D02B0930E02809152079091CB
:1047C000530790932402809323020E9427D460937E
:1047D0005B0570935C0580935D0590935E0508957D
:1047E0004F925F926F927F928F929F92AF92BF9201
:1047F000CF92DF92EF92FF920F931F9340900B02A4
:1048000050900C0260900D0270900E02812C912C41
:10481000EAEFAE2EE5E4BE2E80920B0290920C02DF
:10482000A0920D02B0920E0260934207709343076C
:10483000809344079093450720934607309347079A
:104840004093480750934907E0924A07F0924B077C
:1048500000934C0710934D07E2E2F7E0FF93EF93CC
:10486000F5E58F2E982CF5E0AF2EF3E4BF2EAEE4E5
:10487000CA2EA7E0DA2E0E9470590E94038E409241
:104880000B0250920C0260920D0270920E020F9079
:104890000F901F910F91FF90EF90DF90CF90BF90FE
:1048A000AF909F908F907F906F905F904F90089502
:1048B0002F923F924F925F926F927F928F929F9230
:1048C000AF92BF92CF92DF92EF92FF920F931F931E
:1048D000CF93DF9385E492E00E94AACEEDE2F2E06E
:1048E000608171818281938160930B0270930C02CD
:1048F00080930D0290930E0220E030E040E752E4F6
:104900000E9436DB4B015C01C6E4D7E02881398187
:104910004A815B81E2E4F7E0608171818281938169
:10492000B2E22B2EB7E03B2E3F922F921EE4C12E17
:1049300017E0D12EE12CF12C00E211EC0E9470590D
:104940000E94038E82E00E946B8E4B015C012881E5
:1049500039814A815B81E2E4F7E060817181828183
:104960009381850174010E94EC6388E09CE0E1DEA4
:104970009B01AC01C501B4010E9456DA2B013C0138
:1049800020E030E040E752E460910B0270910C02AD
:1049900080910D0290910E020E9436DB4B015C016A
:1049A000288139814A815B81E2E4F7E0608171818D
:1049B000828193813F922F92830172010E947059EC
:1049C0000E94038E20E030E040E85EE3EDE2F2E09A
:1049D00060817181828193810E9404DE4B015C01C0
:1049E00060930B0270930C0280930D0290930E0261
:1049F00088E09CE09EDE6B017C0120E030E040E737
:104A000052E4C501B4010E9436DB4B015C01A701F1
:104A10009601C701B6010E9456DA9B01AC01C301A1
:104A2000B2010E9455DA7B018C01288139814A81CB
:104A30005B81E2E4F7E060817181828193813F9242
:104A40002F92FEE4CF2EF7E0DF2E0E9470590E94D5
:104A5000038E82E00E946B8E7B018C0160934A077B
:104A600070934B0780934C0790934D0728813981B1
:104A70004A815B81E2E4F7E0608171818281938108
:104A80000E94EC630F900F900F900F900F900F907B
:104A9000DF91CF911F910F91FF90EF90DF90CF901A
:104AA000BF90AF909F908F907F906F905F904F904E
:104AB0003F902F9008952F923F924F925F926F9266
:104AC0007F928F929F92AF92BF92CF92DF92EF929E
:104AD000FF920F931F93CF93DF93CDB7DEB72A9743
:104AE0000FB6F894DEBF0FBECDBF9E838D83FC0151
:104AF000E350F44FB490880F991F880F991F9A873D
:104B000089878E5B984F9A838983DC011D921D9261
:104B10001D921C921397BAE42B2EB7E03B2EF101A5
:104B2000E080F18002811381A6E4B7E02D913D91F0
:104B30004D915C91E2E4F7E0608171818281938123
:104B4000EEE4CE2EE7E0DE2E0E94EC6389859A85A6
:104B5000845F934FEEDD6B017C016B2D772767FD42
:104B60007095872F972F0E94D1DB2B013C0129855F
:104B70003A85205F384F3C832B8320E030E040ECC7
:104B80005FE3C701B6010E9404DEA30192010E9407
:104B900004DEAB81BC816D937D938D939C931397C1
:104BA000E985FA85EB5DFD4FF887EF8360817181C0
:104BB0008281938160930B0270930C0280930D02AB
:104BC00090930E0220E030E040E752E40E9436DB92
:104BD0004B015C01A8E1B7E0ED90FD900D911C91B7
:104BE000E4E1F7E02081318142815381A0E1B7E027
:104BF0006D917D918D919C91A2E2B7E0BF93AF93AF
:104C0000FCE1CF2EF7E0DF2E0E9470590E94038E48
:104C1000A981BA811D921D921D921C921397F101D8
:104C2000E080F18002811381A6E4B7E02D913D91EF
:104C30004D915C91E2E4F7E0608171818281938122
:104C4000AEE4CA2EA7E0DA2E0E94EC6329853A85ED
:104C50002050344F1901C9016CDD9058A301920115
:104C60000E9404DEAB81BC816D937D938D939C93F8
:104C7000139720E030E040E752E460910B0270911E
:104C80000C0280910D0290910E020E9436DB4B01C6
:104C90005C01E8E1F7E0E080F18002811381A4E1AA
:104CA000B7E02D913D914D915C91E0E1F7E060819D
:104CB000718182819381A2E2B7E0BF93AF93BCE19F
:104CC000CB2EB7E0DB2E0E9470590E94038EC101EB
:104CD00030DD9B01AC010E9456DAA30192010E94D3
:104CE00004DEAB81BC816D937D938D939C93139770
:104CF00020E030E040E05FE3EF81F8856081718182
:104D0000828193810E9404DE60930B0270930C02F7
:104D100080930D0290930E0220E030E040E752E4D1
:104D20000E9436DB4B015C01A8E1B7E0ED90FD90FD
:104D30000D911C91E4E1F7E02081318142815381A2
:104D4000A0E1B7E06D917D918D919C91A2E2B7E0D9
:104D5000BF93AF930E9470590E94038E89859A85F4
:104D6000885E934FE6DC09851A850A5C184FD801E6
:104D70002D913D914D915C910E9456DAE981FA8125
:104D8000608371838283938389859A85805D934F45
:104D9000D0DC29853A85265D384F7901D8012D91DF
:104DA0003D914D915C910E9456DAF70160837183C9
:104DB0008283938389859A858C5D934FBADC29859C
:104DC0003A852F5E3D4F7901D8012D913D914D914E
:104DD0005C910E9456DAF70160837183828393832A
:104DE000E981FA8180819181A281B381EB81FC818B
:104DF00080839183A283B38310920B0210920C02E2
:104E000010920D0210920E020E94EF86ED81FE813B
:104E1000E95DF84F81E080830F900F900F900F9025
:104E20000F900F902A960FB6F894DEBF0FBECDBF3D
:104E3000DF91CF911F910F91FF90EF90DF90CF9076
:104E4000BF90AF909F908F907F906F905F904F90AA
:104E50003F902F900895FC012491222341F030913E
:104E6000C00035FFFCCF2093C6000196F4CF22E0AE
:104E700030E086EC94E05CCCFC012491222341F0EC
:104E80003091C00035FFFCCF2093C6000196F4CFCF
:104E90002AE030E086EC94E0A1CBCF93DF931F9221
:104EA0001F92CDB7DEB780914013909141139E01C0
:104EB0002F5F3F4F009719F42654334102C0281B3F
:104EC000390B3A83298389819A810F900F90DF9162
:104ED000CF91089520916505309166052430310504
:104EE0000CF06AC0409167055091680560E6649FC8
:104EF0009001659F300D1124BC01C90181599A4F61
:104F00000E94B4E3ECE3FCE08491882341F09091AB
:104F1000C00095FFFCCF8093C6003196F5CFE2EF3D
:104F2000FBE08491882341F09091C00095FFFCCF75
:104F30008093C6003196F5CF809167059091680502
:104F400020E6289FF001299FF00D1124E159FA4F26
:104F50008191882339F09091C00095FFFCCF809318
:104F6000C600F6CFE0EFFBE08491882341F09091FA
:104F7000C00095FFFCCF8093C6003196F5CF80919D
:104F8000C00085FFFCCF8AE08093C6008091670552
:104F900090916805019664E070E00E94EDDE9093C8
:104FA0006805809367058091650590916605019677
:104FB000909366058093650508952091650530916D
:104FC0006605243031050CF06AC0409167055091A8
:104FD000680560E6649F9001659F300D1124BC0157
:104FE000C90181599A4F0E9437E3ECE3FCE08491B8
:104FF000882341F09091C00095FFFCCF8093C600BC
:105000003196F5CFE5EEFBE08491882341F0909155
:10501000C00095FFFCCF8093C6003196F5CF8091FC
:1050200067059091680520E6289FF001299FF00D03
:105030001124E159FA4F8191882339F09091C000F1
:1050400095FFFCCF8093C600F6CFE3EEFBE08491A2
:10505000882341F09091C00095FFFCCF8093C6005B
:105060003196F5CF8091C00085FFFCCF8AE0809318
:10507000C6008091670590916805019664E070E034
:105080000E94EDDE90936805809367058091650529
:105090009091660501969093660580936505089545
:1050A00060E089E20E94FFD5A09A0895269A2E9882
:1050B0000895F6DFFBDF40E950ED63E070E086EC39
:1050C00094E04CD9EDEDFBE08491882341F0909180
:1050D000C00095FFFCCF8093C6003196F5CF80913C
:1050E000C00085FFFCCF8AE08093C6008CE39CE083
:1050F000FC012491222341F03091C00035FFFCCF08
:105100002093C6003196F5CF24B720FF14C0E5EDFB
:10511000FBE03491332341F04091C00045FFFCCFC8
:105120003093C6003196F5CF3091C00035FFFCCFEB
:105130003AE03093C60021FF14C0E5ECFBE0349167
:10514000332341F04091C00045FFFCCF3093C600AF
:105150003196F5CF3091C00035FFFCCF3AE0309367
:10516000C60022FF14C0E4EBFBE03491332341F08E
:105170004091C00045FFFCCF3093C6003196F5CF7B
:105180003091C00035FFFCCF3AE03093C60023FFDA
:1051900014C0E4EAFBE03491332341F04091C000B5
:1051A00045FFFCCF3093C6003196F5CF3091C0005B
:1051B00035FFFCCF3AE03093C60025FF14C0E4E988
:1051C000FBE02491222341F03091C00035FFFCCF59
:1051D0002093C6003196F5CF2091C00025FFFCCF6B
:1051E0002AE02093C60014BEEDE8FBE024912223C0
:1051F00041F03091C00035FFFCCF2093C6003196BE
:10520000F5CFE7E8FBE02491222341F03091C00084
:1052100035FFFCCF2093C6003196F5CF2091C0001A
:1052200025FFFCCF2AE02093C600FC012491ECE38B
:10523000FCE0222349F03091C00035FFFCCF2093E1
:10524000C60031962491F5CFE7E7FBE024912223B5
:1052500041F03091C00035FFFCCF2093C60031965D
:10526000F5CFE2E6FBE02491222341F03091C0002B
:1052700035FFFCCF2093C6003196F5CFE6E5FBE085
:105280002491222341F03091C00035FFFCCF2093C0
:10529000C6003196F5CFE7E3FBE02491222341F0ED
:1052A0003091C00035FFFCCF2093C6003196F5CF7A
:1052B0002091C00025FFFCCF2AE02093C600ECE23D
:1052C000FBE02491222341F03091C00035FFFCCF58
:1052D0002093C6003196F5CFE0E2FBE02491222333
:1052E00041F03091C00035FFFCCF2093C6003196CD
:1052F000F5CF2091C00025FFFCCF2AE02093C60007
:10530000FC018491ECE3FCE0882349F09091C0001B
:1053100095FFFCCF8093C60031968491F5CFE1E1F3
:10532000FBE08491882341F09091C00095FFFCCF71
:105330008093C6003196F5CFB0DD4AE050E0BC0165
:1053400086EC94E01FD9EAEFFAE08491882341F0DB
:105350009091C00095FFFCCF8093C6003196F5CFA9
:105360004AE050E060ED74E086EC94E00BD9809167
:10537000C00085FFFCCF8AE08093C60010926B05C9
:1053800010926C0510926D0510926E050E9491208E
:105390000E9466900E94EE570E94808D0E9430AB62
:1053A000FFEF23ED80E3F15020408040E1F700C0A3
:1053B0000000089580915F059091600560E070E0C5
:1053C00001960C948EE080915F05909160054AE013
:1053D00050E060E070E001960C94F6E1682F7727CA
:1053E00067FD70952091690530916A0540E6429FFE
:1053F000C001439F900D112481599A4F0E94A9E347
:105400009093600580935F0521E0892B09F420E0EB
:10541000822F08950E9427D460935B0570935C05EA
:1054200080935D0590935E0508950E9427D4609354
:105430005B0570935C0580935D0590935E05E0913C
:105440006905F0916A05E559FA4F8081811114C010
:10545000E9E4F6E08491882341F09091C00095FF43
:10546000FCCF8093C6003196F5CF8091C00085FFB8
:10547000FCCF8AE08093C600089586EC94E00E94F9
:105480000022ECE4F6E08491882341F09091C00082
:1054900095FFFCCF8093C6003196F5CF4091F4067E
:1054A0005091F5066091F6067091F7064F5F5F4FD9
:1054B0006F4F7F4F2AE030E086EC94E040D8809137
:1054C000C00085FFFCCF8AE08093C600AECF2F924C
:1054D0003F924F925F926F927F928F929F92AF9284
:1054E000BF92CF92DF92EF92FF920F931F93CF93D1
:1054F000DF93CDB7DEB76E970FB6F894DEBF0FBE61
:10550000CDBF30E6932E04E010E04DEBE42E49E0F1
:10551000F42E5AE0852E63E3C62E6AE0D62E772459
:1055200073948091470590914805209149053091E9
:105530004A05821B930B8F779927892B09F425C283
:10554000809165059091660504970CF01EC286EC6B
:1055500094E00E94E42180936405209162053091DB
:1055600063058A3061F08D3051F08A3321F49091D7
:105570006105992321F02F3531050CF428C121153F
:10558000310509F442C18091670590916805989EA4
:105590005001999EB00C1124F501E20FF31FE1595F
:1055A000FA4F10822091610521110CC1FC01E559CF
:1055B000FA4F1082950121593A4F19016EE470E0BB
:1055C000C9010E94A9E30097E9F1909360058093D7
:1055D0005F05821993098A0D9B1D4AE050E060E047
:1055E00070E080599A4F0E94F6E16093F80670933C
:1055F000F9068093FA069093FB062091F406309109
:10560000F5064091F6065091F7062F5F3F4F4F4F3A
:105610005F4FA0906705B090680562177307840715
:10562000950709F4F5C09A9CC0019B9C900D11242C
:105630006CED7AE081599A4F0E946EE3892B09F054
:10564000E7C076C16AE270E0C1010E94A9E3892B3C
:1056500009F444C0E2E4FCE08491882341F0909195
:10566000C00095FFFCCF8093C6003196F5CFE6E3EE
:10567000FAE08491882341F09091C00095FFFCCF1F
:105680008093C6003196F5CF4091F4065091F5060F
:105690006091F6067091F7062AE030E086EC94E01F
:1056A0000E949F228091C00085FFFCCF8AE08093FA
:1056B000C6001092630510926205CDC28091F80673
:1056C0009091F906A091FA06B091FB068093F4063A
:1056D0009093F506A093F606B093F70680916705C0
:1056E00090916805989E5001999EB00C1124C501B7
:1056F00081599A4F1C0167E470E00E94A9E300976A
:1057000009F44BC09093600580935F05821993095B
:105710008A0D9B1D60E070E080599A4F0E948EE0D8
:105720000E949EDB6430710508F037C080914D0502
:1057300081111AC080915A0781112FC0F6018491FE
:10574000E3E3FAE0882349F09091C00095FFFCCF95
:105750008093C60031968491F5CF8091C00085FF7B
:10576000FCCF8092C60019C0F7018491EDEBF9E0FF
:10577000882349F09091C00095FFFCCF8093C6002C
:1057800031968491F5CF8091C00085FFFCCF809247
:10579000C60083EB99E00E94BFAA809167059091B3
:1057A00068050196B8010E94EDDE9093680580932C
:1057B0006705809165059091660501969093660551
:1057C000809365051092630510926205AACE8B3313
:1057D00011F470926105909161059111A2CE4091F2
:1057E000670550916805B9016F5F7F4F709363053E
:1057F00060936205949EF001959EF00D1124E20FD6
:10580000F31FE159FA4F80838CCE1092610523C2B9
:105810009A9C10019B9C300C1124C10181599A4F14
:105820005C016AE270E00E94A9E3009789F5E2E476
:10583000FCE08491882341F09091C00095FFFCCF5B
:105840008093C6003196F5CFE0E6FAE08491882394
:1058500041F09091C00095FFFCCF8093C600319637
:10586000F5CF4091F4065091F5066091F6067091DF
:10587000F7062AE030E086EC94E00E949F228091B7
:10588000C00085FFFCCF8AE08093C600F6DD11CF13
:1058900020E0612CF101E20FF11DE159FA4F308156
:1058A0003A3219F02F5F6326F5CF9093600580930D
:1058B0005F058A199B09820D931D60E070E0805995
:1058C0009A4F0E948EE00E949EDB262D30E0261724
:1058D000370709F4F3CEE2E4FCE08491882341F039
:1058E0009091C00095FFFCCF8093C6003196F5CF14
:1058F000EAE8FAE08491882341F09091C00095FF96
:10590000FCCF8093C6003196F5CF4091F4065091BC
:10591000F5066091F6067091F7062AE030E086EC15
:1059200094E00E949F228091C00085FFFCCFABCF06
:10593000E2E4FCE08491882341F09091C00095FF5F
:10594000FCCF8093C6003196F5CFE9EAFAE0849166
:10595000882341F09091C00095FFFCCF8093C60052
:105960003196F5CF4091F4065091F5066091F60618
:105970007091F7062AE030E086EC94E00E949F22C6
:105980008091C00085FFFCCF7ECF80915C0788238B
:1059900009F461C18091620590916305892B09F03A
:1059A0005AC18091650590916605892B11F410927A
:1059B0004B0598EE292E93E0392E412C512C2CE3E7
:1059C000C22ED12CE12CF12C8E010F5F1F4F80E6EF
:1059D000682E772473944091DD095091DE0960911F
:1059E000DF097091E0098091D5099091D609A091C5
:1059F000D709B091D809481759076A077B0708F0FB
:105A00002AC1809165059091660504970CF023C129
:105A100080914B0581111FC180913009909131090E
:105A2000A0913209B09133098093DD099093DE098A
:105A3000A093DF09B093E00988E299E00E94847B9B
:105A4000482F809364058A30B9F04D30A9F0433275
:105A500029F420916105211103C00EC04A33C9F316
:105A600020916205309163052F3531052CF48F3F6D
:105A7000FFEF9F0709F0D1C04091DD095091DE0989
:105A80006091DF097091E0098091D5099091D60964
:105A9000A091D709B091D809481759076A077B0721
:105AA00008F481C0E0EAF9E08491882341F0909104
:105AB000C00095FFFCCF8093C6003196F5CF809152
:105AC000C00085FFFCCFFAE0F093C6000E9427D407
:105AD00060934F0570935005809351059093520544
:105AE0008090530590905405A0905505B0905605B0
:105AF000681979098A099B09A20191010E9400DFB6
:105B000049015A01CA01B901A70196010E9400DFAB
:105B1000CA01B901A70196010E9400DF7F936F932C
:105B2000C501B40120E13EE040E050E00E9400DF0A
:105B30003F932F93ACE8B9E0BF93AF931F930F93BC
:105B40000E94D8E3ECE3FCE084910FB6F894DEBF4A
:105B50000FBECDBF882349F09091C00095FFFCCFC8
:105B60008093C60031968491F5CFF8018191882306
:105B700039F09091C00095FFFCCF8093C600F6CF1E
:105B80008091C00085FFFCCF3AE03093C600C80189
:105B90000E94B0AA8AE597E00E94971A61E08AE520
:105BA00097E00E94F91780916405833211F4709296
:105BB0004B0520916205309163052115310509F4EB
:105BC00024CE8091670590916805689EF001699EDA
:105BD000F00D1124E20FF31FE159FA4F1082FC017E
:105BE000E559FA4F708220916505309166052F5F67
:105BF0003F4F3093660520936505019664E070E0A1
:105C00000E94EDDE90936805809367051092610510
:105C10001092630510926205DECE4B3311F4709240
:105C20006105409161054111D2CE409167055091C7
:105C30006805B9016F5F7F4F7093630560936205DC
:105C4000649EF001659EF00D1124E20FF31FE159EF
:105C5000FA4F8083C0CE6E960FB6F894DEBF0FBEAB
:105C6000CDBFDF91CF911F910F91FF90EF90DF900B
:105C7000CF90BF90AF909F908F907F906F905F90EC
:105C80004F903F902F9008958F929F92AF92BF9226
:105C9000CF92DF92EF92FF920F931F93CF93DF93F8
:105CA00070E5E72E74E0F72E02E417E0C0E1D7E0DC
:105CB000E4E5CE2EE7E0DE2EF70181917F018EDB59
:105CC000882311F177DB4B015C01F60180818111A2
:105CD00003C06091EF0601C061E070E080E090E0F9
:105CE0000E94D1DBF80120813181428153810E94E1
:105CF00004DE9B01AC01C501B4010E9456DA688341
:105D000079838A839B8309C0F80180819181A28174
:105D1000B38188839983AA83BB830C5F1F4F24962A
:105D2000FFEFCF1ADF0A84E5E81684E0F80621F6D3
:105D300086E454DB8823D1F03DDB6B017C0160936A
:105D4000000770930107809302079093030720E0F8
:105D500030E0A9010E9432DD181644F4C0920B0213
:105D6000D0920C02E0920D02F0920E02DF91CF91E0
:105D70001F910F91FF90EF90DF90CF90BF90AF9069
:105D80009F908F90089580DF89E428DB882351F06D
:105D900011DB6093040770930507809306079093C7
:105DA000070708C010920407109205071092060713
:105DB000109207078AE412DB882351F0FBDA609324
:105DC00008077093090780930A0790930B070895BB
:105DD000109208071092090710920A0710920B07F9
:105DE0000895CF92DF92EF92FF92CF93DF93EC0171
:105DF000C0902A07D0902B07E0902C07F0902D0739
:105E0000A7019601688179818A819B810E942FDB9D
:105E100087FF04C0C882D982EA82FB82C0902E0725
:105E2000D0902F07E0903007F0903107A70196013E
:105E30006C817D818E819F810E942FDB87FF04C052
:105E4000CC82DD82EE82FF82C0903207D090330791
:105E5000E0903407F0903507A701960168857985B1
:105E60008A859B850E942FDB87FF04C0C886D98660
:105E7000EA86FB86C0901102D0901202E0901302D5
:105E8000F0901402A7019601688179818A819B8133
:105E90000E9432DD181624F4C882D982EA82FB827D
:105EA000C0901502D0901602E0901702F0901802F0
:105EB000A70196016C817D818E819F810E9432DDD8
:105EC000181624F4CC82DD82EE82FF82C090190283
:105ED000D0901A02E0901B02F0901C02A7019601DC
:105EE000688579858A859B850E9432DD181624F4A1
:105EF000C886D986EA86FB86DF91CF91FF90EF9026
:105F0000DF90CF9008954F925F926F927F928F9221
:105F10009F92AF92BF92CF92DF92EF92FF920F9338
:105F20001F93CF93DF93CDB7DEB728970FB6F894C2
:105F3000DEBF0FBECDBF80E197E053DF0E9427D4C4
:105F400060935B0570935C0580935D0590935E059F
:105F500020911007309111074091120750911307BB
:105F600029833A834B835C83609142077091430796
:105F700080914407909145070E942FDB40901407C1
:105F8000509015076090160770901707209118071A
:105F90003091190740911A0750911B072D833E83BA
:105FA0004F83588781118BC0A301920160914607EE
:105FB0007091470780914807909149070E942FDB15
:105FC00081117DC020E030E040E752E460910B0297
:105FD00070910C0280910D0290910E020E9436DBAE
:105FE0004B015C0182E297E09F938F93FCE1CF2EFF
:105FF000F7E0DF2EED80FE800F811885A30192016E
:1060000069817A818B819C810E9470590F900F90D9
:106010008091100790911107A0911207B09113077A
:106020008093420790934307A0934407B09345079A
:106030008091140790911507A0911607B09117074A
:106040008093460790934707A0934807B09349076A
:106050008091180790911907A0911A07B0911B071A
:1060600080934A0790934B07A0934C07B0934D073A
:1060700080911C0790911D07A0911E07B0911F07EA
:1060800080934E0790934F07A0935007B09351070A
:1060900028960FB6F894DEBF0FBECDBFDF91CF912B
:1060A0001F910F91FF90EF90DF90CF90BF90AF9036
:1060B0009F908F907F906F905F904F900895609128
:1060C000230270912402882777FD8095982F0E94E3
:1060D000D1DB20910B0230910C0240910D025091C6
:1060E0000E020E9404DE20E030E040E752E40E940D
:1060F00036DB20E030E048EC52E470CFAF92BF9244
:10610000CF92DF92EF92FF920F931F93CF93DF9383
:10611000D82F209108073091090740910A07509124
:106120000B07609104077091050780910607909115
:1061300007070E943FDDC62F172F082FF92E609109
:10614000230270912402882777FD8095982F0E9462
:10615000D1DB20910B0230910C0240910D02509145
:106160000E020E9404DE20E030E040E752E40E948C
:1061700036DB20E030E048EC52E40E9436DB209130
:1061800022072F93DF93FF920F931F93CF935B010F
:106190006C01A2E0EA2E01E020E044E057E060E17B
:1061A00077E082E497E00E940D5180911007909172
:1061B0001107A0911207B0911307809342079093A3
:1061C0004307A0934407B09345078091140790912B
:1061D0001507A0911607B091170780934607909373
:1061E0004707A0934807B0934907809118079091FB
:1061F0001907A0911A07B0911B0780934A07909343
:106200004B07A0934C07B0934D0780911C079091CA
:106210001D07A0911E07B0911F0780934E07909312
:106220004F07A0935007B09351070E9427D4609363
:106230005B0570935C0580935D0590935E050F9000
:106240000F900F900F900F900F90DF91CF911F91B3
:106250000F91FF90EF90DF90CF90BF90AF90089597
:10626000F8940E9408915F9A109227078A9A1092D8
:1062700028079FB7F89480910801816080930801F6
:106280009FBF10922907129A60E08CE00E94FFD510
:10629000E2E4FCE08491882341F09091C00095FFF6
:1062A000FCCF8093C6003196F5CFEAE2F6E0849108
:1062B000882341F09091C00095FFFCCF8093C600E9
:1062C0003196F5CF8091C00085FFFCCF8AE08093A6
:1062D000C60081E296E00E94CEAAFFCFCF92DF9265
:1062E000EF92FF920F931F930E9427D400915705BE
:1062F000109158052091590530915A05C0905B05C1
:10630000D0905C05E0905D05F0905E056C197D090C
:106310008E099F09061717072807390728F4012B4C
:10632000022B032B09F09CDF809107029091080259
:10633000A0910902B0910A02892B8A2B8B2B09F1BB
:106340000E9427D400915B0510915C0520915D05AA
:1063500030915E05601B710B820B930B009107025D
:10636000109108022091090230910A0206171707BE
:106370002807390730F49091ED098091EC099817BE
:1063800051F0909BD0CF1F910F91FF90EF90DF9035
:10639000CF900C9437595F9A109227078A9A1092DF
:1063A00028079FB7F89480910801816080930801C5
:1063B0009FBF10922907129AE4CF0E940891809102
:1063C0004D05811138C081E080934D058091F40620
:1063D0009091F506A091F606B091F7068093F0062D
:1063E0009093F106A093F206B093F306E2E4FCE08A
:1063F0008491882341F09091C00095FFFCCF809359
:10640000C6003196F5CFEBEAF5E08491882341F0A0
:106410009091C00095FFFCCF8093C6003196F5CFD8
:106420008091C00085FFFCCF8AE08093C60081EA9E
:1064300095E00C94BFAA089580914D050895CF93DF
:10644000DF93EC018091220780934E0584E50E9442
:10645000EE29811102C080E065C00E94DA290E9405
:10646000A3DB60934E056623B1F3ECE3FCE084917B
:10647000882341F09091C00095FFFCCF8093C60027
:106480003196F5CFC936D10599F034F4C836D10527
:10649000C9F5E1E7F3E015C0CD36D10531F0CA3DCD
:1064A000D10581F5ECE2F3E02AC0E3E4F3E01DC09E
:1064B000EAE5F3E010C09091C00095FFFCCF809317
:1064C000C60081918111F7CF1DC09091C00095FF4A
:1064D000FCCF8093C60081918111F7CF13C09091BA
:1064E000C00095FFFCCF8093C60081918111F7CF4A
:1064F00009C09091C00095FFFCCF8093C6008191A8
:106500008111F7CF40E050E060914E0586EC94E0B9
:106510000E94F9228091C00085FFFCCF8AE0809321
:10652000C60081E0DF91CF9108952F923F924F9264
:106530005F926F927F928F929F92AF92BF92CF9213
:10654000DF92EF92FF920F931F93CF93DF93CDB71C
:10655000DEB7C75FD1090FB6F894DEBF0FBECDBF5F
:1065600087E40E94EE29882311F40C94533D0E9485
:10657000DA290E949EDB6C31710509F4A8C09CF4F5
:106580006230710509F44CC024F477FF41C00C94CB
:106590001B4E6330710509F44AC06430710509F47B
:1065A0004FC00C941B4E6A35710511F40C94E63CF7
:1065B0001CF56D31710509F488C46E31710511F057
:1065C0000C941B4E0E94038E0E949F2380912D02EB
:1065D00090912E02A0912F02B091300280930B0275
:1065E00090930C02A0930D02B0930E020E945824C7
:1065F000E1EBF8E00C94813C6B35710511F40C94DF
:10660000EA3C6C35710511F40C94EF3C0C941B4E74
:1066100080914D05811104C037DB75DC0C94B64FB9
:1066200080914D05811103C0AEDB81E006C08091F1
:106630004D05811105C0A7DB80E060DD0C94B64FED
:1066400083E899E00E94BFAA80E50E94EE29882392
:1066500039F00E94DA290E94A3DB4B015C0103C0E0
:10666000812C912C540183E50E94EE29882361F04E
:106670000E94DA2920E030E04AE754E40E9404DE78
:106680000E94A3DB4B015C010E94038E0E9427D471
:106690006B017C01C80CD91CEA1CFB1C0E9427D48E
:1066A00060935B0570935C0580935D0590935E0538
:1066B0000E9427D46C157D058E059F0510F00C9463
:1066C0001B4E0E9456950ADE0E9457ABF1CF85E41F
:1066D00092E00E94AACE80910B0290910C02A091B0
:1066E0000D02B0910E028093FC069093FD06A093DC
:1066F000FE06B093FF0680912302909124029093AE
:1067000053078093520784E690E09093240280938D
:1067100023020E9427D460935B0570935C058093ED
:106720005D0590935E0581E00E94F68680914207A8
:1067300090914307A0914407B091450780931007BB
:1067400090931107A0931207B09313078091460707
:1067500090914707A0914807B0914907809314078B
:1067600090931507A0931607B093170780914A07D7
:1067700090914B07A0914C07B0914D07809318075B
:1067800090931907A0931A07B0931B0780914E07A7
:1067900090914F07A0915007B091510780931C072B
:1067A00090931D07A0931E07B0931F0710920B0232
:1067B00010920C0210920D0210920E0288E50E94B7
:1067C000EE29882311F090E00AC089E50E94EE29A5
:1067D0008111F9CF8AE50E94EE2991E098279093E4
:1067E0000F0291110C941E4E88E50E94EE29811132
:1067F0000C941E4E80910F0281110C94244E89E559
:106800000E94EE2981110C94244E88E50E94EE2905
:106810008823D1F00E94E329672B682B692BA1F014
:106820000E94DA29209136073091370740913807C6
:10683000509139070E9456DA6093420770934307DC
:10684000809344079093450789E50E94EE298823A9
:10685000D1F00E94E329672B682B692BA1F00E94DD
:10686000DA2920913A0730913B0740913C0750913B
:106870003D070E9456DA609346077093470780935E
:1068800048079093490780910F02882309F4ACC010
:1068900080E090E0A0EFB2E480931007909311079E
:1068A000A0931207B093130780E090E0AEEFB2E43C
:1068B0008093140790931507A0931607B0931707BA
:1068C000EFEFFBE064912CEF6202B0011124882706
:1068D00077FD8095982F0E94D1DB60931807709305
:1068E000190780931A0790931B0780E090E0AAEFA6
:1068F000B5E480930B0290930C02A0930D02B09329
:106900000E0210924A0710924B0710924C071092F9
:106910004D07209146073091470740914807509115
:106920004907609142077091430780914407909115
:106930004507BEE4CB2EB7E0DB2EE12CF12C87011E
:106940000E94EC6380900B0290900C02A0900D02CC
:10695000B0900E02E0901807F090190700911A0706
:1069600010911B07209114073091150740911607CD
:1069700050911707609110077091110780911207CD
:1069800090911307E2E2F7E0FF93EF93ECE1CE2E54
:10699000E7E0DE2E0E9470590E94038E809110075E
:1069A00090911107A0911207B091130780934207AD
:1069B00090934307A0934407B09345078091140731
:1069C00090911507A0911607B0911707809346077D
:1069D00090934707A0934807B093490782E090E05F
:1069E0000E945B250F900F908AE50E94EE29882374
:1069F00009F4F7C080912707882309F4AAC0809181
:106A00002807882309F4A5C0809042079090430787
:106A1000A0904407B090450720E030E0A901C501EF
:106A2000B4010E9456DA6B017C0120E030E0A9013C
:106A30000E9432DD87FDB0C020E030E040E753E443
:106A4000C701B6010E942FDB18160CF4A5C04090B8
:106A5000460750904707609048077090490720E02C
:106A600030E0A901C301B2010E9456DA6B017C013A
:106A700020E030E0A9010E9432DD87FD8DC020E0DA
:106A800030E04EE753E4C701B6010E942FDB181631
:106A90000CF482C010924A0710924B0710924C07D8
:106AA00010924D07FEE4CF2EF7E0DF2EE12CF12C03
:106AB0008701A3019201C501B4010E94EC63EFEFCD
:106AC000FBE064913CEF6302B0011124882777FD5D
:106AD0008095982F0E94D1DB7B018C016093180771
:106AE0007093190780931A0790931B078090370FB4
:106AF0009090380FA090390FB0903A0F80920B020F
:106B000090920C02A0920D02B0920E0220911407F6
:106B100030911507409116075091170760911007A3
:106B2000709111078091120790911307E2E2F7E04C
:106B3000FF93EF93ACE1CA2EA7E0DA2E0E947059C2
:106B40000E94038E82E090E00E945B250F900F90E0
:106B500048C081E799E00E94BFAAECE3FCE0849181
:106B6000882341F09091C00095FFFCCF8093C60030
:106B70003196F5CFEFE5F9E08491882341F09091CB
:106B8000C00095FFFCCF8093C6003196F5CF809171
:106B9000C00085FFFCCF22C08EE499E00E94BFAA0E
:106BA000ECE3FCE08491882341F09091C00095FFD4
:106BB000FCCF8093C6003196F5CFEDE3F9E08491E8
:106BC000882341F09091C00095FFFCCF8093C600D0
:106BD0003196F5CF8091C00085FFFCCF8AE080938D
:106BE000C6008AE50E94EE298823D1F00E94E3299D
:106BF000672B682B692BA1F00E94DA2920913E07B0
:106C000030913F0740914007509141070E9456DA6A
:106C100060934A0770934B0780934C0790934D07FE
:106C200080910F02811105C08AE50E94EE29882318
:106C300039F1C0902307D0902407E0902507F09009
:106C4000260720E030E0A901C701B6010E942FDB32
:106C500087FD02C00C942A4EA701960160914A0755
:106C600070914B0780914C0790914D070E9456DA26
:106C700060934A0770934B0780934C0790934D079E
:106C8000E0904A07F0904B0700914C0710914D0798
:106C90002091460730914707409148075091490796
:106CA0006091420770914307809144079091450796
:106CB000EEE4CE2EE7E0DE2E0E94EC6380E00E9440
:106CC000F6868091FC069091FD06A091FE06B0919B
:106CD000FF0680930B0290930C02A0930D02B093D9
:106CE0000E02809152079091530790932402809353
:106CF00023020E9427D460935B0570935C05809308
:106D00005D0590935E050E94EF86EAE3F9E08491C9
:106D1000882341F09091C00095FFFCCF8093C6007E
:106D20003196F5CF40914207509143076091440757
:106D30007091450722E030E086EC94E00E949823B1
:106D4000E6E3F9E08491882341F09091C00095FF3B
:106D5000FCCF8093C6003196F5CF40914607509105
:106D60004707609148077091490722E030E086ECC0
:106D700094E00E949823E2E3F9E08491882341F0B3
:106D80009091C00095FFFCCF8093C6003196F5CF5F
:106D900040914A0750914B0760914C0770914D0705
:106DA00022E030E086EC94E00E949823EEE2F9E0E5
:106DB0008491882341F09091C00095FFFCCF80938F
:106DC000C6003196F5CF40914E0750914F07609124
:106DD00050077091510722E030E086EC94E00E9469
:106DE0009823E3E2F9E08491882341F09091C00078
:106DF00095FFFCCF8093C6003196F5CF0E945D8E43
:106E00000E94D1DB20911F0F3091200F4091210F64
:106E10005091220F0E9436DBAB01BC0122E030E032
:106E200086EC94E00E949823EFE1F9E084918823B6
:106E300041F09091C00095FFFCCF8093C600319641
:106E4000F5CF81E00E945D8E0E94D1DB2091230F5F
:106E50003091240F4091250F5091260F0E9436DB70
:106E6000AB01BC0122E030E086EC94E00E94982364
:106E7000EBE1F9E08491882341F09091C00095FF07
:106E8000FCCF8093C6003196F5CF82E00E945D8EE4
:106E90000E94D1DB2091270F3091280F4091290FBC
:106EA00050912A0F0E9436DBAB01BC0122E030E09A
:106EB00086EC94E00E9498238091C00085FFFCCF6F
:106EC0008AE08093C6000C941B4E8091270788238C
:106ED00021F080912807811127C089E099E00E9464
:106EE000BFAAECE3FCE08491882341F09091C000BC
:106EF00095FFFCCF8093C6003196F5CFE7EFF8E021
:106F00008491882341F09091C00095FFFCCF80933D
:106F1000C6003196F5CF8091C00085FFFCCF8AE096
:106F20008093C6000C941B4E0E94038E85E492E071
:106F30000E94AACECE0187559F4F0E947563C75508
:106F4000DF4F688179818A819B81C95AD0406093E3
:106F50004207709343078093440790934507C355B6
:106F6000DF4F288139814A815B81CD5AD0402093FF
:106F70004607309347074093480750934907CF543B
:106F8000DF4FE880F9800A811B81C15BD040E0922D
:106F90004A07F0924B0700934C0710934D07BEE44D
:106FA000CB2EB7E0DB2E0E94EC630E949F238091E2
:106FB0002D0290912E02A0912F02B0913002809369
:106FC0000B0290930C02A0930D02B0930E02CB51D2
:106FD000DF4F19821882C55ED04084E190E0CD5128
:106FE000DF4F99838883C35ED040C451DF4F19823D
:106FF0001882CC5ED040AFE5B0E0C851DF4FB98316
:10700000A883C85ED040EFE0F0E0CF51DF4FF983B6
:10701000E883C15ED040C951DF4F1882C75ED040BF
:10702000CE010196CB51DF4FA881B981C55ED0401A
:107030008A0F9B1FC152DF4F99838883CF5DD04059
:10704000C451DF4FE881F981CC5ED040C651DF4F9B
:10705000F983E883CA5ED040212C312CCD51DF4F1B
:1070600088819981C35ED040AA2797FDA095BA2F49
:10707000C251DF4F88839983AA83BB83CE5ED04001
:10708000CB51DF4FA881B981C55ED040EDE6F0E07D
:10709000EC0FFD1FAE0FBF1FCE50DF4FB983A8838B
:1070A000C25FD040C651DF4F28813981CA5ED040CF
:1070B000232B89F020E030E040EA50E460914A0759
:1070C00070914B0780914C0790914D070E9456DAC2
:1070D0006B017C0106C0C12CD12CA0E7EA2EA1E4F3
:1070E000FA2EC251DF4F688179818A819B81CE5E01
:1070F000D0400E94D1DB4B015C01CF51DF4FA88112
:10710000B981C15ED040BD01882777FD8095982F59
:107110000E94D1DB2B013C012091460730914707AB
:107120004091480750914907609142077091430789
:107130008091440790914507870176010E94F023D2
:10714000E0904A07F0904B0700914C0710914D07D3
:10715000A5019401C301B2010E94F0230E945824AA
:10716000C0904A07D0904B07E0904C07F0904D0735
:10717000E6E6F6E08491882341F09091C00095FF07
:10718000FCCF8093C6003196F5CFE1E6F6E084911E
:10719000882341F09091C00095FFFCCF8093C600FA
:1071A0003196F5CF22E030E0B301A20186EC94E005
:1071B0000E949823ECE5F6E08491882341F09091B9
:1071C000C00095FFFCCF8093C6003196F5CF22E03A
:1071D00030E0B501A40186EC94E00E949823E7E535
:1071E000F6E08491882341F09091C00095FFFCCF98
:1071F0008093C6003196F5CF22E030E0B701A601BA
:1072000086EC94E00E949823E5E5F6E084918823DB
:1072100041F09091C00095FFFCCF8093C60031965D
:10722000F5CFCE50DF4FE881F981C25FD040E20D4B
:10723000F31DC082D182E282F382C152DF4FA88166
:10724000B981CF5DD0404D925D926D927D92C152D9
:10725000DF4FB983A883CF5DD040FD0180A291A20A
:10726000A2A2B3A2EC5BFF4F80E090E0A0E8BFE3F6
:1072700080839183A283B383C651DF4FA881B981F4
:10728000CA5ED0401196C651DF4FB983A883CA5E4B
:10729000D040CF51DF4FE881F981C15ED040C85165
:1072A000DF4F28813981C85ED040E20FF31FCF51F4
:1072B000DF4FF983E883C15ED04034E0230E311CF8
:1072C0008CE02816310409F0EDCEC451DF4FA881BF
:1072D000B981CC5ED0401396C451DF4FB983A883E7
:1072E000CC5ED040CD51DF4FE881F981C35ED04004
:1072F000E759FF4FCD51DF4FF983E883C35ED0409C
:10730000EF34F14009F442C0C951DF4FF881C75E44
:10731000D040FF23B1F02FE530E0C851DF4F398373
:107320002883C85ED0408FE090E0CF51DF4F998333
:107330008883C15ED040C951DF4F1882C75ED040FC
:1073400016C0A1EABFEFC851DF4FB983A883C85E5A
:10735000D040EDECF0E0CF51DF4FF983E883C15E20
:10736000D040F1E0C951DF4FF883C75ED040CB5128
:10737000DF4F28813981C55ED040245F3F4FCB511C
:10738000DF4F39832883C55ED0404ACE0E94CA238E
:107390009E0123593F4FAE014F5F5F4F63E070E0A6
:1073A00089E090E00E942576C152DF4F998388835F
:1073B000CF5DD040E1EEF8E08491882341F09091D8
:1073C000C00095FFFCCF8093C6003196F5CFC15227
:1073D000DF4FA881B981CF5DD0404D915D916D9116
:1073E0007C9122E030E086EC94E00E949823ECED62
:1073F000F8E08491882341F09091C00095FFFCCF84
:107400008093C6003196F5CFC152DF4FE881F981F4
:10741000CF5DD040448155816681778122E030E0A4
:1074200086EC94E00E949823E7EDF8E084918823AD
:1074300041F09091C00095FFFCCF8093C60031963B
:10744000F5CFC152DF4FA881B981CF5DD0401896EA
:107450004D915D916D917C911B9722E030E086EC1F
:1074600094E00E9498238091C00085FFFCCF8AE0C1
:107470008093C600C152DF4FE881F981CF5DD040D3
:107480000481158126813781305840815181628184
:10749000738170583E01FDE96F0E711CC12CD12C17
:1074A000F0E8EF2EFFE3FF2EC3010E945CCC67E9FA
:1074B00073E0C3010E94D9CDD301CC901196DC902A
:1074C00011971296EC9012971396FC9013971496BE
:1074D0000C91149715961C91159716962C9116974A
:1074E00017963C91179718964C91189719965C919E
:1074F00019971A966C911A971B967C91CE01875416
:107500009F4F0E94D4CE84E2FE01E754FF4FA5E4D2
:10751000B2E001900D928A95E1F7FE01EF56FF4F20
:10752000C352DF4FF983E883CD5DD040CF010E9485
:107530007563CF56DF4F88809980AA80BB80C15980
:10754000D0408092420790924307A0924407B092A5
:107550004507CB56DF4F288039804A805B80C5596C
:10756000D0402092460730924707409248075092F9
:107570004907C0902307D0902407E0902507F0909A
:10758000260720E030E0A901C701B6010E942FDBE9
:1075900087FD04C0F7FAF094F7F8F094C0924A0718
:1075A000D0924B07E0924C07F0924D07E0904A07CB
:1075B000F0904B0700914C0710914D078EE4C82EB8
:1075C00087E0D82EA2019101C501B4010E94EC63AD
:1075D000C152DF4F88819981CF5DD0400E94FFDF8B
:1075E0000E94038E82E00E945D8E0E94D1DB20917A
:1075F000270F3091280F4091290F50912A0F0E9498
:1076000036DB6B017C018E010B541F4F20E030E014
:10761000A9016091420770914307809144079091BE
:1076200045070E9456DAD8016D937D938D939C9304
:10763000139720E030E0A901609146077091470759
:1076400080914807909149070E9456DAF3016083C0
:1076500071838283938380914A0790914B07A09115
:107660004C07B0914D07CF56DF4F88839983AA838B
:10767000BB83C159D040C252DF4FF881CE5DD040AC
:10768000FF93C352DF4F2881CD5DD0402F937F926F
:107690006F921F930F938DB79EB784970FB6F89490
:1076A0009EBF0FBE8DBFADB7BEB7119684E2E5E4B5
:1076B000F2E001900D928A95E1F70E943DCEA7017C
:1076C0009601CF56DF4F688179818A819B81C159AC
:1076D000D0400E9455DA20914A0730914B074091E3
:1076E0004C0750914D070E9456DA7B018C01609344
:1076F0004A0770934B0780934C0790934D070FB642
:10770000F894DEBF0FBECDBF2091460730914707EA
:107710004091480750914907609142077091430793
:107720008091440790914507EEE4CE2EE7E0DE2EEF
:107730000E94EC63E4EDF8E08491882341F090919D
:10774000C00095FFFCCF8093C6003196F5CF4091E5
:10775000420750914307609144077091450722E02A
:1077600030E086EC94E00E949823E0EDF8E084910C
:10777000882341F09091C00095FFFCCF8093C60014
:107780003196F5CF409146075091470760914807E1
:107790007091490722E030E086EC94E00E94982343
:1077A000ECECF8E08491882341F09091C00095FFC3
:1077B000FCCF8093C6003196F5CF40914A07509197
:1077C0004B0760914C0770914D0722E030E086EC4A
:1077D00094E00E949823E8ECF8E08491882341F03B
:1077E0009091C00095FFFCCF8093C6003196F5CFF5
:1077F00040914E0750914F0760915007709151078B
:1078000022E030E086EC94E00E949823EDEBF8E073
:107810008491882341F09091C00095FFFCCF809324
:10782000C6003196F5CF0E945D8E0E94D1DB20917B
:107830001F0F3091200F4091210F5091220F0E9475
:1078400036DBAB01BC0122E030E086EC94E00E9424
:107850009823E9EBF8E08491882341F09091C000EF
:1078600095FFFCCF8093C6003196F5CF81E00E9452
:107870005D8E0E94D1DB2091230F3091240F409127
:10788000250F5091260F0E9436DBAB01BC0122E090
:1078900030E086EC94E00E949823E5EBF8E08491D8
:1078A000882341F09091C00095FFFCCF8093C600E3
:1078B0003196F5CF82E00E945D8E0E94D1DB20914F
:1078C000270F3091280F4091290F50912A0F0E94C5
:1078D00036DBAB01BC0122E030E086EC94E00E9494
:1078E00098238091C00085FFFCCF8AE08093C6007A
:1078F0000C941B4E9091C00095FFFCCF8093C60066
:10790000319684918111F6CFECEAF8E084918823D6
:1079100041F09091C00095FFFCCF8093C600319656
:10792000F5CF409142075091430760914407709111
:10793000450722E030E086EC94E00E949823E7EAD5
:10794000F8E08491882341F09091C00095FFFCCF2E
:107950008093C6003196F5CF409146075091470776
:10796000609148077091490722E030E086EC94E08E
:107970000E949823E2EAF8E08491882341F09091F4
:10798000C00095FFFCCF8093C6003196F5CF4091A3
:107990004A0750914B0760914C0770914D0722E0C8
:1079A00030E086EC94E00E949823E0EAF8E08491CD
:1079B000882341F09091C00095FFFCCF8093C600D2
:1079C0003196F5CF0E94CA230C941B4E1092EF06FD
:1079D0000C941B4E81E08093EF060C941B4E85E4C3
:1079E0000E94EE29811102C00E94038EF0E56F2EE5
:1079F000F4E07F2EA6E38A2EA7E09A2EB2E4AB2E07
:107A0000B7E0BB2E512CF30181913F010E94EE297A
:107A10008823E9F1F3E05F120DC00E94DA29D50155
:107A20006D937D938D939C9313978EE497E00E94C2
:107A3000CD642DC00E94DA29F40120813181428178
:107A400053810E9456DAD5016D937D938D939C935B
:107A50001397E0904A07F0904B0700914C07109164
:107A60004D072091460730914707409148075091B4
:107A700049076091420770914307809144079091B4
:107A80004507EEE4CE2EE7E0DE2E0E94EC63539431
:107A9000B4E08B0E911CE4E0AE0EB11CF4E05F127A
:107AA000B2CF0C941B4E8DE40E94EE29882311F472
:107AB0000C944A4D0E94DA290E949EDB63377105BF
:107AC00011F40C9471450CF092C06F31710509F4FA
:107AD0004CC3A4F56631710509F4EBC1BCF4613106
:107AE000710509F4A1C134F46230710508F441C193
:107AF0000C941B4E6431710509F4A7C10CF0D3C17D
:107B00006231710509F422C70C941B4E6A3171056C
:107B100009F404C23CF46831710509F4E9C10CF4BC
:107B2000CEC1F6C16C31710509F40CC20CF404C26B
:107B30006E31710509F43CC20C941B4E653571051C
:107B400009F43CC7ECF46135710509F4DDC674F441
:107B50006A32710509F490C36035710509F4C7C62E
:107B60006032710511F00C941B4E61C263357105D2
:107B700009F4E7C60CF0EAC6109257070C941B4EA6
:107B80006A36710509F483C6FCF46836710509F498
:107B90009EC30CF0CBC36C35710511F00C941B4ED9
:107BA00020E534E0C152DF4F39832883CF5DD040D8
:107BB0000FE11FE02FE2822E2FE0922E33EEA32E54
:107BC0003EE0B32E312C73C76D36710509F4BBC48A
:107BD0006237710509F4A9C76B36710511F00C9471
:107BE0001B4E10922107109220070C941B4E623EF0
:107BF000710511F40C9484480CF05DC0683C71056B
:107C000011F40C94FA462CF56837710511F40C94B4
:107C100074466CF46537710509F472C767377105EE
:107C200011F00C941B4EE3EAF3E00C947E466C38A2
:107C3000710509F46AC36E3B710509F424C56937FF
:107C4000710511F00C941B4E81E00E94F6860C9495
:107C50001B4E6D3C710511F40C94F147ACF46B3C78
:107C6000710511F40C94B54714F00C94D147693C9C
:107C7000710511F00C941B4E00E514E09FE0E92E15
:107C80009FE0F92E0C949A476C3D710511F40C9409
:107C900066486D3D710511F40C9475486E3C710594
:107CA00011F00C941B4E00E514E0B6E3EB2EB7E0A8
:107CB000FB2E0C945748663F21E0720711F40C9498
:107CC000F7494CF56F3281E0780711F40C94B9490B
:107CD00084F46D32A1E07A0711F40C94E54814F0B5
:107CE0000C94AB496C32714011F40C94AF480C9475
:107CF0001B4E643FF1E07F0711F40C94F14914F03E
:107D00000C94F4496039714011F00C941B4E0E94A0
:107D1000038E0C941B4E693482E0780711F40C94A6
:107D20006F4AACF46533A2E07A0711F40C94FA4977
:107D30006F33B2E07B0711F40C94334A673F714014
:107D400011F00C941B4E0E944A1C0C941B4E603A7E
:107D5000F3E07F0709F4D5C1673E23E0720711F411
:107D60000C94334D6835724011F00C941B4E0C94FA
:107D7000864A8FE898E00E94BFAA80E50E94EE291B
:107D8000882339F00E94DA290E94A3DB6B017C0171
:107D900003C0C12CD12C760183E50E94EE298823F3
:107DA00061F00E94DA2920E030E04AE754E40E94C2
:107DB00004DE0E94A3DB6B017C010E94038E0E9403
:107DC00027D460935B0570935C0580935D05909369
:107DD0005E05C114D104E104F104A9F00E9427D486
:107DE0004B015C018C0C9D1CAE1CBF1C0E9427D457
:107DF000681579058A059B0588F40E9418AC8111E5
:107E00000DC00C94384E0E9418AC811107C00E941E
:107E100056950E946E310E9457ABF5CF80E898E0EE
:107E20000E94BFAA0C941B4E87E798E00E94BFAA4D
:107E30005F988A989FB7F894809108018E7F80930D
:107E400008019FBF12980C941B4EE7E6F8E084915E
:107E5000882341F09091C00095FFFCCF8093C6002D
:107E60003196F5CF8091C00085FFFCCF8AE08093EA
:107E7000C6008AE597E00E945D11E9E5F8E084918B
:107E8000882341F09091C00095FFFCCF8093C600FD
:107E90003196F5CF8091C00085FFFCCF8AE08093BA
:107EA000C6000C941B4E8AE597E00E94B3110C9417
:107EB0001B4E8AE597E00E9479120C941B4E0091AC
:107EC0005F05109160050C5F1F4F6AE270E0C8010A
:107ED0000E94A9E3009719F0FC013197108221E07C
:107EE00041E0B8018AE597E00E94E8120C941B4E2D
:107EF0008AE597E00E947D120E9427D46093530583
:107F00007093540580935505909356050C941B4E21
:107F10008AE597E00E9484120C941B4E80915D07C5
:107F2000882311F40C941B4E83E50E94EE298111E5
:107F30000C94404E0C941B4E8AE597E00E94331738
:107F40000C941B4E80915F05909160056AE270E091
:107F500004960E94A9E38C010097E1F02091690545
:107F600030916A0540E6429FC001439F900D112465
:107F70006EE470E081599A4F0E94A9E360E270E0DC
:107F80000E94A9E301969093600580935F05F80134
:107F90003197108260915F05709160056C5F7F4F33
:107FA00021E040E08AE597E00E94E8120C941B4E25
:107FB00080915D07882311F40C941B4E60E08AE5E4
:107FC00097E00E94ED1880915F05909160056AE24C
:107FD00070E004960E94A9E38C010097E1F02091E3
:107FE000690530916A0540E6429FC001439F900DAC
:107FF00011246EE470E081599A4F0E94A9E360E277
:1080000070E00E94A9E301969093600580935F055C
:10801000F8013197108260915F05709160056C5F87
:108020007F4F8AE597E00E94FB150C941B4E8091D0
:108030005C0781110E94038E00915F05109160051D
:108040000C5F1F4F6AE270E0C8010E94A9E37C0147
:1080500061E270E0C8010E94A9E3009719F08C0169
:108060000F5F1F4FE114F10419F0F70131971082EF
:1080700080E50E94EE29F82E20915F053091600581
:108080000217130708F4F12C80915D07882311F47F
:108090000C941B4E21E02F2541E0B8018AE597E0C2
:1080A0000E94E81283E50E94EE298823B9F020910E
:1080B0005F05309160052017310780F40E94E329A5
:1080C000AB01BC014093DD095093DE096093DF09E9
:1080D0007093E00988E299E00E944D7C8AE597E080
:1080E0000E947D12F1100C941B4E0E9427D46093C5
:1080F00053057093540580935505909356050C9441
:108100001B4E80915F05909160056AE270E00596D4
:108110000E94A9E38C010097E1F02091690530915C
:108120006A0540E6429FC001439F900D11246EE412
:1081300070E081599A4F0E94A9E360E270E00E94CA
:10814000A9E301969093600580935F05F80131974C
:10815000108260915F05709160056B5F7F4F8AE5CB
:1081600097E00E94F6150C941B4E0E9427D4609352
:108170004F057093500580935105909352050091DF
:108180005305109154052091550530915605601BFB
:10819000710B820B930B28EE33E040E050E00E941D
:1081A00000DFCA01B9012CE330E040E050E00E945A
:1081B00000DF7F936F933F932F938AE498E09F9320
:1081C0008F93CE0101969F938F930E94D8E3ECE3A7
:1081D000FCE084910FB6F894DEBF0FBECDBF8823BC
:1081E00049F09091C00095FFFCCF8093C600319676
:1081F0008491F5CFFE0131968191882339F09091D9
:10820000C00095FFFCCF8093C600F6CF8091C000E0
:1082100085FFFCCF8AE08093C600CE0101960E94C4
:10822000B0AA8091BE0E882311F40C941B4E1092BC
:10823000BE0E0091220710E0000F111F05511E4EC7
:10824000F80160817181882777FD8095982F0E94C1
:10825000D1DB20913D0230913E0240913F0250918E
:1082600040020E9432DD181614F00C941B4ED80107
:108270001D921C920C941B4E83E50E94EE298823CC
:1082800011F40C941B4E0E94DA296B017C0180E5ED
:108290000E94EE29882351F0C701B6010E949EDB9F
:1082A0006F3F710509F010F40C94514E6DE070E0D1
:1082B00020E0E22FEE0FFF0BE85EFB4F8081918103
:1082C0008617970711F40C941B4E2F5FF2CF88E6A8
:1082D00090E00E941F3281110C941B4E83E50E9496
:1082E000EE29882371F000914E050E94DA2910E0F2
:1082F000000F111F05511E4E0E949EDBF801718375
:1083000060830E9407910C941B4E83E50E94EE2926
:10831000882311F40C941B4E0E94DA290E949EDBE4
:108320007093E6116093E5110C941B4E89E690E082
:108330000E941F3281110C941B4EE4E4F8E08491FA
:10834000882341F09091C00095FFFCCF8093C60038
:108350003196F5CFE0914E0524E0E29FF001112423
:10836000E152FE4E408151816281738121E030E013
:1083700086EC94E00E949823E1E4F8E0849188235D
:1083800041F09091C00095FFFCCF8093C6003196DC
:10839000F5CFE0914E05F0E0EE0FFF1FE551FE4EE8
:1083A00060817181882777FD8095982F0E94D1DBAD
:1083B000AB01BC0121E030E086EC94E00E94982300
:1083C000EDE3F8E08491882341F09091C00095FF9F
:1083D000FCCF8093C6003196F5CF4091D9115091D2
:1083E000DA116091DB117091DC1121E030E086EC54
:1083F00094E00E949823EAE3F8E08491882341F016
:108400009091C00095FFFCCF8093C6003196F5CFC8
:108410006091E5117091E611882777FD8095982F7E
:108420000E94D1DBAB01BC0121E030E086EC94E09E
:108430000E949823E7E3F8E08491882341F090912B
:10844000C00095FFFCCF8093C6003196F5CF4AE07F
:1084500050E060E070E086EC94E00E94C222E5E328
:10846000F8E08491882341F09091C00095FFFCCF03
:108470008093C6003196F5CF4091DF115091E01105
:108480006091E1117091E21121E030E086EC94E01E
:108490000E949823E2E3F8E08491882341F09091D0
:1084A000C00095FFFCCF8093C6003196F5CF609158
:1084B000EB117091EC11882777FD8095982F0E9421
:1084C000D1DBAB01BC0121E030E086EC94E00E94FE
:1084D0009823EEE2F8E08491882341F09091C00067
:1084E00095FFFCCF8093C6003196F5CF80914E0565
:1084F00090E00E945B904AE050E0BC0186EC94E082
:108500000E94C222E9E2F8E08491882341F0909130
:10851000C00095FFFCCF8093C6003196F5CF8FEF5A
:108520009FEF0E945B904AE050E0BC0186EC94E033
:108530000E94C2228091C00085FFFCCF8AE0809318
:10854000C6000C94B64F8DE690E00E941F32811158
:108550000C941B4E8EE198E00E94BFAA1092BE0EB2
:1085600083E50E94EE29882391F000914E050E9438
:10857000DA2910E0000F111F05511E4E0E949EDBEC
:10858000D8016D937C9381E08093060215C082E54B
:108590000E94EE29882381F000914E050E94DA297D
:1085A00010E0000F111F05511E4E0E949EDBF801C6
:1085B000718360831092060283E50E94EE2988236E
:1085C00051F00E94DA2960933D0270933E0280933D
:1085D0003F029093400282E40E94EE29882351F0EA
:1085E0000E94DA2960934102709342028093430211
:1085F0009093440286E40E94EE29882369F00E9449
:10860000DA296093390270933A0280933B02909387
:108610003C0281E08093BE0E0E9407910E9427D405
:108620004B015C0100914E0510E0F801EE0FFF1FB9
:10863000E551FE4E60817181882777FD8095982FE6
:108640000E94D1DBF801EE0FFF1FEE0FFF1FE1527A
:10865000FE4E11E020813181428153810E9432DD42
:1086600018160CF010E010934C05CC24CA94DC2CA6
:10867000760138EE432E33E0532E612C712C4AE004
:10868000342E0C94B44E88EF97E00E94BFAA83E585
:108690000E94EE29882361F00E94DA290E949EDB65
:1086A0007093E6116093E51181E0809306020FC09C
:1086B00082E50E94EE29882351F00E94DA290E9467
:1086C0009EDB7093E6116093E511109206020E9402
:1086D00027D44B015C016091E5117091E611882768
:1086E00077FD8095982F0E94D1DB11E02091D91160
:1086F0003091DA114091DB115091DC110E9432DD92
:1087000018160CF010E010934C0505EF17E041EF40
:10871000E42E47E0F42E5DEEC52E57E0D52E6AE03C
:10872000762E80914C056091E5117091E6118823B9
:1087300009F486C0882777FD8095982F0E94D1DBA9
:108740002091D9113091DA114091DB115091DC1157
:108750000E9432DD18160CF08AC00E9427D46819D6
:1087600079098A099B09693E73408105910508F4DE
:1087700060C0E091220724E0E29FF0011124E15261
:10878000FE4E4081518162817381F8018491E5EF51
:10879000F7E0882349F09091C00095FFFCCF8093CB
:1087A000C60031968491F5CF22E030E086EC94E06B
:1087B0000E949823F7018491E1EFF7E0882349F0C4
:1087C0009091C00095FFFCCF8093C60031968491B4
:1087D000F5CF6091220770E04AE050E086EC94E02B
:1087E0000E94C222F6018491EDEEF7E0882349F061
:1087F0009091C00095FFFCCF8093C6003196849184
:10880000F5CF4091D9115091DA116091DB1170913F
:10881000DC1121E030E086EC94E00E949823809106
:10882000C00085FFFCCF7092C6000E9427D44B0188
:108830005C010E9456950E946E310E9457AB71CF29
:10884000882777FD8095982F0E94D1DB2091D91140
:108850003091DA114091DB115091DC110E942FDB35
:1088600087FF05C080910602882309F476CF83EE46
:1088700097E00E94BFAA0E9427D460935B05709383
:108880005C0580935D0590935E050C941B4E83E51B
:108890000E94EE29882319F10E94DA2920E030E0B5
:1088A000A9010E942FDB87FD0FC00E94DA2920E07A
:1088B00030E04FE753E40E9432DD181644F00E9486
:1088C000DA290E949EDB05C060E070E002C06FEF15
:1088D00070E070932107609320070C941B4E8FEF7C
:1088E00090E090932107809320070C941B4E269ACA
:1088F0002E9881E0809310028FEC97E00E94BFAA2F
:108900000E9457AB0C941B4E0E9408910E94038E4C
:10891000129A0E947E8E109221071092200768EE14
:1089200073E080E090E00E9456D4269A2E9A10922E
:1089300010028DEB97E00E94BFAA0E9457AB0C94E7
:108940001B4E81E0809357070C941B4E83E50E94D9
:10895000EE298823A1F00E94DA2920E030E04AE7DE
:1089600054E40E9404DE0E94A3DB6093070270932C
:1089700008028093090290930A020C941B4E88E52A
:108980000E94EE2981110C948D4F89E50E94EE29F9
:1089900081110C948D4F8AE50E94EE2981110C946F
:1089A0008D4F85E40E94EE2981110C948D4F0E9419
:1089B000038E129A0E947E8E0C941B4E83E50E94B9
:1089C000EE290E94DA2920E030E04AE754E40E94D0
:1089D00004DE0E94A3DB60935705709358058093D3
:1089E000590590935A050C941B4EB3E03B1271C08D
:1089F0000E94DA296B017C0120E030E040EA51E47A
:108A00000E942FDB87FF3FC0A7019601F80160811C
:108A10007181828193810E9436DB2B013C019B0195
:108A2000AC016091F70E7091F80E8091F90E909163
:108A3000FA0E0E9404DE6093F70E7093F80E809396
:108A4000F90E9093FA0EA3019201D4016D917D91DC
:108A50008D919C910E9404DEF40160837183828376
:108A60009383D5016D917D918D919C910E94CFDB77
:108A7000A30192010E9404DE0E94A3DBF501608342
:108A8000718382839383D801CD92DD92ED92FC9223
:108A9000139733940C5F1F4FF4E08F0E911C24E06A
:108AA000A20EB11C34E0331611F40C941B4EC152CB
:108AB000DF4FA881B981CF5DD0408D91C152DF4F8A
:108AC000B983A883CF5DD0400E94EE29882309F3A3
:108AD0008CCF0E94DA29F8016083718382839383AB
:108AE000D8CFEAEEF6E08491882311F40C941B4E63
:108AF0009091C00095FFFCCF8093C6003196F3CFD4
:108B000000915F05109160050B5F1F4F6AE270E0F6
:108B1000C8010E94A9E3009719F0FC013197108267
:108B2000C8010E94B0AA0C941B4EE7EEF6E08491B7
:108B3000882341F09091C00095FFFCCF8093C60040
:108B40003196F5CF40914207509143076091440719
:108B50007091450722E030E086EC94E00E94982373
:108B6000E3EEF6E08491882341F09091C00095FFF8
:108B7000FCCF8093C6003196F5CF409146075091C7
:108B80004707609148077091490722E030E086EC82
:108B900094E00E949823EFEDF6E08491882341F061
:108BA0009091C00095FFFCCF8093C6003196F5CF21
:108BB00040914A0750914B0760914C0770914D07C7
:108BC00022E030E086EC94E00E949823EBEDF6E0A2
:108BD0008491882341F09091C00095FFFCCF809351
:108BE000C6003196F5CF40914E0750914F076091E6
:108BF00050077091510722E030E086EC94E00E942B
:108C00009823E0EDF6E08491882341F09091C00034
:108C100095FFFCCF8093C6003196F5CF0E945D8E04
:108C20000E94D1DB20911F0F3091200F4091210F26
:108C30005091220F0E9436DBAB01BC0122E030E0F4
:108C400086EC94E00E949823ECECF6E08491882373
:108C500041F09091C00095FFFCCF8093C600319603
:108C6000F5CF81E00E945D8E0E94D1DB2091230F21
:108C70003091240F4091250F5091260F0E9436DB32
:108C8000AB01BC0122E030E086EC94E00E94982326
:108C9000E8ECF6E08491882341F09091C00095FFC4
:108CA000FCCF8093C6003196F5CF82E00E945D8EA6
:108CB0000E94D1DB2091270F3091280F4091290F7E
:108CC00050912A0F0E9436DBAB01BC0122E030E05C
:108CD00086EC94E00E9498238091C00085FFFCCF31
:108CE0008AE08093C600A7C780E00E94F686A3C7EB
:108CF0009091C00095FFFCCF8093C60081918111B7
:108D0000F7CF8091C00085FFFCCF8AE08093C6003A
:108D1000E0ECF6E08491882341F09091C00095FF4B
:108D2000FCCF8093C6003196F5CF659B03C0E8E881
:108D3000F3E009C0E2E9F3E006C09091C00095FFBE
:108D4000FCCF8093C60081918111F7CF8091C00044
:108D500085FFFCCF8AE08093C600E8EBF6E08491C3
:108D6000882341F09091C00095FFFCCF8093C6000E
:108D70003196F5CF8091030181FF03C0E8E8F3E06D
:108D800009C0E2E9F3E006C09091C00095FFFCCF76
:108D90008093C60081918111F7CF8091C00085FF3B
:108DA000FCCF8AE08093C600E0EBF6E08491882354
:108DB00041F09091C00095FFFCCF8093C6003196A2
:108DC000F5CF4B9903C0E8E8F3E009C0E2E9F3E02E
:108DD00006C09091C00095FFFCCF8093C6008191A2
:108DE0008111F7CF8091C00085FFFCCF8AE080938E
:108DF000C60021C784E40E94EE29882309F41BC71A
:108E00000E94DA2920E030E040E05FE30E9404DEC7
:108E10006B017C0120E030E0A9010E942FDB882358
:108E200079F0A7019601C701B6010E9404DE2BED7F
:108E30003FE049E450E40E9404DE9B01AC0104C021
:108E400020E030E040E85FE30091220700934E0508
:108E500084E5CC50DF4F2883C45FD040CB50DF4F38
:108E60003883C55FD040CA50DF4F4883C65FD040CB
:108E7000C950DF4F5883C75FD0400E94EE29CC50C5
:108E8000DF4F2881C45FD040CB50DF4F3881C55FB2
:108E9000D040CA50DF4F4881C65FD040C950DF4F35
:108EA0005881C75FD040882391F10E94DA290E943F
:108EB000A3DB60934E05611109C040E050E0609172
:108EC0004E0586EC94E00E94F92219C0ECE3FCE028
:108ED0008491882341F09091C00095FFFCCF80934E
:108EE000C6003196F5CFEEEBF3E08191882329F3AC
:108EF0009091C00095FFFCCF8093C600F6CF809183
:108F0000C00085FFFCCF8AE08093C60094C684E051
:108F1000089F80011124035E1D4F60E070E080E82F
:108F20009FE30E9436DBD8016D937D938D939C93D4
:108F3000139781C6F80181918F010E94EE29882341
:108F400051F00E94DA290E94A3DBD7016D937D9333
:108F50008D939C931397B4E0EB0EF11CE4E0043581
:108F60001E0741F70E94FA6466C600E514E08FE22E
:108F7000E82E8FE0F82ED8018D918D010E94EE2908
:108F8000882339F00E94DA29F70160837183828394
:108F90009383F4E0EF0EF11C24E00435120759F737
:108FA0004AC683E50E94EE29882351F00E94DA29FF
:108FB0006093070F7093080F8093090F90930A0F27
:108FC00084E50E94EE29882309F435C60E94DA2937
:108FD0006093030F7093040F8093050F9093060F17
:108FE0002AC683E50E94EE29882351F00E94DA29DF
:108FF00060930B0F70930C0F80930D0F90930E0FD7
:1090000084E50E94EE29882351F00E94DA296093BA
:10901000F30E7093F40E8093F50E9093F60E82E4A7
:109020000E94EE29882361F00E94DA290E94A3DBC6
:1090300060933F0F7093400F8093410F9093420FC6
:1090400088E50E94EE29882351F00E94DA29609376
:10905000FF0E7093000F8093010F9093020F8AE52B
:109060000E94EE29882351F00E94DA296093FB0EBA
:109070007093FC0E8093FD0E9093FE0E85E40E948B
:10908000EE29882309F4D7C50E94DA296093F70EE8
:109090007093F80E8093F90E9093FA0ECCC5F4E01D
:1090A000EF0EF11C24E00335120709F4C4C5D80102
:1090B0008D918D010E94EE29882389F30E94DA297F
:1090C000F7016083718382839383E9CF83E50E94F4
:1090D000EE29882309F4AFC50E94DA290E949EDB9D
:1090E0007093240260932302A6C583E50E94EE29B3
:1090F000882309F4A0C50E94DA290E949EDB7093A0
:1091000022026093210297C580E50E94EE29882300
:1091100009F491C50E94DA290E949EDB8B0183E548
:109120000E94EE29882329F00E94DA290E949EDB02
:1091300002C06FEF7FEF6F5F7F4F6330710508F004
:109140007AC520E0E22FEE0FFF0BE85EFB4F808137
:1091500091818017910709F46EC52F5FF3CF83E5E6
:109160000E94EE29882331F00E94DA290E949EDBBA
:109170008B0102C00EE610E080E50E94EE298823F4
:1091800031F00E94DA290E949EDBCB0102C088EEFA
:1091900093E06C01EE24D7FCE094FE2C101611062F
:1091A0007CF420E030E0A901B80185E20E94C1D63C
:1091B000C701B6010E9456D485E20E94E2D93BC5A0
:1091C000C701B6010E9456D436C580E50E94EE293B
:1091D000882351F00E94DA29609380027093810203
:1091E000809382029093830289E40E94EE2988236F
:1091F00061F00E94DA290E94C49960937C02709306
:109200007D0280937E0290937F0284E40E94EE2987
:10921000882361F00E94DA290E94D0996093780235
:109220007093790280937A0290937B0283E40E9488
:10923000EE29882351F00E94DA296093740270931A
:10924000750280937602909377020E944490E5ED38
:10925000F3E08191882339F09091C00095FFFCCF15
:109260008093C600F6CFE8EDF3E08191882339F0D2
:109270009091C00095FFFCCF8093C600F6CF40913F
:10928000800250918102609182027091830222E0FB
:1092900030E086EC94E00E949823ECEDF3E08191BD
:1092A000882339F09091C00095FFFCCF8093C600D1
:1092B000F6CF60917C0270917D0280917E02909148
:1092C0007F020E94CA99AB01BC0122E030E086EC2B
:1092D00094E00E949823E0EEF3E08191882339F036
:1092E0009091C00095FFFCCF8093C600F6CF6091AF
:1092F00078027091790280917A0290917B020E94AB
:10930000D699AB01BC0122E030E086EC94E00E94EB
:109310009823E4EEF3E08191882339F09091C00026
:1093200095FFFCCF8093C600F6CF40917402509118
:109330007502609176027091770222E030E086EC4F
:1093400094E00E9498238091C00085FFFCCF8AE0C2
:109350008093C60070C483E50E94EE29882319F02B
:109360000E94DA2903C060E070E0CB010E94F16442
:1093700062C485E40E94EE29882341F00E94DA2924
:109380000E949EDB8B0177FD0AC002C000E010E066
:10939000C12CD12CA6E1EA2EA3E4FA2E06C0C12CE2
:1093A000D12CFCE8EF2EF2E4FF2E83E50E94EE299B
:1093B000882321F00E94DA296B017C0183E40E945A
:1093C000EE29882331F00E94DA290E949EDB9B015E
:1093D00002C025E030E0A801C701B6010E94289133
:1093E0002AC40E945F1B27C40E94912024C40E94AB
:1093F0001D1F21C48AE50E94EE29882359F00E948E
:10940000DA296093230770932407809325079093AC
:10941000260711C4EEE9F6E08491882341F090918B
:10942000C00095FFFCCF8093C6003196F5CF4091E8
:10943000230750912407609125077091260722E0A9
:1094400030E086EC94E00E949823ECE9F6E0849109
:10945000882309F4F0C39091C00095FFFCCF80935E
:10946000C6003196F4CF8AE50E94EE29882379F070
:109470000E94DA29609323077093240780932507BD
:10948000909326070E945F1B0E94912028C0E1E96B
:10949000F6E08491882341F09091C00095FFFCCFC5
:1094A0008093C6003196F5CF409123075091240751
:1094B000609125077091260722E030E086EC94E069
:1094C0000E949823EFE8F6E08491882341F0909180
:1094D000C00095FFFCCF8093C6003196F5CF89B1CF
:1094E000992787FD9095692F661F6627661F4AE0BA
:1094F00050E070E086EC94E00E94C2228091C000AF
:1095000085FFFCCF8AE08093C60095C3C0904207D8
:10951000D0904307E0904407F0904507E196CCAE29
:10952000DDAEEEAEFFAEE197009146071091470722
:109530002091480730914907E5960CAF1DAF2EAF3B
:109540003FAFE59740914A0750914B0760914C0718
:1095500070914D07E9964CAF5DAF6EAF7FAFE99765
:1095600080914E0790914F07A0915007B0915107FD
:10957000ED968CAF9DAFAEAFBFAFED97C982DA82EB
:10958000EB82FC820D831E832F83388749875A879D
:109590006B877C878D879E87AF87B88B85E40E9419
:1095A000EE29882369F00E94DA299B01AC01ED962F
:1095B0006CAD7DAD8EAD9FADED970E9456DA0CC0BF
:1095C00020E030E040E050E4ED966CAD7DAD8EAD36
:1095D0009FADED970E9455DAED966CAF7DAF8EAFE3
:1095E0009FAFED9720E030E040E752E460910B023E
:1095F00070910C0280910D0290910E020E9436DB58
:109600004B015C01E996ECACFDAC0EAD1FADE997EA
:10961000E5962CAD3DAD4EAD5FADE597E1966CADF9
:109620007DAD8EAD9FADE197E2E2F7E0FF93EF9362
:10963000EDE6CE2ED12CCC0EDD1EACE0CA0ED11C38
:109640000E9470598AE50E94EE290F900F9088239E
:1096500029F00E94DA299B01AC0104C020E030E02F
:1096600040E251E4E9966CAD7DAD8EAD9FADE997DA
:109670000E9456DAE9966CAF7DAF8EAF9FAFE99747
:1096800020E030E040E752E460910B0270910C0260
:1096900080910D0290910E020E9436DB4B015C011D
:1096A000E996ECACFDAC0EAD1FADE997E5962CAD9F
:1096B0003DAD4EAD5FADE597E1966CAD7DAD8EAD48
:1096C0009FADE197E2E2F7E0FF93EF93BDE6CB2E8B
:1096D000D12CCC0EDD1EBCE0CB0ED11C0E947059EB
:1096E00088E50E94EE290F900F90882399F00E9440
:1096F000DA299B01AC01E1966CAD7DAD8EAD9FADDD
:10970000E1970E9456DAE1966CAF7DAF8EAF9FAFC6
:10971000E1970AC080E090E0A0E4B0E4E1968CAF6D
:109720009DAFAEAFBFAFE19789E50E94EE298823D8
:1097300049F00E94DA29E5966CAF7DAF8EAF9FAFFE
:10974000E5970AC080E090E0A0E4B0E4E5968CAF35
:109750009DAFAEAFBFAFE59720E030E040E752E409
:1097600060910B0270910C0280910D0290910E029B
:109770000E9436DB4B015C01E996ECACFDAC0EAD12
:109780001FADE997E5962CAD3DAD4EAD5FADE597CC
:10979000E1966CAD7DAD8EAD9FADE197E2E2F7E075
:1097A000FF93EF93ADE6CA2ED12CCC0EDD1EECE07C
:1097B000CE0ED11C0E9470598CE40E94EE290F90AD
:1097C0000F90882369F00E94DA299B01AC01ED9685
:1097D0006CAD7DAD8EAD9FADED970E9456DA0CC09D
:1097E00020E030E048EC52E4ED966CAD7DAD8EADFE
:1097F0009FADED970E9455DAED966CAF7DAF8EAFC1
:109800009FAFED9720E030E040E752E460910B021B
:1098100070910C0280910D0290910E020E9436DB35
:109820004B015C01E996ECACFDAC0EAD1FADE997C8
:10983000E5962CAD3DAD4EAD5FADE597E1966CADD7
:109840007DAD8EAD9FADE197E2E2F7E0FF93EF9340
:10985000FDE6CF2ED12CCC0EDD1EFCE0CF0ED11CB0
:109860000E9470590E94038E129A64E670E080E0B4
:1098700090E00E9456D48FE796E00E94CEAA0F9007
:109880000F9010E00E9418AC811119C01F5F0E9458
:1098900056950E946E310E9457AB1111F3CF389A42
:1098A000409A63E070E080E090E00E9456D44098D7
:1098B00063E070E080E090E00E9456D4E3CF8CE457
:1098C0000E94EE29882369F00E94DA299B01AC01ED
:1098D000ED966CAD7DAD8EAD9FADED970E9455DAE6
:1098E0000CC020E030E048EC52E4ED966CAD7DAD6C
:1098F0008EAD9FADED970E9456DAED966CAF7DAFC1
:109900008EAF9FAFED97ED968CAD9DADAEADBFAD7B
:10991000ED9780934E0790934F07A0935007B09315
:1099200051078EE497E00E94CD6420E030E040E7EC
:1099300052E460910B0270910C0280910D029091A3
:109940000E020E9436DB4B015C01BDE64B2E512C12
:109950004C0E5D1E2CE0420E511CE996ECACFDACA9
:109960000EAD1FADE997E5962CAD3DAD4EAD5FADAB
:10997000E597E1966CAD7DAD8EAD9FADE197E2E2EE
:109980006E2EE7E07E2E7F926F9262010E947059E8
:1099900020E030E040E752E460910B0270910C024D
:1099A00080910D0290910E020E9436DB4B015C010A
:1099B000E996ECACFDAC0EAD1FADE9972D813E8173
:1099C0004F81588569817A818B819C817F926F92CA
:1099D0000E94705920E030E040E752E460910B02B1
:1099E00070910C0280910D0290910E020E9436DB64
:1099F0004B015C01E984FA840B851C852D813E8135
:109A00004F81588569817A818B819C817F926F9289
:109A10000E94705920E030E040E752E460910B0270
:109A200070910C0280910D0290910E020E9436DB23
:109A30004B015C01E984FA840B851C852D813E81F4
:109A40004F81588569817A818B819C817F926F9249
:109A5000DE011D966D010E9470590FB6F894DEBFAD
:109A60000FBECDBFE8C010924D050E94D4AA8091D0
:109A7000F0069091F106A091F206B091F306809362
:109A8000F4069093F506A093F606B093F7060E94AD
:109A90003D2AD1C084E50E94EE29882309F487C0BD
:109AA0000E94DA290E94A3DB60934E056623A9F188
:109AB000ECE3FCE08491882341F09091C00095FF95
:109AC000FCCF8093C6003196F5CFE8EEF3E08191AC
:109AD000882339F09091C00095FFFCCF8093C60099
:109AE000F6CF40E050E060914E0586EC94E00E9495
:109AF000F922EAEEF3E08191882339F09091C000D9
:109B000095FFFCCF8093C600F6CF8091C00085FF03
:109B1000FCCF8AE08093C6008EC086E40E94EE29C6
:109B20008823D9F00E94DA296B017C016093000739
:109B300070930107809302079093030720E030E0C1
:109B4000A9010E9432DD181644F4C0920B02D09293
:109B50000C02E0920D02F0920E02ECE3FCE0849124
:109B6000882341F09091C00095FFFCCF8093C60000
:109B70003196F5CFEBEFF3E08191882339F09091A6
:109B8000C00095FFFCCF8093C600F6CF60912207FE
:109B900070E04AE050E086EC94E00E94C22280919E
:109BA000C00085FFFCCF8AE08093C60044C0ECE390
:109BB000FCE08491882341F09091C00095FFFCCF98
:109BC0008093C6003196F5CFECE6F6E084918823C9
:109BD00041F09091C00095FFFCCF8093C600319674
:109BE000F5CF8091690590916A0520E6289FF001E4
:109BF000299FF00D1124E159FA4F8191882339F002
:109C00009091C00095FFFCCF8093C600F6CFEAE6A6
:109C1000F6E08491882341F09091C00095FFFCCF3D
:109C20008093C6003196F5CF8091C00085FFFCCFB0
:109C30008AE08093C6000E94152A98C180E090E0D7
:109C40000E945B250C94FA3381E090E00E945B2532
:109C50000C940534A701960160914A0770914B0757
:109C600080914C0790914D070E9455DA0C9438363C
:109C70000E9456950E946E310E9457AB0C94F63E9E
:109C80000E94E329AB01BC014093DD095093DE093A
:109C90006093DF097093E00988E299E00E944D7CAF
:109CA000CACF0E94DA290E949EDB0C9458410E9480
:109CB00027D48B019C01C701B601605F784D8F4F9F
:109CC0009F4F601B710B820B930BA30192010E94AB
:109CD00000DFBA01A9012AE030E086EC94E00E949E
:109CE000EE228091C00085FFFCCF3092C6000E941A
:109CF00027D44B015C010E9456950E946E310E9450
:109D000057ABFFEFCF16DF06EF06FF0609F0A5C041
:109D100080914C05E0914E05F0E08F01000F111F7E
:109D2000000F111F01521E4EEE0FFF1FE551FE4E98
:109D300060817181882309F478C0882777FD809538
:109D4000982F0E94D1DB20E030E040E85FE30E94E2
:109D500055DA9B01AC01D8016D917D918D919C915B
:109D60000E9432DD87FFB5C00E9427D468197909A7
:109D70008A099B09693E73408105910508F4BBCFB0
:109D8000EBE1F8E08491882341F09091C00095FFC9
:109D9000FCCF8093C6003196F5CFE0914E0524E0CC
:109DA000E29FF0011124E152FE4E40815181628117
:109DB000738121E030E086EC94E00E949823E7E193
:109DC000F8E08491882341F09091C00095FFFCCF8A
:109DD0008093C6003196F5CF60914E0570E04AE061
:109DE00050E086EC94E00E94C222E3E1F8E0849126
:109DF000882341F09091C00095FFFCCF8093C6006E
:109E00003196F5CFF7FE53CFECEBF3E006C090911F
:109E1000C00095FFFCCF8093C60081918111F7CFE0
:109E20008091C00085FFFCCF60CF882777FD8095AB
:109E3000982F0E94D1DB20E030E040E85FE30E94F1
:109E400056DA9B01AC01F8016081718182819381B6
:109E50000E942FDB1816ECF587CFF7FC2FC0E0919E
:109E60004E05F0E08F01000F111F000F111F01526E
:109E70001E4EEE0FFF1FE551FE4E60817181882757
:109E800077FD8095982F0E94D1DB9B01AC01D80112
:109E90006D917D918D919C910E9455DA0E949EDB7F
:109EA00097FF07C090958095709561957F4F8F4F74
:109EB0009F4F64307105810591055CF4F7FC14C077
:109EC0000E9427D46C197D096031774208F44CCF89
:109ED0000BC00E9427D46B017C016F3FFFEF7F070F
:109EE0008F079F0759F740CF85E098E00E94BFAAEF
:109EF0000E9427D4609353057093540580935505B1
:109F0000909356050E9427D460935B0570935C057F
:109F100080935D0590935E058ECE0E94038E88E54A
:109F20000E94EE29882319F05F9A1092270789E58D
:109F30000E94EE29882319F08A9A109228078AE550
:109F40000E94EE29882351F09FB7F8948091080170
:109F50008160809308019FBF1092290785E40E94C9
:109F6000EE29882309F467CE129A65CEC950DF4FD7
:109F70000FB6F894DEBF0FBECDBFDF91CF911F911A
:109F80000F91FF90EF90DF90CF90BF90AF909F9098
:109F90008F907F906F905F904F903F902F9008959B
:109FA000CF93DF938091650590916605039714F434
:109FB0000E94672A60E08AE597E00E94F917809185
:109FC000650590916605892B09F464C080915A0754
:109FD0008823E1F08091690590916A0520E6289F29
:109FE000E001299FD00D1124C159DA4F66EF7AE0C4
:109FF000CE010E946EE3892BF1F4BE018AE597E061
:10A000000E94881780915B07882319F00E9495327F
:10A010002BC0E3EFFAE08491882341F09091C000D7
:10A0200095FFFCCF8093C6003196F5CF8091C0009C
:10A0300085FFFCCF16C060E08AE597E00E94ED182E
:10A04000E1EEFAE08491882341F09091C00095FF01
:10A05000FCCF8093C6003196F5CF8091C00085FF7C
:10A06000FCCF8AE08093C6008091650590916605DB
:10A07000019790936605809365058091690590919D
:10A080006A05019664E070E00E94EDDE90936A0537
:10A09000809369050E9456950E946E310E945486F5
:10A0A0000E9457AB659B10C080915807909159074B
:10A0B000892B51F48091030181FD06C080915C07DA
:10A0C000811102C04F9934C080915807909159076F
:10A0D000029709F047C08091030181FD3EC060ED09
:10A0E00077E080E090E00E9456D48091030181FFE8
:10A0F00034C08AE597E00E94B3118AE597E00E9498
:10A100005D1121E041E06DE074E08AE597E00E9496
:10A11000E8128AE597E00E947D120E9427D460939E
:10A12000530570935405809355059093560515C0BB
:10A1300081E090E0909359078093580768EC70E0B5
:10A1400080E090E00E9456D4659907C082E090E0DC
:10A150009093590780935807B7CF109259071092E0
:10A160005807B2CFDF91CF9108958F929F92AF920F
:10A17000BF92CF92DF92EF92FF920F931F93CF93F4
:10A18000DF938C0186539E4F0E94500F68018FE62B
:10A19000C80ED11CC114D10421F178018BE5E81A55
:10A1A0008EEFF80AE70157018FE1A81AB108F8E528
:10A1B0008F2EF4E09F2ECC15DD0599F0FE01EE19EF
:10A1C000FF09EA0DFB1D91828082FE017897808154
:10A1D000811102C06F97EFCFCE014B970E94307D67
:10A1E000F9CFC801805B9F4F0E94500FC8018F9626
:10A1F000DF91CF911F910F91FF90EF90DF90CF9063
:10A20000BF90AF909F908F900C94500F8AE597E08D
:10A210000C945C0F8AE597E0A8CF2F923F924F9263
:10A220005F926F927F928F929F92AF92BF92CF92E6
:10A23000DF92EF92FF920F931F93CF93DF93CDB7EF
:10A24000DEB7C954D1090FB6F894DEBF0FBECDBF3B
:10A250003C011B014A012DA70FA7EDAE2296ACAE23
:10A26000BDAECEAEDFAE229734E0239F2001112495
:10A27000440D551D5AAB49ABDA01CD90DD90ED9000
:10A28000FC90FC01E40DF51D208131814281538158
:10A29000C701B6010E9456DA6BAB7CAB8DAB9EABAF
:10A2A000B4E00B9F80011124F401E00FF11FF8AF1F
:10A2B000EFAB80809180A280B380F301E00FF11FAB
:10A2C0002081318142815381C501B4010E9456DA57
:10A2D00069AF7AAF8BAF9CAF2DADF4E02F9FC0017B
:10A2E0001124F301E80FF91F20813181428153814C
:10A2F0002F8F38A349A35AA3F101E80FF91F6081FA
:10A300007181828193810E9455DA6F8B788F898F5A
:10A310009A8FD1011C968D919D910D90BC91A02D8D
:10A3200089A79AA7ABA7BCA7D3011C962D913D91F5
:10A330004D915C911F972DA33EA34FA358A7A70152
:10A34000960150582B8F3C8F4D8F5E8FD501C401E5
:10A35000B0588B8B9C8BAD8BBE8BF101E40DF51D42
:10A360002BA93CA94DA95EA960817181828193814D
:10A370000E9455DA6B017C01F101E00FF11F29AD5C
:10A380003AAD4BAD5CAD60817181828193810E9459
:10A3900055DA4B015C01A70196016B8D7C8D8D8D8B
:10A3A0009E8D0E9404DE2B013C01A50194016B8966
:10A3B0007C898D899E890E9404DE9B01AC01C301CA
:10A3C000B2010E9456DA2B013C01A50194016B8D6C
:10A3D0007C8D8D8D9E8D0E9404DE4B015C01A7015A
:10A3E00096016B897C898D899E890E9404DE9B0180
:10A3F000AC01C501B4010E9455DAA30192010E948B
:10A40000C9DA6B017C0120E030E0A9010E942FDB5A
:10A4100087FF0AC02BED3FE049EC50E4C701B601CD
:10A420000E9456DA6B017C01A4968FADA497882315
:10A4300051F02BED3FE049EC50E4C701B6010E941A
:10A4400055DA6B017C01A3962CAD3DAD4EAD5FADF1
:10A45000A397C701B6010E9404DE2F89388D498D6C
:10A460005A8D5F770E943FDD4B015C012FE632E1A0
:10A4700043E85AE30E942FDB87FDDEC1C501B4012A
:10A480000E940CDC0E94A3DB7CA36BA3DB01AB2B43
:10A4900021F4E1E0F0E0FCA3EBA32BA13CA1B90186
:10A4A00080E090E00E94CFDB4B015C019B01AC019E
:10A4B000C701B6010E9436DB2B013C01A5019401C6
:10A4C0006F89788D898D9A8D0E9436DB26966CAFC8
:10A4D0007DAF8EAF9FAF26972DA13EA14FA158A56E
:10A4E00069A57AA58BA59CA50E9455DAA5019401C2
:10A4F0000E9436DB2A966CAF7DAF8EAF9FAF2A9756
:10A5000020E030E040E05FE3C301B2010E9404DEDE
:10A51000A30192010E9404DE9B01AC0160E070E0A7
:10A5200080E89FE30E9455DA69A77AA78BA79CA7CA
:10A53000CE010196FC014DAD34E0439FE00DF11DCD
:10A5400011242F8D38A149A15AA120833183428340
:10A5500053832DA13EA14FA158A52D873E874F873C
:10A56000588B1F8A41E050E058A34F8F81E090E064
:10A570008C0F9D1FBDA5A4E0BA9F800D911D1124D5
:10A580009EA78DA721E030E02C0F3D1F5FA544E082
:10A59000549F200D311D112438AB2FA7FEA3EDA32E
:10A5A000CE018C599F4F9A8B898B2F8D38A14BA14F
:10A5B0005CA12417350708F01CC19F8999310CF064
:10A5C00042C029A53AA54BA55CA56B897C898D89DC
:10A5D0009E890E9404DE6B017C01A30192016B8DB8
:10A5E0007C8D8D8D9E8D0E9404DEA70196010E94B8
:10A5F00056DA7B018C0129A53AA54BA55CA56B8D8C
:10A600007C8D8D8D9E8D0E9404DE4B015C01A3012B
:10A6100092016B897C898D899E890E9404DE9B0151
:10A62000AC01C501B4010E9455DA6B8F7C8F8D8F10
:10A630009E8FAF89AF5FAF8BA701B8014B8B5C8B4F
:10A640006D8B7E8B6AC0EF8DF8A1BF0180E090E03A
:10A650000E94CFDBA30192010E9404DE6B017C010A
:10A660000E9433DB6B8B7C8B8D8B9E8BC701B6017D
:10A670000E9467DE4B015C01A9A9BAA9CD90DD90CB
:10A68000ED90FC90F7FAF094F7F8F094AFA9B8AD1C
:10A690002D913D914D915C912F8B388F498F5A8F21
:10A6A0002B893C894D895E89C701B6010E9404DE71
:10A6B0006B8F7C8F8D8F9E8FA50194016F89788D14
:10A6C000898D9A8D0E9404DE9B01AC016B8D7C8D7F
:10A6D0008D8D9E8D0E9456DA6B8F7C8F8D8F9E8F15
:10A6E000A5019401C701B6010E9404DE6B017C0143
:10A6F0002B893C894D895E896F89788D898D9A8DEA
:10A700000E9404DE9B01AC01C701B6010E9455DA2C
:10A710006B8B7C8B8D8B9E8B1F8A2B8D3C8D4D8DF7
:10A720005E8D6BA97CA98DA99EA90E9456DAEDA524
:10A73000FEA560837183828393832B893C894D8935
:10A740005E8969AD7AAD8BAD9CAD0E9456DAAFA53E
:10A75000B8A96D937D938D939C93139726962CADFA
:10A760003DAD4EAD5FAD2697EDA1FEA1608171813B
:10A77000828193810E9456DAADA1BEA16D937D9333
:10A780008D939C9313972A962CAD3DAD4EAD5FAD46
:10A790002A976D857E858F8598890E9456DA6D8708
:10A7A0007E878F87988BCE0101960E94F12EE984D7
:10A7B000FA840B851C852D813E814F8158856981E6
:10A7C0007A818B819C81BA89BF93E989EF93229624
:10A7D0008CAC9DACAEACBFAC2297DE011D966D017A
:10A7E0007FD5EF8DF8A13196F8A3EF8F0F900F90E2
:10A7F000DCCE61015CE0C50ED11CD1011896ED9054
:10A80000FD900D911C911B9714962D913D914D91AA
:10A810005C9117976D917D918D919C91FE01EC5902
:10A82000FF4FFF93EF9322968CAC9DACAEACBFACC8
:10A83000229756D50F900F90C75BDF4F0FB6F89455
:10A84000DEBF0FBECDBFDF91CF911F910F91FF9063
:10A85000EF90DF90CF90BF90AF909F908F907F90C0
:10A860006F905F904F903F902F9008952F923F925E
:10A870004F925F926F927F928F929F92AF92BF9210
:10A88000CF92DF92EF92FF920F931F93CF93DF93BC
:10A89000CDB7DEB768970FB6F894DEBF0FBECDBF59
:10A8A0001C012A013B0148015901DC01D8966D9138
:10A8B0007D918D919C91DB970E94CFDB6B017C0198
:10A8C000A30192010E9404DE0E941CDB0E94A3DB14
:10A8D00069877A878B879C87A5019401C701B60198
:10A8E0000E9404DE0E941CDB0E94A3DB6D877E8732
:10A8F0008F87988B29853A854B855C85283731056C
:10A900004105510540F488E790E0A0E0B0E0898778
:10A910009A87AB87BC872D853E854F855889283718
:10A9200031054105510540F488E790E0A0E0B0E032
:10A930008D879E87AF87B88B91012C5B3F4FD901E4
:10A940008D919D910D90BC91A02D8D839E83AF83A1
:10A95000B887BC01CD010E94D1DB69837A838B83E8
:10A960009C8369857A858B859C850E94CFDB698B6A
:10A970007A8B8B8B9C8B20E030E0A90169817A81F6
:10A980008B819C810E942FDB882339F1A7019601DE
:10A99000C701B6010E9404DE4B015C0129893A8996
:10A9A0004B895C89CA01B9010E9404DE9B01AC019C
:10A9B000C501B4010E9455DA4B015C0129813A813D
:10A9C0004B815C81CA01B9010E9456DA9B01AC013E
:10A9D000C501B4010E9436DB03C060E070E0CB012A
:10A9E0000E941CDB0E949EDB2B013C016D817E815D
:10A9F0008F81988590958095709561957F4F8F4F49
:10AA00009F4F0E94D1DB4B015C016D857E858F8558
:10AA100098890E94CFDB6D837E838F83988720E0A7
:10AA200030E0A901C501B4010E942FDB882349F160
:10AA30002D813E814F815885CA01B9010E9404DEF3
:10AA40006D8B7E8B8F8B988FA7019601C701B60106
:10AA50000E9404DE9B01AC016D897E898F89988DEF
:10AA60000E9455DA6B017C01A5019401C501B40176
:10AA70000E9456DA9B01AC01C701B6010E9436DB89
:10AA800003C060E070E0CB010E940CDCF101808823
:10AA90009188A288B38875016401C418D508E608B6
:10AAA000F7080E949EDBC61AD70AE80AF90AF7FEE1
:10AAB0006BC020E030E0A90169817A818B819C81A3
:10AAC0000E942FDB882309F447C029813A814B81FA
:10AAD0005C81CA01B9010E9456DA6B017C01C50193
:10AAE000B4010E94CFDB9B01AC01C701B6010E94FB
:10AAF00004DE6B017C0129893A894B895C89CA0192
:10AB0000B9010E9404DE9B01AC01C701B6010E949D
:10AB100055DA6B017C012D813E814F815885CA0138
:10AB2000B9010E9404DE9B01AC01C701B6010E947D
:10AB300056DA6B017C0120E030E040E850E46981A6
:10AB40007A818B819C810E9404DE9B01AC01C7014C
:10AB5000B6010E9436DB03C060E070E0CB010E94CA
:10AB60001CDB0E949EDB2B013C0197FF03C0412CA4
:10AB7000512C3201481459046A047B0410F024015A
:10AB80003501C12CD12C76018FB7F894F101E45B2B
:10AB9000FF4F9081911125C0D10154964D925D9245
:10ABA0006D927C925797C40CD51CE61CF71CF101E2
:10ABB000C08ED18EE28EF38E29853A854B855C85D9
:10ABC000DC962D933D934D935C93DF97A05CBF4F34
:10ABD0002D853E854F8558892D933D934D935C93EC
:10ABE00013978FBF68960FB6F894DEBF0FBECDBF28
:10ABF000DF91CF911F910F91FF90EF90DF90CF9059
:10AC0000BF90AF909F908F907F906F905F904F908C
:10AC10003F902F9008954F925F926F927F92AF92E4
:10AC2000BF92CF92DF92EF92FF920F931F93CF9339
:10AC3000DF93EB017A01209709F458C041155105C3
:10AC400009F454C0AAA4BBA40CA51DA59501A80194
:10AC50006EA17FA188A599A50E942FDB882309F406
:10AC600045C08FA981113AC0F70146A057A060A442
:10AC700071A4A3019201B501C8010E9432DD18162A
:10AC80006CF5A3019201C301B2010E9404DE6B01C5
:10AC90007C018AA99BA9ACA9BDA9BC01CD01905892
:10ACA0009B01AC010E9456DA2EA53FA548A959A9DF
:10ACB0000E9404DE9B01AC01C701B6010E9455DA77
:10ACC0000E9471DE6B017C019B01AC01B501C801E2
:10ACD0000E942FDB87FD02C056018701A501B80144
:10ACE0004EA35FA368A779A781E08EABDF91CF91D8
:10ACF0001F910F91FF90EF90DF90CF90BF90AF909A
:10AD00007F906F905F904F900895DF92EF92FF9247
:10AD10000F931F93CF93DF938091ED098FB7F89432
:10AD2000E090EC098FBF8091ED0990E08E199109B8
:10AD30008F7099270497F4F01091ED0913501F704C
:10AD400040E050E000E0F12C8DE4D82E1E1591F08B
:10AD5000111101C010E11150D19EE0011124C25126
:10AD6000D64F602F7F2DCE0156DF402F5F2D0C2F49
:10AD7000FD2EECCFDF91CF911F910F91FF90EF90BF
:10AD8000DF9008954F925F926F927F92AF92BF9241
:10AD9000CF92DF92EF92FF920F931F93CF93DF93A7
:10ADA0008C01EB01009709F453C0FC0187A98111C4
:10ADB0004FC046A057A060A471A4AEA0BFA0C8A475
:10ADC000D9A49501A601C301B2010E942FDB87FF20
:10ADD0003FC0A3019201C301B2010E9404DE2B0116
:10ADE0003C01F80182A993A9A4A9B5A9BC01CD0190
:10ADF00090589B01AC010E9456DAF80126A537A5B0
:10AE000040A951A90E9404DE9B01AC01C301B2011B
:10AE10000E9455DA0E9471DE7B018C019B01AC011E
:10AE2000B501C6010E942FDB87FF02C075018601B4
:10AE30009701A801B501C6010E942FDB882341F0CC
:10AE4000A701B8014EA35FA368A779A781E08EABE5
:10AE5000DF91CF911F910F91FF90EF90DF90CF90F6
:10AE6000BF90AF907F906F905F904F900895EF925A
:10AE7000FF920F931F93CF93DF93F090EC0900E0C4
:10AE800010E080E090E02DE4E22E2091ED09F21632
:10AE900089F0EF9CE0011124C251D64FAE01B801F8
:10AEA00071DF81E08F0D803109F480E0F82EC80158
:10AEB0008E01EBCF40E050E0B801DF91CF911F91C0
:10AEC0000F91FF90EF905ECF4F925F926F927F92C3
:10AED0008F929F92AF92BF92CF92DF92EF92FF92AA
:10AEE0000F931F93CF93DF939090EC09C0E0D0E0D5
:10AEF0003DE4832E892D992787FD90952091ED09BA
:10AF000030E082179307B9F1889E5001899EB00CFA
:10AF10001124C5018251964F5C01209729F18EA919
:10AF2000811104C0F50186A98823F1F0CAA0DBA035
:10AF3000ECA0FDA0A7019601F50166A177A180A56F
:10AF400091A50E9436DB2B013C01A70196016EA161
:10AF50007FA188A599A50E9436DBAB01BC019301B6
:10AF60008201CE0183DC1EAA9394F0E19F1201C0FE
:10AF7000912CE501BFCF2097E9F0CAA0DBA0ECA09F
:10AF8000FDA0A70196016DEC7CEC8CE49DE30E9492
:10AF900036DB4B015C01A70196016EA17FA188A55C
:10AFA00099A50E9436DBAB01BC0195018401CE015D
:10AFB0005DDC1EAADF91CF911F910F91FF90EF9062
:10AFC000DF90CF90BF90AF909F908F907F906F90C9
:10AFD0005F904F90089599DE4ADF76CF1092ED0989
:10AFE0001092EC0980E1E3EDFEE0DF011D928A950D
:10AFF000E9F71092C30E1092C40E1092C50E109273
:10B00000C60E1092C70E1092C80E1092C90E109262
:10B01000CA0E1092CB0E1092CC0E1092CD0E109242
:10B02000CE0E1092CF0E1092D00E1092D10E109222
:10B03000D20E1092BF0E1092C00E1092C10E10923E
:10B04000C20E08954F925F926F927F928F929F925D
:10B05000AF92BF92CF92DF92EF92FF920F931F9326
:10B06000CF93DF938091BE0E882309F4EFC0C09088
:10B070003D02D0903E02E0903F02F090400260918D
:10B08000EB117091EC11882777FD8095982F0E9425
:10B09000D1DB20E030E040E050E40E9456DA960137
:10B0A000A7010E942FDB87FDD1C05090EC09612CD5
:10B0B000712C00E010E04DE4442E8091ED0958160B
:10B0C00009F453C0852D90E0489EF001499EF00D93
:10B0D0001124E251F64F4081518162817381452BE9
:10B0E000462B472B81F44481558166817781452B1E
:10B0F000462B472B41F44085518562857385452B4E
:10B10000462B472B69F1489EE001499ED00D112442
:10B11000C251D64F6C857D858E859F850E94D1DB7F
:10B120004B015C01688979898A899B890E94CFDB00
:10B130009B01AC01C501B4010E9436DB2AA13BA1F1
:10B140004CA15DA10E9404DE5B01D82FC92F9301A1
:10B15000A8010E9432DD18161CF435010D2F1C2F9A
:10B160005394852D8F70582EA8CF2091390230919D
:10B170003A0240913B0250913C02B301C8010E9447
:10B1800004DE9B01AC01B601C7010E9456DA8B01B7
:10B19000D82FC92F9601A7010E942FDB87FD03C07E
:10B1A0006801ED2EFC2E0091410210914202D091D7
:10B1B0004302C091440298014D2F5C2FB601C70194
:10B1C0000E9432DD18161CF08601DE2DCF2D8090F6
:10B1D000E8099090E909A090EA09B090EB0998017C
:10B1E0004D2F5C2FC501B4010E9432DD1816D4F436
:10B1F00020E037ED43EA5CE3B8018D2F9C2F0E94DD
:10B2000004DE6B017C0128E431EE4AE75FE3C5010F
:10B21000B4010E9404DEA70196010E9456DA8B0158
:10B22000D82FC92FC801AD2FBC2F8093E809909368
:10B23000E909A093EA09B093EB09B8018D2F9C2F7F
:10B240000E949EDB7093EC116093EB11DF91CF9124
:10B250001F910F91FF90EF90DF90CF90BF90AF9034
:10B260009F908F907F906F905F904F900895609126
:10B2700020079091EC098091ED09981711F1209128
:10B28000EC098DE4289FF0011124EA5CF54F608100
:10B2900030E04DE48091ED09281789F0429FF001DC
:10B2A0001124E251F64F80859185A285B385892BC3
:10B2B0008A2B8B2B09F03F5F2F5F2F70EBCF311163
:10B2C0000AC09FB7F89480910801816080930801BB
:10B2D0009FBF1092290770E089E00E94E7D4B2CEA8
:10B2E0002F923F924F925F926F927F928F929F9296
:10B2F000AF92BF92CF92DF92EF92FF920F931F9384
:10B30000CF93DF93CDB7DEB7C857D1090FB6F89406
:10B31000DEBF0FBECDBF69A37AA38BA39CA32DA3D1
:10B320003EA34FA358A7E9A6FAA60BA71CA7182D62
:10B33000092DAFAE2496BFAE24972091ED092F5F63
:10B340002D962FAF2D97203119F42D961FAE2D97E6
:10B350002D963FAD2D97E32EFF24E7FCF0948091CE
:10B36000EC0990E08E159F0539F40E9456950E94D5
:10B370006E310E9457ABF3CFCE0189969F938F9386
:10B3800004979F938F9304979F938F934DB75EB7C6
:10B39000445251090FB6F8945EBF0FBE4DBFADB712
:10B3A000BEB7119684E2E5E4F2E001900D928A9531
:10B3B000E1F70E943DCE0FB6F894DEBF0FBECDBFC1
:10B3C00020911F0F3091200F4091210F5091220F9B
:10B3D00069A17AA18BA19CA10E9404DE0E94D4DD08
:10B3E000A5966CAF7DAF8EAF9FAFA5972091230F31
:10B3F0003091240F4091250F5091260F6DA17EA111
:10B400008FA198A50E9404DE0E94D4DDA9966CAF9E
:10B410007DAF8EAF9FAFA9972091270F3091280F56
:10B420004091290F50912A0F69A57AA58BA59CA55B
:10B430000E9404DE0E94D4DDAD966CAF7DAF8EAF6E
:10B440009FAFAD9720912B0F30912C0F40912D0F76
:10B4500050912E0FD6016D917D918D919C910E94FE
:10B4600004DE0E94D4DD2C966CAF7DAF8EAF9FAF13
:10B470002C978091DF0E9091E00EA091E10EB0919B
:10B48000E20E2C962CAD3DAD4EAD5FAD2C9728173E
:10B4900039074A075B0709F4ADC0E091220734E0A1
:10B4A000E39FF0011124E152FE4E209135023091CC
:10B4B0003602409137025091380260817181828159
:10B4C00093810E942FDB87FF2FC02C968CAD9DAD02
:10B4D000AEADBFAD2C978093DF0E9093E00EA0939E
:10B4E000E10EB093E20EE1E8FCE08491882341F0A4
:10B4F0009091C00095FFFCCF8093C6003196F5CFA8
:10B50000E7E6FCE08491882341F09091C00095FF2C
:10B51000FCCF8093C6003196F5CF8091C00085FFA7
:10B52000FCCF8AE08093C6008091DF0E9091E00E00
:10B53000A091E10EB091E20E2C962CAD3DAD4EAD3A
:10B540005FAD2C97281B390B4A0B5B0BCA01B90165
:10B5500057FF07C090958095709561957F4F8F4FED
:10B560009F4F0E94D1DB6B017C0120E030E047EF70
:10B5700053E460912B0F70912C0F80912D0F9091BF
:10B580002E0F0E9404DE9B01AC01C701B6010E9490
:10B5900032DD18167CF52C968CAD9DADAEADBFADF1
:10B5A0002C978093DF0E9093E00EA093E10EB09362
:10B5B000E20EE1E8FCE08491882341F09091C00024
:10B5C00095FFFCCF8093C6003196F5CFE9E4FCE00F
:10B5D0008491882341F09091C00095FFFCCF809327
:10B5E000C6003196F5CF8091C00085FFFCCF8AE080
:10B5F0008093C6008091ED099DE4899F100111247C
:10B60000D101A251B64F1D01FD01E45BFF4F108235
:10B610002091D30E3091D40E4091D50E5091D60E7C
:10B620002FA738AB49AB5AABA5964CAC5DAC6EAC12
:10B630007FACA597421A530A640A750A77FE08C0C0
:10B640007094609450944094411C511C611C711C76
:10B65000D1014D925D926D927C9213972091D70EFD
:10B660003091D80E4091D90E5091DA0E2BAB3CABF5
:10B670004DAB5EABA9968CAC9DACAEACBFACA99704
:10B68000821A930AA40AB50AB7FE08C0B094A0941F
:10B6900090948094811C911CA11CB11CD101149622
:10B6A0008D929D92AD92BC9217972091DB0E3091B6
:10B6B000DC0E4091DD0E5091DE0E2BAF3CAF4DAF56
:10B6C0005EAFAD96CCACDDACEEACFFACAD97C21AC4
:10B6D000D30AE40AF50AF7FE08C0F094E094D09487
:10B6E000C094C11CD11CE11CF11CD1011896CD9253
:10B6F000DD92ED92FC921B972091DF0E3091E00ECF
:10B700004091E10E5091E20E2FAB38AF49AF5AAFE6
:10B710002C966CAD7DAD8EAD9FAD2C97621B730BDF
:10B72000840B950B97FF07C0909580957095619558
:10B730007F4F8F4F9F4F0E94D1DBE091220734E073
:10B74000E39FF0011124E35EFD4F208131814281AE
:10B7500053810E9404DE0E949EDB9B01AC01A091FC
:10B760002102B09122020E944EDF24E630E040E048
:10B7700050E00E9422DFD1011C962D933D934D9302
:10B780005C931F97C814D904EA04FB0414F47501F0
:10B790006401C216D306E406F50614F469017A01C1
:10B7A000D301C2014C145D046E047F0414F4D7016C
:10B7B000C601F101808B918BA28BB38B0697A105FB
:10B7C000B10508F478C7E85BFF4F8091200790919E
:10B7D0002107AA2797FDA095BA2F80839183A28382
:10B7E000B383A5962CAD3DAD4EAD5FADA5978FA5AE
:10B7F00098A9A9A9BAA9281739074A075B0724F00D
:10B80000D10190961C9203C081E0F10180A3A9961A
:10B810002CAD3DAD4EAD5FADA9978BA99CA9ADA94F
:10B82000BEA9281739074A075B073CF4D101909657
:10B830008C919097826090968C93AD962CAD3DAD97
:10B840004EAD5FADAD978BAD9CADADADBEAD281728
:10B8500039074A075B073CF4D10190968C91909789
:10B86000846090968C932C962CAD3DAD4EAD5FAD23
:10B870002C978FA998ADA9ADBAAD281739074A07FB
:10B880005B073CF4D10190968C91909788609096DC
:10B890008C93C257DF4FE881F981CE58D040808128
:10B8A000F10181A345284628472809F05F98F10156
:10B8B00084819581A681B781892B8A2B8B2B09F0F6
:10B8C0008A98F10180859185A285B385892B8A2B81
:10B8D0008B2B41F09FB7F894809108018E7F809365
:10B8E00008019FBFF10184859585A685B785892BC1
:10B8F0008A2B8B2B09F01298D1011C962D913D912A
:10B900004D915C911F9761962CAF3DAF4EAF5FAFED
:10B910006197232B242B252B19F5B091F30EBFA78C
:10B92000E091F40EEBABF091F50EFBAF2091F60E2B
:10B930002FAB2B2F3E2F4F2F5FA9612F702F8FAD75
:10B9400024969FAD24970E942FDB87FD1AC01FA766
:10B950000BAB3FAD3BAF24964FAD24974FAB11C01F
:10B9600050910B0F5FA780910C0F8BAB90910D0F37
:10B970009BAFA0910E0FAFAB252F382F492F5A2F19
:10B98000DCCF8091D30E9091D40EA091D50EB091C2
:10B99000D60EA5962CAD3DAD4EAD5FADA597281B3F
:10B9A000390B4A0B5B0BCA01B9010E94D1DB209114
:10B9B0001F0F3091200F4091210F5091220F0E94B4
:10B9C00036DB2B013C01698B7A8B8B8B9C8B8091B6
:10B9D000D70E9091D80EA091D90EB091DA0EA996FB
:10B9E0002CAD3DAD4EAD5FADA997281B390B4A0B71
:10B9F0005B0BCA01B9010E94D1DB2091230F30916A
:10BA0000240F4091250F5091260F0E9436DB4B01E9
:10BA10005C016D8B7E8B8F8B988F8091DB0E90916C
:10BA2000DC0EA091DD0EB091DE0EAD962CAD3DADDD
:10BA30004EAD5FADAD97281B390B4A0B5B0BCA01AE
:10BA4000B9010E94D1DB2091270F3091280F40913E
:10BA5000290F50912A0F0E9436DB6B017C01698F00
:10BA60007A8F8B8F9C8F8091DF0E9091E00EA0914A
:10BA7000E10EB091E20E2C962CAD3DAD4EAD5FAD1A
:10BA80002C97281B390B4A0B5B0BCA01B9010E948A
:10BA9000D1DB20912B0F30912C0F40912D0F509125
:10BAA0002E0F0E9436DBE091220734E0E39FF00185
:10BAB0001124E35EFD4F20813181428153810E9438
:10BAC00004DE23966CAF7DAF8EAF9FAF239760915E
:10BAD000210270912202882777FD8095982F0E947D
:10BAE000D1DB9B01AC0123966CAD7DAD8EAD9FADDE
:10BAF00023970E9404DE20E030E048EC52E40E94EC
:10BB000036DB6D8F7E8F8F8F98A3D1012D913D9164
:10BB10004D915C91139728962CAF3DAF4EAF5FAF20
:10BB200028972630310541055105FCF414960D91F6
:10BB30001D912D913C911797063011052105310576
:10BB4000A4F418960D911D912D913C911B970630F0
:10BB50001105210531054CF4DC01CB01BF77F10162
:10BB600086A797A7A0ABB1AB25C0C301B2010E94C5
:10BB7000AFDE2B013C01C501B4010E94AFDE9B0189
:10BB8000AC01C301B2010E9456DA4B015C01C7014E
:10BB9000B6010E94AFDE9B01AC01C501B4010E9459
:10BBA00056DA0E9471DED1019E966D937D938D933E
:10BBB0009C93D197D1019E962D913D914D915C9191
:10BBC000D197A1962CAF3DAF4EAF5FAFA19760E08C
:10BBD00070E080E89FE30E9436DB9B01AC016FA51B
:10BBE0007BA98BAD9FA90E9404DE2B013C019091A3
:10BBF000ED098091EC09E92FF0E0E81BF109EF7005
:10BC0000FF27FCAFEBAFA301920160E074E284E791
:10BC100099E40E9436DB0E94D4DD6B017C012BADE0
:10BC20003CAD223031050CF442C04901AA2497FCF6
:10BC3000A094BA2CC501B4010E94D1DB20E030E011
:10BC400040E051E40E942FDB87FF31C080913F0F1D
:10BC50009091400FA091410FB091420FC816D906A4
:10BC6000EA06FB0620F5BC01CD016C197D098E09A1
:10BC70009F09660F771F881F991FA50194010E94D5
:10BC800000DFCA01B9010E94CFDB0E94D4DD6C0D38
:10BC90007D1D8E1D9F1D0E94CFDB9B01AC0160E0CE
:10BCA00074E284E799E40E9436DB2B013C01A30196
:10BCB0009201A1966CAD7DAD8EAD9FADA1970E9416
:10BCC00004DE65966CAF7DAF8EAF9FAF6597D101F7
:10BCD00092966D937D938D939C93959750966D91CD
:10BCE0007D918D919C9153970E94CFDB6FA778AB8C
:10BCF00089AB9AABA30192010E9404DE0E941CDB77
:10BD00000E94A3DB6B017C01F10160AF71AF82AFD8
:10BD100093AF8E010F5E1F4F2FE23FE06D963FAF56
:10BD20002EAF6D97AE014F5D5F4F5EA74DA7CE0161
:10BD300001966B969FAF8EAF6B971BAA1FAA90E8D8
:10BD40009FAFAFE32496AFAF2497F8016191719153
:10BD5000819191918F01A30192010E9404DE6B9663
:10BD6000AEADBFAD6B976D937D938D939D936B96A9
:10BD7000BFAFAEAF6B979B01AC015F7769962CAFFD
:10BD80003DAF4EAF5FAF69976D96AEADBFAD6D97EE
:10BD90008D909D90AD90BD906D96BFAFAEAF6D97FD
:10BDA000A501940169966CAD7DAD8EAD9FAD69978F
:10BDB0000E9432DD181614F569962CAD3DAD4EADDE
:10BDC0005FAD6997C501B4010E9436DBB62EA72E80
:10BDD000982E892E262F372F482F592F6BA97FA9F0
:10BDE0008FAD24969FAD24970E942FDB87FD06C060
:10BDF000BBAAAFAA9FAE24968FAE2497EDA5FEA551
:10BE00000E171F0709F0A1CF20E030E040E85FE304
:10BE10006BA97FA98FAD24969FAD24970E942FDB3D
:10BE200087FF45C05E01F1E1AF0EB11C8E010F5FCF
:10BE30001F4F2BA93FA94FAD24965FAD2497D80182
:10BE40006D917D918D919C910E9404DEF80161932A
:10BE50007193819391938F01EA15FB0551F72BA9FB
:10BE60003FA94FAD24965FAD249765966CAD7DAD2F
:10BE70008EAD9FAD65970E9404DED10192966D93C1
:10BE80007D938D939C939597C701B6010E94CFDB5C
:10BE90002BA93FA94FAD24965FAD24970E9404DEE5
:10BEA0000E94A3DBF10160AF71AF82AF93AFA196A7
:10BEB0002CAD3DAD4EAD5FADA1976FA578A989A919
:10BEC0009AA90E9436DB6B017C0128962CAD3DAD12
:10BED0004EAD5FAD2897232B242B252B59F5F1016F
:10BEE00084819581A681B781892B8A2B8B2B11F5B3
:10BEF00080859185A285B385892B8A2B8B2BD1F4E4
:10BF00002091030F3091040F4091050F5091060FBF
:10BF1000C701B6010E9404DE0E941CDB81010C5B9C
:10BF20001F4F0E94A3DBD8016D937D938D939C934B
:10BF30001397F8C02091070F3091080F4091090F17
:10BF400050910A0FC701B6010E9404DE0E941CDB5B
:10BF50000E94A3DB81010C5B1F4FF801608371839A
:10BF6000828393834090E30E5090E40E6090E50E40
:10BF70007090E60E0E94CFDB4B015C0128966CAD01
:10BF80007DAD8EAD9FAD28970E94D1DB9B01AC01AA
:10BF9000C501B4010E9404DE2FA538A949A95AA9F8
:10BFA0000E9436DB4B015C01C301B2010E94CFDB72
:10BFB0009B01AC01C501B4010E9432DD181634F4B6
:10BFC000D8014D925D926D927C9213974090E70E4E
:10BFD0005090E80E6090E90E7090EA0EF8016081D2
:10BFE0007181828193810E94CFDB4B015C01D10181
:10BFF00014966D917D918D919C9117970E94D1DB44
:10C000009B01AC01C501B4010E9404DE2FA538A933
:10C0100049A95AA90E9436DB4B015C01C301B20158
:10C020000E94CFDB9B01AC01C501B4010E9432DD4F
:10C0300018162CF4F801408251826282738240907B
:10C04000EF0E5090F00E6090F10E7090F20E8101A4
:10C050000C5B1F4FD8016D917D918D919C910E9439
:10C06000CFDB4B015C0161966CAD7DAD8EAD9FADBC
:10C0700061970E94D1DB9B01AC01C501B4010E9414
:10C0800004DE2FA538A949A95AA90E9436DB4B0125
:10C090005C01C301B2010E94CFDB9B01AC01C50171
:10C0A000B4010E9432DD18162CF4F801408251824E
:10C0B000628273824090EB0E5090EC0E6090ED0E19
:10C0C0007090EE0ED8016D917D918D919C910E94A2
:10C0D000CFDB4B015C01F101608571858285938521
:10C0E0000E94D1DB9B01AC01C501B4010E9404DEBA
:10C0F0002FA538A949A95AA90E9436DB4B015C013A
:10C10000C301B2010E94CFDB9B01AC01C501B401A8
:10C110000E9432DD181634F4D8014D925D926D9272
:10C120007C921397F101EC5BFF4F608171818281FA
:10C1300093810E94CFDB4B015C01A70196010E9415
:10C1400036DBE1966CAF7DAF8EAF9FAFE197F1012B
:10C1500062AB73AB84AB95AB2DEB37E346E051E4B8
:10C16000C501B4010E9404DE0E949EDBD1015C96F1
:10C170006D937D938D939C935F97C090FF0ED090AD
:10C18000000FE090010FF090020F20E030E040E05F
:10C190005FE3C701B6010E9404DE6FA77BAB8C0191
:10C1A00029853A854B855C85E5962CAF3DAF4EAF32
:10C1B0005FAFE5978091FB0E9091FC0EA091FD0E74
:10C1C000B091FE0E61968CAF9DAFAEAFBFAF6197E1
:10C1D00020E030E040E05FE3BC01CD010E9404DEDE
:10C1E000B62EA72E982E892EE5966CAD7DAD8EAD20
:10C1F0009FADE5979F772B2D3A2D492D582D0E9405
:10C2000032DD18167CF42B2D3A2D492D582D6FA5B3
:10C210007BA9C8010E942FDB87FD04C0BFA6ABAA83
:10C22000092D182D2D853E854F855889E9962CAF0F
:10C230003DAF4EAF5FAFE9978091F70E9091F80E4A
:10C24000A091F90EB091FA0E65968CAF9DAFAEAF8E
:10C25000BFAF659720E030E040E05FE3BC01CD0177
:10C260000E9404DEB62EA72E982E892EE9966CAD7C
:10C270007DAD8EAD9FADE9979F772B2D3A2D492D42
:10C28000582D0E9432DD18167CF42B2D3A2D492DA5
:10C29000582D6FA57BA9C8010E942FDB87FD04C024
:10C2A000BFA6ABAA092D182DD1019296BC91BFABA8
:10C2B000F101F3A1FFAFD1019496BC912496BFAFD9
:10C2C0002497F101F5A12596FFAF25972FA93FAD42
:10C2D0004B2F5F2F6FA57BA9C8010E942FDB87FD25
:10C2E0000AC02FA92FA73FAD3BAB24960FAD2497D3
:10C2F00025961FAD25974BAD5CAD423051050CF432
:10C300000DC15091BF0E5BAF8091C00E66968FAF8E
:10C3100066979091C10E6A969FAF6A97A091C20EE0
:10C320006C96AFAF6C9727E137EB41ED58E36BADFF
:10C33000782F892F9A2F0E9432DD18160CF0EEC04C
:10C340002091C30E3091C40E4091C50E5091C60E7F
:10C3500069817A818B819C810E9455DA2B013C0195
:10C360002091C70E3091C80E4091C90E5091CA0E4F
:10C370006D817E818F8198850E9455DA4B015C0129
:10C38000A3019201C301B2010E9404DE2B013C0112
:10C39000A5019401C501B4010E9404DE9B01AC011A
:10C3A000C301B2010E9456DA0E9471DE4B015C01AA
:10C3B000A70196010E9432DD18164CF4A5019401E4
:10C3C000C701B6010E9436DB5B014C0106C0A12CFF
:10C3D000B12C50E8852E6FE3962E2091CB0E309134
:10C3E000CC0E4091CD0E5091CE0EE5966CAD7DAD4C
:10C3F0008EAD9FADE5970E9455DA6B017C01E89404
:10C40000F7F861962CAD3DAD4EAD5FAD6197C701BC
:10C41000B6010E9432DD1816E4F4A7019601619678
:10C420006CAD7DAD8EAD9FAD61970E9436DBF62E73
:10C43000E72ED82EC92E262F372F482F592FB5017A
:10C44000C4010E942FDB87FD04C0AF2CBE2C8D2CB5
:10C450009C2C2091CF0E3091D00E4091D10E509156
:10C46000D20EE9966CAD7DAD8EAD9FADE9970E9481
:10C4700055DA6B017C01E894F7F865962CAD3DAD7B
:10C480004EAD5FAD6597C701B6010E9432DD18164B
:10C49000E4F4A701960165966CAD7DAD8EAD9FADC0
:10C4A00065970E9436DBF62EE72ED82EC92E262F52
:10C4B000372F482F592FB501C4010E942FDB87FD6C
:10C4C00004C0AF2CBE2C8D2C9C2C9501A4016FA90F
:10C4D0007FAD24968FAD249725969FAD25970E941A
:10C4E00004DE4B015C019B01AC016BAD66967FAD38
:10C4F00066976A968FAD6A976C969FAD6C970E940F
:10C500002FDB87FF0EC08BAC66969FAC66976A9652
:10C51000AFAC6A976C96BFAC6C9703C08FA49BA816
:10C520005801C401D501F10182A793A7A4A7B5A71B
:10C53000E1966CAD7DAD8EAD9FADE19790589B01BE
:10C54000AC010E9456DAA1962CAD3DAD4EAD5FAD6B
:10C55000A1970E9404DE9B01AC016BE077ED83E2C2
:10C560009BE30E9455DA0E9471DE7B01D82EC92E12
:10C570009B01482F592FB401C5010E942FDB87FD75
:10C5800003C04701AD2CBC2CC401D501F10186A329
:10C5900097A3A0A7B1A797014D2D5C2D6FA97FADE3
:10C5A00024968FAD249725969FAD25970E942FDB6B
:10C5B00018162CF081E0D101D7968C9302C0F101BE
:10C5C00017AA81E0D101D6968C9380E1FE013196C5
:10C5D000A3ECBEE001900D928A95E1F78FA99FAD83
:10C5E0002496AFAD24972596BFAD25978093BF0EB7
:10C5F0009093C00EA093C10EB093C20E9C01AD01EA
:10C600006FA57BA9C8010E9436DB6B017C012FA9B5
:10C610003FAD24964FAD249725965FAD2597B40185
:10C62000C5010E9436DBAB01BC0197018601C10147
:10C630000E9436542D96BFAD2D97B093ED09A59667
:10C640002CAD3DAD4EAD5FADA5972093D30E30938D
:10C65000D40E4093D50E5093D60EA9968CAD9DADB9
:10C66000AEADBFADA9978093D70E9093D80EA0938F
:10C67000D90EB093DA0EAD962CAD3DAD4EAD5FAD9B
:10C68000AD972093DB0E3093DC0E4093DD0E50937C
:10C69000DE0E2C968CAD9DADAEADBFAD2C978093CC
:10C6A000DF0E9093E00EA093E10EB093E20E0E9495
:10C6B000EB570E94F986C858DF4F0FB6F894DEBFDB
:10C6C0000FBECDBFDF91CF911F910F91FF90EF90E3
:10C6D000DF90CF90BF90AF909F908F907F906F90A2
:10C6E0005F904F903F902F9008956F927F928F921E
:10C6F0009F92AF92BF92CF92DF92EF92FF920F93F1
:10C700001F93CF93DF93CDB7DEB7A4970FB6F894FE
:10C71000DEBF0FBECDBF3C0182E00E946B8E6B017D
:10C720007C0181E00E946B8E4B015C0180E00E94E5
:10C730006B8EAB01BC0195018401C3010E945CCCEE
:10C740008DB79EB784970FB6F8949EBF0FBE8DBF6E
:10C75000ADB7BEB7119684E2E5E4F2E001900D9228
:10C760008A95E1F7CE0101960E94E3CF8DB79EB77F
:10C7700084960FB6F894DEBF0FBECDBF84970FB678
:10C78000F8949EBF0FBE8DBFADB7BEB7119684E2C1
:10C79000FE01319601900D928A95E1F7C3010E9446
:10C7A000F2CC0FB6F894DEBF0FBECDBFC301A49686
:10C7B0000FB6F894DEBF0FBECDBFDF91CF911F91B2
:10C7C0000F91FF90EF90DF90CF90BF90AF909F9030
:10C7D0008F907F906F900895CF92DF92EF92FF92AB
:10C7E0000F931F93CF93DF93CDB7DEB72C970FB680
:10C7F000F894DEBF0FBECDBF69837A838B839C83A1
:10C800002D833E834F835887E986FA860B871C87E2
:10C81000CE0109969F938F9304979F938F930497CC
:10C820009F938F938DB79EB784970FB6F8949EBF52
:10C830000FBE8DBFADB7BEB7119684E2E5E4F2E05E
:10C8400001900D928A95E1F70E943DCE0FB6F894C3
:10C85000DEBF0FBECDBF20911F0F3091200F409142
:10C86000210F5091220F69817A818B819C810E94D6
:10C8700004DE0E94D4DD6093D30E7093D40E8093B7
:10C88000D50E9093D60E2091230F3091240F409116
:10C89000250F5091260F6D817E818F8198850E9492
:10C8A00004DE0E94D4DD6093D70E7093D80E80937F
:10C8B000D90E9093DA0E2091270F3091280F4091D6
:10C8C000290F50912A0F69857A858B859C850E9456
:10C8D00004DE0E94D4DD6093DB0E7093DC0E809347
:10C8E000DD0E9093DE0E20912B0F30912C0F409196
:10C8F0002D0F50912E0FF6016081718182819381FD
:10C900000E9404DE0E94D4DD6093DF0E7093E00E7F
:10C910008093E10E9093E20E2FED3EE04BED5EE052
:10C9200067ED7EE083ED9EE00E94108E1092BF0EB8
:10C930001092C00E1092C10E1092C20E1092C30E31
:10C940001092C40E1092C50E1092C60E1092C70E11
:10C950001092C80E1092C90E1092CA0E1092CB0EF1
:10C960001092CC0E1092CD0E1092CE0E1092CF0ED1
:10C970001092D00E1092D10E1092D20E2C960FB6AD
:10C98000F894DEBF0FBECDBFDF91CF911F910F9105
:10C99000FF90EF90DF90CF90089520912B0F309172
:10C9A0002C0F40912D0F50912E0FFC016081718151
:10C9B000828193810E9404DE0E94D4DD6093DF0EA9
:10C9C0007093E00E8093E10E9093E20E8FED9EE067
:10C9D0000C944C8E8091ED099091EC09891B8F701D
:10C9E00008956093350270933602809337029093D6
:10C9F00038020895CF92DF92EF92FF920F931F9328
:10CA0000CF93DF9300D01F92CDB7DEB7FFE0CF2EDC
:10CA1000FFE0DF2EAFE1EA2EAFE0FA2E03EE1EE0DC
:10CA2000F60161917191819191916F01F7012191CD
:10CA30003191419151917F0129833A834B835C83EA
:10CA40000E94CFDB29813A814B815C810E9404DE08
:10CA50000E94A3DBF80161937193819391938F01FD
:10CA6000FFE1CF16FFE0DF06D9F60F900F900F9091
:10CA70000F90DF91CF911F910F91FF90EF90DF907A
:10CA8000CF9008954F925F926F927F92AF92BF9234
:10CA9000CF92DF92EF92FF920F931F93CF93DF938A
:10CAA000EC018B017A0163E070E00E94EDDE5C0135
:10CAB000F801D70120E030E028173907A4F44081BD
:10CAC0005181628173814D905D906D907C90139740
:10CAD00041925192619271924D935D936D937D93CA
:10CAE0002F5F3F4FE9CFDC01AA0FBB1FAA0FBB1F6F
:10CAF000F801EA0FFB1FAE0DBF1DAC16BD060CF012
:10CB000040C040815181628173810D911D912D91B1
:10CB10003C91139700831183228333834D935D935C
:10CB20006D937C9313974481558166817781149628
:10CB30000D911D912D913C911797048315832683A8
:10CB4000378314964D935D936D937C93179700856F
:10CB50001185228533851896CD90DD90ED90FC905F
:10CB60001B97C086D186E286F38618960D931D9397
:10CB70002D933C931B9783E0A80EB11C3C961C960A
:10CB8000BCCFDF91CF911F910F91FF90EF90DF907D
:10CB9000CF90BF90AF907F906F905F904F9008952F
:10CBA0002F923F924F925F926F927F928F929F92BD
:10CBB000AF92BF92CF92DF92EF92FF920F931F93AB
:10CBC000CF93DF9300D000D0CDB7DEB75C017C837C
:10CBD0006B838A01FA01C080D180E280F38020E07B
:10CBE00030E0A901C701B6010E9432DD87FF04C011
:10CBF000F7FAF094F7F8F0949501220F331F220F03
:10CC0000331F3A8329831E821D828D819E81EB8191
:10CC1000FC818E179F070CF03FC0812C912C212C9A
:10CC2000312C2A143B0474F5F801E80DF91D4080FD
:10CC300051806280738020E030E0A901C301B2011D
:10CC40000E9432DDA301920187FD5058C701B60151
:10CC50000E942FDB87FF0FC020E030E0A901C30155
:10CC6000B2010E9432DD7301620187FF04C0F7FA4E
:10CC7000F094F7F8F0943FEF231A330A84E0880E1B
:10CC8000911CCFCFED81FE813196FE83ED8329810A
:10CC90003A81020F131FB9CFC701B60126960FB60E
:10CCA000F894DEBF0FBECDBFDF91CF911F910F91E2
:10CCB000FF90EF90DF90CF90BF90AF909F908F90BC
:10CCC0007F906F905F904F903F902F9008952F929C
:10CCD0003F924F925F926F927F928F929F92AF920C
:10CCE000BF92CF92DF92EF92FF920F931F93CF9359
:10CCF000DF93EC017B016A01C69FC001C79F900DC5
:10CD0000D69F900D1124880F991F880F991F0E949C
:10CD100067DFAE01440F551F440F551F20E030E080
:10CD200000E010E00E151F0544F5E0E0F0E0212CD6
:10CD3000312C5601A20EB31E4C01820E931E2C16EE
:10CD40003D06B4F4B5016E0F7F1FDB014D905D9081
:10CD50006D907C90B4016E0F7F1FDB014D925D9250
:10CD60006D927C921397BFEF2B1A3B0A3496E7CF54
:10CD70000F5F1F4F240F351FD5CFDF91CF911F912C
:10CD80000F91FF90EF90DF90CF90BF90AF909F906A
:10CD90008F907F906F905F904F903F902F9008956D
:10CDA0002F923F924F925F926F927F928F929F92BB
:10CDB000AF92BF92CF92DF92EF92FF920F931F93A9
:10CDC000CF93DF9300D000D0CDB7DEB79E838D83A5
:10CDD0004A015B013901181619060CF028C120E040
:10CDE00030E0A901C501B4010E942FDB882309F4BA
:10CDF0001EC10130110529F421E0C216D10489F4C5
:10CE000073C017FF0EC021E030E04D815E81241B0E
:10CE1000350B209FC001219F900D309F900D112454
:10CE200002C080E090E0D7FE0EC021E030E0ED814E
:10CE3000FE812E1B3F0B2C9DA0012D9D500D3C9D76
:10CE4000500D112402C040E050E09601220F331F24
:10CE5000220F331F3C832B83F801EE0FFF1FEE0FD1
:10CE6000FF1FFA83E9838A01000F111F000F111FB2
:10CE70000E0D1F1D7C01EE0CFF1CEE0CFF1CE60CC2
:10CE8000F71C612C712CC12CD12C412C512C180178
:10CE90002C0C3D1CF701E60DF71D208131814281EC
:10CEA0005381C501B4010E9404DE9B01AC01F10174
:10CEB00060817181828193810E9456DAF1016083E1
:10CEC000718382839383FFEF4F1A5F0A2B813C812A
:10CED000C20ED31E49815A81640E751E8D819E81BA
:10CEE00048165906A1F6A3C0CD80DE8093E0C92282
:10CEF000DD2413018701412C512C4C145D04ECF40A
:10CF0000F10121913191419151911F01C501B4016C
:10CF10000E9404DE9B01AC01F80160817181828175
:10CF200093810E9456DAF8016193719381939193F2
:10CF30008F01FFEF4F1A5F0AE0CFC601880F991FDC
:10CF4000880F991F8701080F191F7C0124E0E20E4A
:10CF5000F11CE60CF71C4D815E81C416D5060CF061
:10CF600066C0F70134972081318142815381C50128
:10CF7000B4010E9404DE9B01AC01F8016081718163
:10CF8000828193810E9456DAF801608371838283E3
:10CF90009383F7012081318142815381C501B4011E
:10CFA0000E9404DE9B01AC01F801648175818681D9
:10CFB00097810E9456DAF80164837583868397838C
:10CFC000F7012481358146815781C501B4010E9452
:10CFD00004DE9B01AC01F801608571858285938533
:10CFE0000E9456DAF8016087718782879387F7017C
:10CFF0002085318542855385C501B4010E9404DE38
:10D000009B01AC01F80164857585868597850E9432
:10D0100056DAF8016487758786879787F4E0CF0E24
:10D02000D11C005F1F4F20E1E20EF11C94CF269629
:10D030000FB6F894DEBF0FBECDBFDF91CF911F9129
:10D040000F91FF90EF90DF90CF90BF90AF909F90A7
:10D050008F907F906F905F904F903F902F900895AA
:10D060002F923F924F925F926F927F928F929F92F8
:10D07000AF92BF92CF92DF92EF92FF920F931F93E6
:10D08000CF93DF9300D01F92CDB7DEB79C838B8305
:10D090006B017901181619060CF020C141305105B9
:10D0A00021F40130110589F46EC057FF0EC021E054
:10D0B00030E08B819C81281B390B249FC001259F68
:10D0C000900D349F900D112402C080E090E017FF76
:10D0D0000EC061E070E0EB81FC816E1B7F0B609FF6
:10D0E0009001619F300D709F300D112402C020E02F
:10D0F00030E01A01220C331C220C331CA801440F0F
:10D10000551F440F551F5A8349838C01000F111F6F
:10D11000000F111F0C0D1D1D6901CC0CDD1CCC0C6A
:10D12000DD1CCE0CDF1C612C712CE12CF12C412C70
:10D13000512C812C912C5401F801EE0DFF1DD601CC
:10D14000A60DB71D2D913D914D915C91608171812E
:10D15000828193810E9404DE9B01AC01C501B40170
:10D160000E9456DA4B015C015FEF451A550AE20C4A
:10D17000F31C89819A81680E791EEB81FC814E1621
:10D180005F06D1F6AEC08B819C8165E070E00E94A5
:10D19000EDDE8C012C01DA82C9821901612C712C1F
:10D1A000812C912C540160167106E4F4E981FA8116
:10D1B0006191719181919191FA83E983F1012191BA
:10D1C0003191419151911F010E9404DE9B01AC01FC
:10D1D000C501B4010E9456DA4B015C01FFEF6F1AE2
:10D1E0007F0AE1CF000F111F000F111FC00ED11ECB
:10D1F000E00EF11E4B815C81441655060CF071C0A7
:10D20000F7012081318142815381F6016081718172
:10D21000828193810E9404DE9B01AC01C501B401AF
:10D220000E9456DA4B015C01F70124813581468169
:10D230005781F60164817581868197810E9404DEA1
:10D240009B01AC01C501B4010E9456DA4B015C019F
:10D25000F7012085318542855385F601608571850A
:10D26000828593850E9404DE9B01AC01C501B40157
:10D270000E9456DA4B015C01F7012485358546850D
:10D280005785F60164857585868597850E9404DE3D
:10D290009B01AC01C501B4010E9456DA4B015C014F
:10D2A000F7012089318942895389F60160897189A2
:10D2B000828993890E9404DE9B01AC01C501B401FF
:10D2C0000E9456DA4B015C01F5E04F0E511C24E13F
:10D2D000C20ED11C34E1E30EF11C8CCF812C912CB9
:10D2E0005401C501B4010F900F900F900F90DF9182
:10D2F000CF911F910F91FF90EF90DF90CF90BF9053
:10D30000AF909F908F907F906F905F904F903F90E5
:10D310002F9008952F923F924F925F926F927F923B
:10D320008F929F92AF92BF92CF92DF92EF92FF9235
:10D330000F931F93CF93DF9300D01F92CDB7DEB72B
:10D340009C838B83181619060CF09AC014161506C8
:10D350000CF096C0019799F4FB01C080D180E28067
:10D36000F38020E030E0A901C701B6010E9432DD60
:10D3700087FF89C0F7FAF094F7F8F09484C0CA01E7
:10D38000880F991F880F991F9A8389838B01812C9D
:10D39000912C30E8A32E3FE3B32E412C512C612C6D
:10D3A000712C212C312CF801C080D180E280F380D7
:10D3B00020E030E0A901C701B6010E942FDB8823DD
:10D3C00009F444C020E030E0A901C701B6010E9481
:10D3D00032DD87FF04C0F7FAF094F7F8F094A70164
:10D3E0009601B201C3010E942FDB87FF1DC0A70178
:10D3F0009601B201C3010E9436DB2B013C019B0167
:10D40000AC01C501B4010E9404DEA30192010E9497
:10D4100004DE20E030E040E85FE30E9456DA4B0192
:10D420005C012601370112C09201A301C701B601B8
:10D430000E9436DB9B01AC010E9404DE9B01AC0123
:10D44000C501B4010E9456DA4B015C01FFEF2F1AAF
:10D450003F0A89819A81080F191FEB81FC812E16E2
:10D460003F0609F0A0CFC501B4010E9471DE9B0107
:10D47000AC01B201C3010E9404DE6B017C0103C058
:10D48000C12CD12C7601C701B6010F900F900F90DF
:10D490000F90DF91CF911F910F91FF90EF90DF9050
:10D4A000CF90BF90AF909F908F907F906F905F9044
:10D4B0004F903F902F9008952F923F924F925F92FE
:10D4C0006F927F928F929F92AF92BF92CF92DF9294
:10D4D000EF92FF920F931F93CF93DF93CDB7DEB7F9
:10D4E000E4970FB6F894DEBF0FBECDBF9C878B8745
:10D4F0007A876987588B4F8729011CA30BA31501D5
:10D500009C8E8B8E6096EEADFFAD6097CF01815FF4
:10D51000984D21E030E08F319E4410F420E030E05F
:10D52000CF0160E177E20E94EDDE61E070E07E8B8A
:10D530006D8B892B11F41E8A1D8ACF0168EE73E072
:10D540000E94EDDE8D599F4FA1E0B0E0BAA3A9A3E0
:10D55000873C910510F41AA219A2CF0164E670E08D
:10D560000E94EDDE099641E050E05E8F4D8F4397BB
:10D5700010F41E8E1D8ECF016AE070E00E94EDDE79
:10D5800061E070E078A36F8F892B11F418A21F8ED1
:10D590006F84788871E0671A7108461457040CF498
:10D5A00032016114710409F062C0232B51F0F701BC
:10D5B00080819181A281B381F60180839183A283CE
:10D5C000B3832D893E89232B51F0F701808191810E
:10D5D000A281B381F10180839183A283B3832F8DD4
:10D5E00038A1232B69F0F70180819181A281B38159
:10D5F0002E96EEADFFAD2E9780839183A283B383E9
:10D6000029A13AA1232BF9F0AB85BC858D909D9083
:10D61000AD90BC9020E030E0A901C501B4010E94AA
:10D620002FDB882391F0A5019401F70160817181BE
:10D63000828193810E9436DBAB8DBC8D6D937D938F
:10D640008D939C9313971D8202C0B1E0BD831D860C
:10D65000ED8DFE8DEF2B09F40BC42C96AEADBFAD56
:10D660002C971D921D921D921C92139701C4211597
:10D67000310529F4ED89FE89EF2BB9F413C0F701C8
:10D68000D60181E090E04F8558894817590794F3F7
:10D6900041915191619171914D935D936D937D9302
:10D6A0000196F1CF232BA1F46DC0F701D10181E0E8
:10D6B00090E06F85788968177907A4F341915191BB
:10D6C000619171914D935D936D937D930196F1CF2F
:10D6D000A985BA85A095B095AA0FBB1FAA0FBB1F3D
:10D6E000BE83AD839301220F331F220F331FEBA1A3
:10D6F000FCA1E20FF31FFAABE9AB49855A854F5FF6
:10D700005F4FC3010197849F5001859FB00C949F88
:10D71000B00C1124AA0CBB1CAA0CBB1C4B855C854D
:10D72000A40EB51EB601620F731FA985BA858A9F24
:10D7300040018B9F900C9A9F900C1124860C971C93
:10D74000880C991C880C991C840E951E18A61FA283
:10D750001EA21DA21E861D86E1E0F0E0FA83E98389
:10D76000645071097CA76BA7F4E08F1A91082F858C
:10D770003889261937093CAB2BABA981BA816A16C7
:10D780007B0634F48D899E89892B09F07CC09CC06E
:10D79000E9A9FAA94D855E85E40FF51F3497C0808D
:10D7A000D180E280F38020E030E0A901C701B6011A
:10D7B0000E942FDB882309F44CC06DA17EA16A0D65
:10D7C0007B1D7AA769A7DB018D919D910D90BC917E
:10D7D000A02D8DA79EA7AFA7B8ABFB01C082D182B9
:10D7E000E282F38201E010E02BA53CA54D855E8529
:10D7F000240F351F3A8B298B41E050E06FA178A5AB
:10D80000680D791D78876F838BA99CA9A981BA813E
:10D810008A0F9B1F9C838B8323DC9058A701960162
:10D820000E9436DBAB01BC01CC24C394D12CE98827
:10D83000FA882F8138858B819C81B2DA2DA53EA58F
:10D840004FA558A9A9A5BAA52D933D934D935C93D7
:10D850001397E981FA813196FA83E9832D853E8514
:10D86000245031093E872D874DA15EA16D817E81B7
:10D87000460F571F5EA34DA38FA198A5860F971F34
:10D8800098A78FA37ACF2BA13CA138872F83A98497
:10D89000BA843FEFA31AB30AAA0CBB1CAA0CBB1C88
:10D8A0004B855C855A8349836F8578897E836D8338
:10D8B0003E862D864A0181E090E09C838B838B819C
:10D8C0009C816816790634F4E9A1FAA1EF2B09F0DE
:10D8D0006DC060C0AF81B885CD90DD90ED90FD90BA
:10D8E000B887AF8320E030E0A901C701B6010E94EC
:10D8F0002FDB8823A9F1A981BA812D913D914D910A
:10D900005C911397298B3A8B4B8B5C8BFD01C0820A
:10D91000D182E282F38201E010E02D853E8541E074
:10D9200050E0B4018D819E819BDB9058A701960148
:10D930000E9436DBAB01BC01CC24C394D12CED8416
:10D94000FE8494018D819E812BDA29893A894B8945
:10D950005C89A981BA812D933D934D935C93139774
:10D96000EB81FC813196FC83EB8329813A812A0D7E
:10D970003B1D3A8329834D815E81415051095E836D
:10D980004D838A0C9B1C6D857E856C5F7F4F7E87E7
:10D990006D8795CFAF8DB8A1AB2B91F1B1012E96CC
:10D9A0004EAD5FAD2E9721E030E017C0B1014B8D39
:10D9B0005C8D21E030E04216530664F3FB01819157
:10D9C0009191A191B191BF01FA0181939193A1939A
:10D9D000B193AF012F5F3F4FEECF421653060CF4C9
:10D9E00041C0FB0181919191A191B191BF01FA01D7
:10D9F00081939193A193B193AF012F5F3F4FEDCFEF
:10DA0000ED8DFE8DEF2BC1F12F853889421653061F
:10DA1000E4F59201B201660F771F660F771FA1012F
:10DA2000460F571F2C968EAD9FAD2C97680F791F10
:10DA300080E090E02F5F3F4FAF85B889A217B30712
:10DA40000CF4F2C1FA01E80FF91FC080D180E28026
:10DA5000F380FB01E80FF91FC082D182E282F382DA
:10DA60000496E8CF2D8D3E8D232B71F6EF85F88936
:10DA70004E165F060CF4DDC1A9A1BAA1AB2BA1F42F
:10DA800062C08D8D9E8D892BB9F32C96EEADFFADC6
:10DA90002C9781E090E04816590674F31192119288
:10DAA000119211920196F7CFF201EE0FFF1FEE0FC8
:10DAB000FF1F2B8D3C8D2E0F3F1F3A8329832CEFA8
:10DAC00049855A852403B001259F700D11247AA33E
:10DAD00069A340955095440F551F440F551F5E8B09
:10DAE0004D8B29853A852F5F3F4FC2010197829F59
:10DAF0004001839F900C929F900C1124880C991CDC
:10DB0000880C991CAB85BC858A0E9B1EE985FA851D
:10DB10008E9F50018F9FB00C9E9FB00C1124AA0CB9
:10DB2000BB1CAA0CBB1CAA0EBB1E12011A8A198AA6
:10DB300018861F8221E030E03C832B83EB81FC813F
:10DB40004E165F061CF41D821D865CC0A2016B810F
:10DB50007C81461B570B5EA34DA32D823D86E98930
:10DB6000FA89E80DF91DC080D180E280F38020E0C1
:10DB700030E0A901C701B6010E942FDB882309F418
:10DB800041C0A7019601A981BA819E918E917E9193
:10DB90006E91BA83A9830E9436DBE981FA816083A2
:10DBA000718382839383F1E02F16310489F0AB01F6
:10DBB000BC017058CC24C394D12CEB8CFC8C01E0BC
:10DBC00010E02F8138852A0D3B1D8DA19EA1E8D83C
:10DBD0002B813C812F5F3F4F3C832B8331E0231A05
:10DBE00031084F81588569A17AA1460F571F588780
:10DBF0004F8389899A89AD89BE898A0F9B1F9A8B29
:10DC0000898B9CCF2D8D3E8D232B29F44F8D58A1D0
:10DC1000452B09F42DC169857A8560957095660F4D
:10DC2000771F660F771F7A83698389859A850196A6
:10DC3000930121503109289F1001299F300C389FF2
:10DC4000300C1124220C331C220C331C8B859C8538
:10DC5000280E391EC301880F991F880F991FABA189
:10DC6000BCA1A80FB91FBCA3ABA32C96EEADFFAD12
:10DC70002C97E80FF91FF88FEF8B49855A85249F61
:10DC80002001259F500C349F500C1124460C571C2A
:10DC9000440C551C440C551C6B857C85460E571E48
:10DCA0002E96AEADBFAD2E97A80FB91F1C821B825A
:10DCB0001C861B86E1E0F0E0FA87E9871497BA8FAB
:10DCC000A98FF4E04F1A51082F8538892619370992
:10DCD000388B2F874F89588D44505109588F4F8B5F
:10DCE00089859A85681679060CF4C2C0EBA1FCA15F
:10DCF0006B857C85E60FF71F3497C080D180E2806A
:10DD0000F38020E030E0A901C701B6010E942FDBBB
:10DD1000882309F473C0D1018D919D910D90BC9120
:10DD2000A02D898B9A8BAB8BBC8BF101C082D182E9
:10DD3000E282F3822D8D3E8D232B49F101E010E02C
:10DD40004F89588D6B857C85460F571F58874F83A9
:10DD50009A0141E050E08B809C80840C951CB401BA
:10DD6000AF84B88889859A85A80EB91EC50178D96F
:10DD70009058A70196010E9436DBAB01BC01CC2470
:10DD8000C394D12CEF80F8849401C50109D8AF8DDC
:10DD9000B8A1AB2B49F101E010E0E98CFA8CEB85DE
:10DDA000FC85EE0EFF1E970141E050E08B809C80C9
:10DDB000840C951CB401AF84B88889859A85A80E17
:10DDC000B91EC5014DD99058D1012D913D914D916C
:10DDD0005C910E9436DBAB01BC01CC24C394D12CF6
:10DDE0009401C5010E94D06629893A894B895C89D2
:10DDF000D1012D933D934D935C931397E985FA855B
:10DE00003196FA87E9872B853C85245031093C8778
:10DE10002B8749815A81240E351E6B817C81640FCA
:10DE2000751F7C836B835CCFAF8DB8A1AB2B09F4DE
:10DE30002CCEC201A201440F551F440F551F2E9630
:10DE40002EAD3FAD2E97420F531F20E030E00196DC
:10DE50006F857889681779070CF413CEFA01E20F01
:10DE6000F31F10821182128213822C5F3F4FEFCF7B
:10DE70008D819D85E4960FB6F894DEBF0FBECDBFB1
:10DE8000DF91CF911F910F91FF90EF90DF90CF9096
:10DE9000BF90AF909F908F907F906F905F904F90CA
:10DEA0003F902F9008952F923F924F925F926F92E2
:10DEB0007F928F929F92AF92BF92CF92DF92EF921A
:10DEC000FF920F931F93CF93DF931F921F92CDB7B3
:10DED000DEB73A8329833801260165011401011553
:10DEE000110591F01F922EE62F93DF92AF92DF92F1
:10DEF000AF924201088D198D9301DEDA0F900F90D9
:10DF00000F900F900F900F90F10180E090E0298129
:10DF10003A81821793074CF4208131813195219504
:10DF20003109219331930196F2CF9301220F331FD0
:10DF3000220F331F240D351D80E090E0A981BA81A6
:10DF40006A167B0664F4F901E80FF91F108211824A
:10DF5000128213824FEF641A740A0496EFCF3201D3
:10DF6000B10141E050E0E981FA81E417F507E4F1FD
:10DF7000FB01208131811216130674F13195219530
:10DF80003109318320832417350731F1D3018D9076
:10DF90009D90AD90BC901397F901E150F04CEE0FBD
:10DFA000FF1FEE0FFF1FE40DF51DC080D180E28042
:10DFB000F380CD92DD92ED92FC9213978082918254
:10DFC000A282B382F901E150F048EE0FFF1FE20D8B
:10DFD000F31D20813181D2CF4F5F5F4F6E5F7F4F46
:10DFE000B4E06B0E711CBFCF0F900F90DF91CF91FB
:10DFF0001F910F91FF90EF90DF90CF90BF90AF9067
:10E000009F908F907F906F905F904F903F902F9058
:10E0100008952F923F924F925F926F927F928F92CC
:10E020009F92AF92BF92CF92DF92EF92FF920F93A7
:10E030001F93CF93DF934C016A017B0139011816BE
:10E0400019060CF0A3C00130110509F069C065E0A4
:10E0500070E00E94EDDEEC012C01590100E010E0BF
:10E060000C171D0794F4A7019601F50160817181D9
:10E07000828193810E9404DEF50161937193819303
:10E0800091935F010F5F1F4FEBCFCC0FDD1FCC0FC4
:10E09000DD1FC60DD71D481459040CF077C0A70129
:10E0A0009601688179818A819B810E9404DE688360
:10E0B00079838A839B83A70196016C817D818E8100
:10E0C0009F810E9404DE6C837D838E839F83A701E2
:10E0D0009601688579858A859B850E9404DE68871C
:10E0E00079878A879B87A70196016C857D858E85B8
:10E0F0009F850E9404DE6C877D878E879F87A7019E
:10E100009601688979898A899B890E9404DE688BD7
:10E11000798B8A8B9B8BF5E04F0E511C6496BBCF9D
:10E1200017FF0CC081E090E088199909809F2001B9
:10E13000819F500C909F500C112402C0412C512CF7
:10E140001801220C331C220C331C440C551C440CAB
:10E15000551C460C571C00E010E0C0E0D0E0520116
:10E16000A00EB11EA7019601F50160817181828127
:10E1700093810E9404DEF50160837183828393831F
:10E180002196020D131DC815D90549F7DF91CF91CE
:10E190001F910F91FF90EF90DF90CF90BF90AF90C5
:10E1A0009F908F907F906F905F904F903F902F90B7
:10E1B00008952F923F924F925F926F927F928F922B
:10E1C0009F92AF92BF92CF92DF92EF92FF920F9306
:10E1D0001F93CF93DF93CDB7DEB7E8970FB6F894D0
:10E1E000DEBF0FBECDBF98878F83788F6F8B3A01CC
:10E1F0003A8B298B1AA709A7FE8EED8EDCA6CBA63B
:10E20000AB2809F4C7C06C0144244394512C01E0AD
:10E2100010E029893A89201731070CF44BC0D70147
:10E220008D919C91119797FF07C088279927801B94
:10E23000910B8D939C9335C0F70111830083892B3B
:10E2400081F104151505D1F0C20101972F89388D90
:10E25000829FB001839F700D929F700D1124660FF5
:10E26000771F660F771F4F815885640F751F16142F
:10E27000170424F4A601C3010E944265F201E15093
:10E28000F048EE0FFF1F8D8D9E8DE80FF91F8081E6
:10E290009181D7018D939C9311830083BFEF4B1A1B
:10E2A0005B0A0F5F1F4FE2E0EE0EF11CF4E0CF0EB1
:10E2B000D11CAFCF8901000F111F4D8D5E8D040F52
:10E2C000151F2CEF4F89588D24035001259FB00C4A
:10E2D000112489899A890197849F7001859FF00C88
:10E2E000949FF00C1124EE0CFF1CEE0CFF1C8F8190
:10E2F0009885E80EF91E29883A886101812C912CB5
:10E300001C141D040CF04BC0D8019E918E918D0100
:10E3100097FF3AC09195819591098D939C93C21472
:10E32000D30479F1A4014E0D5F1DC1010197EF895E
:10E33000F88D8E9FB0018F9F700D9E9F700D1124E0
:10E34000660F771F660F771F2F813885620F731F47
:10E35000161417041CF4C3010E944265F101E15038
:10E36000F048EE0FFF1F4D8D5E8DE40FF51F80818D
:10E370009181D8012D913C911197318320838D9308
:10E380009C93B1E02B1A3108E1E0CE1AD1088A0C37
:10E390009B1CB6CF212C312C44244394512C2F8923
:10E3A000388D220F331F220F331F3A8F298FAF80F2
:10E3B000B884A21AB30A9201215031094F89588DAD
:10E3C000249FC001259F900D349F900D1124880F2C
:10E3D000991F880F991FA80EB91E8201000F111FE7
:10E3E000000F111F89A49AA4800E911E9201E12CA6
:10E3F000F12CC12CD12C898D9A8DC80ED91E94E098
:10E40000E90EF11C22163306BCF041E050E0B501E4
:10E410006C0D7D1DC3012FAB38AF0E948A69F401DA
:10E42000EE0DFF1D389760837183828393832FA93C
:10E4300038AD2F5F3F4FDFCFABA5BCA5A00FB11FFD
:10E44000920180E090E00496221633069CF0F401DD
:10E45000E80FF91F38974081518162817381FD0176
:10E46000E80FF91F389740835183628373832F5FCE
:10E470003F4FE9CFA989BA89B8ABAFA76A167B0627
:10E4800014F478AA6FA6E98DFA8D3496FEA7EDA74D
:10E4900029A53AA53C8F2B8F4BA55CA558A34F8F80
:10E4A000C30101979AA389A3AF81B885B8A7AFA389
:10E4B000BA83A9834D01AA24A394B12C4FA558A9CE
:10E4C0004A155B050CF45CC2A414B5040CF4A0C09E
:10E4D000A214B3040CF09CC0BAAAA9AA7501C12C5D
:10E4E000D12C1B8A1B821D8A10E0EB8DFC8D34968B
:10E4F000FCA3EBA3EBA1FCA1EC0DFD1D3497208147
:10E50000298731813B8742814F870381502F6B8957
:10E510007B818D89912F0E942FDB87FD08C05B894D
:10E5200059878B818B879D899F87012F02C0FAAA0B
:10E53000E9AAAFEFEA1AFA0AB4E0CB0ED11C2E1406
:10E540003F0444F0E985EB8BFB85FB832F852D8B06
:10E55000102FD0CF49A95AA94A155B0509F458C014
:10E56000CA010197AF89B88D8A9FA0018B9F500D7A
:10E570009A9F500D1124440F551F440F551FEF81D2
:10E58000F8854E0F5F1F161417042CF46FA178A5A1
:10E59000C3010E94426589A99AA98150904C880FB5
:10E5A000991F880F991FAB8DBC8D4D915D916D9119
:10E5B0007C91E9A5FAA5E80FF91F40835183628396
:10E5C0007383EF8DF8A14081518162817381EBA546
:10E5D000FCA5E80FF91F408351836283738349A927
:10E5E0005AA941505048440F551F2D8D3E8D420F62
:10E5F000531FDA018D919C911197F501EE0FFF1FCA
:10E60000E20FF31F329122912D933C9391838083EB
:10E61000EB8DFC8D1192119211921192FC8FEB8F68
:10E62000A614B70409F48BC129A13AA12F5F3F4F6B
:10E630003E8B2D8B41E050E0B401C9010E948A69F4
:10E640006B877C878D879E8720E030E0A9010E9440
:10E650002FDB882309F473C1A981BA81CD90DD90A5
:10E66000ED90FC9020E030E0A901C701B6010E94C6
:10E670002FDB8823E1F020E030E0A901C701B601DB
:10E680000E942FDB87FF05C020E030E040E85FEB11
:10E6900004C020E030E040E85FE36B857C858D8539
:10E6A0009E850E9404DE6B877C878D879E872B85E5
:10E6B0003C854D855E8560E070E080E89FE30E94C8
:10E6C00036DBAB01BC0101E010E094018D899E892D
:10E6D000A0DC20E030E040E85FE3E981FA8160817E
:10E6E0007181828193810E9456DAA981BA816D93EA
:10E6F0007D938D939C931397F5013196FA87E98763
:10E70000298D3A8D280D391D3EAB2DAB4F8D58A16B
:10E710004C5F5F4F5C8B4B8B8B8D9C8D988B8F8769
:10E7200029853A8549895A89421753070CF4EDC067
:10E7300001E010E02DA93EA941E050E0B4018D892F
:10E740009E890E9430689058A981BA812D913D918F
:10E750004D915C910E9436DBAB01BC01CC24C3948B
:10E76000D12CEDA8FEA894018D899E890E94D066C7
:10E77000E985FA85E415F5050CF4ADC02E163F06C3
:10E780000CF4A9C0AF85B8892D913D914D915C9154
:10E790002B833C834D835E8320E030E0A9016B81B5
:10E7A0007C818D819E810E942FDB882309F493C098
:10E7B000EDA9FEA9C080D180E280F38020E030E0A6
:10E7C000A901C701B6010E9432DD87FF04C0F7FA34
:10E7D000F094F7F8F0942B813C814D815E81C70164
:10E7E000B6010E9436DB9B01AC010E9404DE9B0156
:10E7F000AC0160E070E080E89FE30E9455DA6B01B5
:10E800007C0120E030E0A9010E9432DD18161CF0E6
:10E81000C12CD12C7601AB89BC892D913D914D91B4
:10E820005C916B817C818D819E810E9436DB6BA324
:10E830007CA38DA39EA32DEC3CEC4CE45DE3C701CF
:10E84000B6010E9404DE69AB7AAB8BAB9CAB2BA10B
:10E850003CA14DA15EA1CA01B9010E9404DE9B0149
:10E86000AC0169A97AA98BA99CA90E9404DE20E0C9
:10E8700030E040E85FE30E9456DA20E030E040E814
:10E880005FE30E942FDB882379F0C701B6010E9465
:10E8900071DE9B01AC016B817C818D819E810E9428
:10E8A00004DEEF85F88913C041E050E06DA97EA930
:10E8B0006C5F7F4F89A19AA10E948A69AF85B88950
:10E8C0006D937D938D939C931397EB89FC89608363
:10E8D00071838283938329853A852F5F3F4F3A87DF
:10E8E00029874F8558894C5F5F4F588B4F878B899D
:10E8F0009C8904969C8B8B8BADA9BEA9E98DFA8D62
:10E90000AE0FBF1FBEABADAB0BCFE981FA818081EB
:10E910009181A281B3812B8D3C8D24503109F90165
:10E9200080839183A283B3838B859C85AD85BE85CF
:10E93000B058E981FA8180839183A283B383FFEF8A
:10E94000AF1ABF0A2DA53EA5820E931E49815A819A
:10E95000420F531F5A8349838F8D98A1049698A321
:10E960008F8FAFA1B8A5E98DFA8DAE0FBF1FB8A7E5
:10E97000AFA329A13AA1215031093AA329A39ECDE1
:10E98000E8960FB6F894DEBF0FBECDBFDF91CF91F2
:10E990001F910F91FF90EF90DF90CF90BF90AF90BD
:10E9A0009F908F907F906F905F904F903F902F90AF
:10E9B00008952F923F924F925F926F927F928F9223
:10E9C0009F92AF92BF92CF92DF92EF92FF920F93FE
:10E9D0001F93CF93DF93CDB7DEB72C970FB6F89484
:10E9E000DEBF0FBECDBF9A8389837E836D831A01FC
:10E9F0003901E986FA860B871C87D886CF82750194
:10EA00008401F50180E090E08615970524F41192C9
:10EA100011920196F9CFC301880F991F880F991F92
:10EA20000E9467DF9C838B83AA24A394B12C6C0182
:10EA30009301A1016D817E8189819A81BADBEF8189
:10EA4000F885118210822301261437040CF4210169
:10EA50000D811E810F5F1F4F000F111F000F111F2F
:10EA600029803A80612C712C641475040CF03FC02D
:10EA7000F101C080D180E280F38020E030E0A90184
:10EA8000C701B6010E9432DD87FF04C0F7FAF09497
:10EA9000F7F8F094E981FA8180809180A280B380B8
:10EAA00020E030E0A901C501B4010E9432DD87FFFA
:10EAB00004C0B7FAB094B7F8B094200E311EA50187
:10EAC000940169857A858B859C850E9404DE9B0173
:10EAD000AC01C701B6010E942FDB181624F5FFEF29
:10EAE0006F1A7F0AEF81F88571826082BDCF8B81BA
:10EAF0009C812C960FB6F894DEBF0FBECDBFDF9180
:10EB0000CF911F910F91FF90EF90DF90CF90BF902A
:10EB1000AF909F908F907F906F905F904F903F90BD
:10EB20002F900C94FFDF2C960FB6F894DEBF0FBE2B
:10EB3000CDBFDF91CF911F910F91FF90EF90DF90AC
:10EB4000CF90BF90AF909F908F907F906F905F908D
:10EB50004F903F902F9008952F923F924F925F9247
:10EB60006F927F928F929F92AF92BF92CF92DF92DD
:10EB7000EF92FF920F931F93CF93DF93CDB7DEB742
:10EB80002A970FB6F894DEBF0FBECDBF9A83898354
:10EB90002B011A013901DC82CB82B886AF829A86BA
:10EBA00089868CA18D839DA19E838EA19FA16417D0
:10EBB000750754F11216130654F51816190654F574
:10EBC000019739F48D809E80AAA0BBA089819A818B
:10EBD000F0DEEB81FC8100811181FE81FF938D814C
:10EBE0008F938AA09BA0A8A0B9A0C984DA84EF80E3
:10EBF000F8849301A101B20189819A8154D90F90BF
:10EC00000F9080E090E008C08FEF9FEF05C08EEF7F
:10EC10009FEF02C08DEF9FEF2A960FB6F894DEBFEC
:10EC20000FBECDBFDF91CF911F910F91FF90EF905D
:10EC3000DF90CF90BF90AF909F908F907F906F901C
:10EC40005F904F903F902F9008952F923F924F9258
:10EC50005F926F927F928F929F92AF92BF92CF926C
:10EC6000DF92EF92FF920F931F93CF93DF93CDB775
:10EC7000DEB72E970FB6F894DEBF0FBECDBF3C01B6
:10EC80002B0159010E9467661C01AC01B201C3014E
:10EC90000E94D0659B01AC018201000F111F000F83
:10ECA000111FC8012B873C874D875E870E9467DF55
:10ECB0009C838B83C201880F991F0E9467DF8D831D
:10ECC0009E83C8010E9467DF8F839887C301880FE6
:10ECD000991F880F991F0E9467DF89879A872B8564
:10ECE0003C854D855E8560E070E080E895E20E949D
:10ECF00036DB1F9221E02F9328852F933F813F938E
:10ED00002E812F933D813F932A852F9339853F9301
:10ED10008B809C809E012F5F3F4F69017B018C019E
:10ED20009201A301B301C10117DFC1010E94FFDFFE
:10ED30008D819E810E94FFDF8F8198850E94FFDF79
:10ED400089859A850E94FFDF0FB6F894DEBF0FBE5B
:10ED5000CDBF8B819C812E960FB6F894DEBF0FBE7F
:10ED6000CDBFDF91CF911F910F91FF90EF90DF907A
:10ED7000CF90BF90AF909F908F907F906F905F905B
:10ED80004F903F902F9008958FEF8EBD0DB407FEEA
:10ED9000FDCF8EB508958EBD0DB407FEFDCF08954D
:10EDA00061E0FC0180810C9438D6FC012281322F75
:10EDB000306A36953CBD20FD06C031E0263009F4AE
:10EDC00030E0232F01C020E02DBD60E0FC018081F8
:10EDD0000C9438D6CF92DF92EF92FF920F931F934D
:10EDE000CF93DF93EC018B017A010E9427D46B0152
:10EDF000CBDF8B838F3F49F40E9427D46C197D09A8
:10EE00006D327140A8F381E103C08E3F31F08FE095
:10EE10008983CE01C5DF80E024C0E114F104E1F074
:10EE200081E0E81AF1088FEF8EBDF8012FEFCF01D6
:10EE3000801B910B8E159F0538F40DB407FEFDCF96
:10EE40008EB581932EBDF3CF0DB407FEFDCF8EB5E9
:10EE5000F801EE0DFF1D808397DF96DFCE01A0DF66
:10EE600081E0DF91CF911F910F91FF90EF90DF90A4
:10EE7000CF9008950F931F93CF93DF93EB010E94E0
:10EE800027D48B0181DF8F3F49F00E9427D4601B7C
:10EE9000710B6C177D07B0F380E001C081E0DF915A
:10EEA000CF911F910F910895CF92DF92FF920F9310
:10EEB0001F93CF93DF9300D01F92CDB7DEB76C01C5
:10EEC000F62E29833A834B835C836FDF6CE271E01B
:10EED000C601D0DF8F2D80645EDF08E110E05C8129
:10EEE0004B813A812981DA01C901002E04C0B6950F
:10EEF000A795979587950A94D2F729833A834B83F0
:10EF00005C8349DF0850110929813A814B815C817A
:10EF1000083F8FEF180739F7FF2029F0E8E0FE16C9
:10EF200021F08FEF03C085E901C087E834DFFCE002
:10EF3000FF1201C029DF10E027DFF601838387FF7E
:10EF400004C01F3F11F01F5FF7CF0F900F900F907D
:10EF50000F90DF91CF911F910F91FF90DF90CF9095
:10EF60000895BF92CF92DF92EF92FF920F931F937B
:10EF7000CF93DF93EC01B62E1C82198248830E9446
:10EF800027D48B0161E088810E94FFD5CE0108DF84
:10EF900060E082E30E94FFD561E083E30E94FFD539
:10EFA00061E084E30E94FFD561E085E30E94FFD524
:10EFB00061E085E30E9438D685E08A8382E58CBDD6
:10EFC0001DBC2AE0F22E8FEFE6DEFA94E1F720E096
:10EFD00030E0A90160E0CE0167DFF82E8B8381E08D
:10EFE000F81649F00E9427D4601B710B613D7740F1
:10EFF00070F381E046C02AEA31E040E050E068E08A
:10F00000CE0152DF82FF02C0FC820CC094E0F92ED8
:10F01000BBDE8B83FA94E1F78A3A11F082E031C0CB
:10F0200082E08C838C81823031F4C12CD12CE12C94
:10F0300080E4F82E03C0C12CD12C760120E030E012
:10F04000A90167E3CE0130DFA701960169E2CE0195
:10F050002BDF8B83882349F00E9427D4601B710B20
:10F06000613D774058F38AE00CC08C818230B1F466
:10F0700020E030E0A9016AE3CE0116DF882329F001
:10F0800088E08983CE018CDE14C07EDE807C803CEB
:10F0900011F483E08C8378DE77DE76DECE0180DECD
:10F0A00086E08B1518F488E1898303C0BA8281E079
:10F0B00001C080E0DF91CF911F910F91FF90EF9001
:10F0C000DF90CF90BF9008950F931F93CF93DF935E
:10F0D000EC0189018C81833039F039E0440F551FF0
:10F0E000661F771F3A95D1F79A01AB0161E1CE0116
:10F0F000DBDE811109C040E052E0B801CE01DF91B2
:10F10000CF911F910F9166CE84E08983CE0148DEB6
:10F1100080E0DF91CF911F910F910895CF93DF93FE
:10F12000EC016EBD20E030E00DB407FEFDCFFA012A
:10F13000E20FF31F80818EBD0DB407FEFDCF8181EC
:10F140008EBD2E5F3F4F211582E0380769F70DB461
:10F1500007FEFDCF8FEF1FDE8FEF1DDE15DE8B83E9
:10F160008F71853031F083E18983CE0119DE80E033
:10F1700001C081E0DF91CF9108950F931F93CF934A
:10F18000DF93EC0189018C81833039F089E0440FF1
:10F19000551F661F771F8A95D1F79A01AB0168E169
:10F1A000CE0182DE882311F086E01EC0A8016EEF3A
:10F1B000CE01B4DF8823C9F068E572E0CE015ADEE3
:10F1C000182F811102C087E10FC020E030E0A901B3
:10F1D0006DE0CE0169DE811106C0D6DD811103C06C
:10F1E000CE01DEDD05C086E18983CE01D9DD10E0E8
:10F1F000812FDF91CF911F910F910895CF93DF93CE
:10F20000EC019C012C5F3F4F41E050E060E070E07A
:10F21000898D9A8D0E94BA83882399F04D895E89E1
:10F220006F89788D452B462B472B59F44C815D8196
:10F230006E817F814D8B5E8B6F8B788F998190680B
:10F240009983DF91CF910895CF92DF92EF92FF9251
:10F250000F931F93CF93DF93EC0189899A89AB8930
:10F26000BC89803E9F4FAF41B10510F080E06AC07D
:10F27000CE01C4DF8823D1F30E94CE81182F8823CA
:10F28000A9F3E98DFA8DCC80DD80EE80FF8032E03D
:10F29000C31AD108E108F108058404C0CC0CDD1CB8
:10F2A000EE1CFF1C0A94D2F786859785A089B18948
:10F2B000C80ED91EEA1EFB1E81E08093490FC09242
:10F2C0004C11D0924D11E0924E11F0924F1180E00E
:10F2D00092E0ECE4FFE0DF019C011D922150304000
:10F2E000E1F701E0E98DFA8D8481081788F42CE4B8
:10F2F0003FE0B701A601400F511D611D711D8091B6
:10F300004A0F90914B0F39DF8823E1F00F5FEACF6E
:10F31000C12C82E0D82EE12CF12C058404C0CC0C49
:10F32000DD1CEE1CFF1C0A94D2F749895A896B89AF
:10F330007C894C0D5D1D6E1D7F1D498B5A8B6B8B1F
:10F340007C8B812FDF91CF911F910F91FF90EF90D8
:10F35000DF90CF900895CF93DF93EC0141E06111EE
:10F3600001C040E06C857D858E859F850E940E8260
:10F37000882341F0888920E2829FC0011124845BA8
:10F38000904F02C080E090E0DF91CF91089530E08F
:10F3900020E04EE2DC015C91503271F0383029F40B
:10F3A000FB01E20FF11D40832F5FFB01E20FF11D16
:10F3B000DC015C9150832F5F3F5F01963B3051F73A
:10F3C000FB01E20FF11D10820895CF93DF93EB0153
:10F3D000FC012381211102C080E00EC022502230A6
:10F3E00020F48FE28883198206C060E0B4DF0097C2
:10F3F00099F3BE01CCDF81E0DF91CF910895FB014D
:10F400002BE030E231932150E9F7DC0190E027E076
:10F410003A2FEB2F8D9181110AC0DA013C9311969E
:10F42000EC9381E0FB019081903239F525C08F3259
:10F43000A1F38E3219F0E7E8FCE008C02A30E1F0D1
:10F4400098E02AE0E5CF31963817B1F034913111C8
:10F45000FACF291788F03FED380F3E3568F431E0D8
:10F46000390FFB01E90FF11D9FE9980F9A3108F45C
:10F4700080528083932FCCCF80E008950F931F9309
:10F48000CF93DF93EC018B018B81882311F080E017
:10F4900042C0FB018789803139F18032C1F783E0B6
:10F4A0008B83F801428D538D648D758D4D8B5E8BF2
:10F4B0006F8B788F9E012F5E3F4FC8010E94C582DF
:10F4C000882329F31A8F098F81E089831C821D828A
:10F4D0001E821F82188619861A861B861C861D8628
:10F4E0001E861F86188A17C082E08B831D8A1E8A9B
:10F4F0001F8A188EFB01408D518D60E070E095E011
:10F50000440F551F661F771F9A95D1F7498B5A8B69
:10F510006B8B7C8BD7CFDF91CF911F910F9108958B
:10F520002F923F924F925F926F927F928F929F9213
:10F53000AF92BF92CF92DF92EF92FF920F931F9301
:10F54000CF93DF93EC015B016A018B81811103C0D2
:10F550008FEF9FEFC6C0898180FFFACF49895A8912
:10F560006B897C8988859985AA85BB852601612C54
:10F57000712C8A019B01081B190B2A0B3B0B4016AF
:10F5800051066206730618F06A01C81AD90A760194
:10F590003E0124E0620E711CE114F10409F476C00E
:10F5A000488559856A857B854A0181E098222B81AF
:10F5B0001A012B01E9E05694479437942794EA9571
:10F5C000D1F7898D9A8DFC01223049F4628D738DBB
:10F5D000848D958D620D731D841D951D3CC0148115
:10F5E0001150122181149104C1F4111116C0452B40
:10F5F000462B472B49F48D899E89AF89B88D8C8322
:10F600009D83AE83BF8309C04C815D816E817F8104
:10F6100093013CD7882309F49BCFE98DFA8D6C8147
:10F620007D818E819F8162507109810991090584D4
:10F6300004C0660F771F881F991F0A94D2F726858A
:10F64000378540895189620F731F841F951F610F91
:10F65000711D811D911D20E032E0281939098701B3
:10F660002E153F0508F489010115F2E01F0761F529
:10F6700020914C1130914D1140914E1150914F11EC
:10F68000621773078407950719F41EC0C60129C0C5
:10F690009501AB01BC0180914A0F90914B0F14DD95
:10F6A000882309F455CFA00EB11E88859985AA85B7
:10F6B000BB85800F911FA11DB11D88879987AA87DF
:10F6C000BB87E01AF10A68CF40E0A8D6882309F486
:10F6D0003FCFB401645B704FA801C5010E9495E360
:10F6E000E2CFDF91CF911F910F91FF90EF90DF90CC
:10F6F000CF90BF90AF909F908F907F906F905F90D2
:10F700004F903F902F900895CF93DF931F92CDB7E6
:10F71000DEB741E050E0BE016F5F7F4F01DF019730
:10F7200019F4898190E002C08FEF9FEF0F90DF9175
:10F73000CF910895CF92DF92EF92FF920F931F9394
:10F74000CF93DF936C01EB017A01FC01838182305E
:10F7500060F000851185228533850F7111272227DE
:10F760003327012B022B032B11F08FEF5CC04115C7
:10F77000510511F0F70110821DE040E250E0BE019A
:10F78000C601CEDE8032910539F021E0892B09F4E3
:10F7900020E0822F819547C028812223C1F0253E99
:10F7A00061F32E3251F33B853F733F3061F4E11436
:10F7B000F10449F04A8D5B8D452B29F42F713FEF01
:10F7C000320F323030F02B8523FDD7CF2CC080E0B4
:10F7D0002AC030E021503109129FC001139F900DC3
:10F7E0001124F701E80FF91F298120832B81218340
:10F7F0002D8122832F812383298524832E852583B0
:10F80000288926832A8927832C8920872E89218786
:10F81000288D22872C8D23872E8D2487288126FFF3
:10F82000D2CF1586D0CFDF91CF911F910F91FF904E
:10F83000EF90DF90CF9008951F93CF93DF93EC016B
:10F840008B81823018F480E090E023C04885598590
:10F850006A857B85A5E07695679557954795AA9526
:10F86000D1F7142F1F70CE014FDF97FDECCF4885E5
:10F8700059856A857B85415E5F4F6F4F7F4F488713
:10F8800059876A877B8720E2129FC0011124845B1D
:10F89000904FDF91CF911F9108954F925F926F9299
:10F8A0007F92AF92BF92CF92DF92EF92FF920F932F
:10F8B0001F93CF93DF93EC016A017B012B812223FD
:10F8C00049F089899A89AB89BC8984179507A6076D
:10F8D000B70710F480E06BC0223009F463C0C11494
:10F8E000D104E104F10449F41C821D821E821F82AE
:10F8F000188619861A861B8659C088859985AA8517
:10F90000BB85E98DFA8DE585F0E03996AC01BD0146
:10F9100041505109610971090E2E04C07695679511
:10F92000579547950A94D2F797018601015011091E
:10F930002109310904C03695279517950795EA9551
:10F94000D2F7041715072607370720F0892B8A2BD3
:10F950008B2B49F48D899E89AF89B88D8C839D83CB
:10F96000AE83BF8304C0041B150B260B370B280185
:10F9700039015E0184E0A80EB11C411451046104F8
:10F98000710481F04C815D816E817F819501898D4B
:10F990009A8D7CD591E0491A51086108710881114E
:10F9A000ECCF05C0C886D986EA86FB8681E0DF9168
:10F9B000CF911F910F91FF90EF90DF90CF90BF906C
:10F9C000AF907F906F905F904F9008950F931F932B
:10F9D000CF93DF93EC018B818823D1F1898187FF5D
:10F9E00032C061E0CE01B7DC8C01009789F1FC01E7
:10F9F0008081853E69F18B81823040F449895A8942
:10FA00006B897C89448F558F668F778F4D895E898E
:10FA10006F89788DF801538F428F758B648BE091DD
:10FA2000430FF091440F309759F0B8016A5E7F4F51
:10FA3000C80148961995F801808D918D938B828B22
:10FA400089818F778983DF91CF911F910F91A6C410
:10FA500081E0888380E0DF91CF911F910F9108951D
:10FA6000CF93DF93EC01B2DF1B82DF91CF9108953A
:10FA7000FC0123812111F4CF08954F925F926F9280
:10FA80007F92AF92BF92CF92DF92EF92FF920F934D
:10FA90001F93CF93DF9300D01F92CDB7DEB75C01E9
:10FAA0006A017B01FC0183818130E9F4818181FF5E
:10FAB0001AC0F50181899289A389B48984179507B1
:10FAC000A607B70780F0892B8A2B8B2B09F472C00D
:10FAD000F5014084518462847384B701A601C50195
:10FAE000DCDE811102C080E066C0F501818D928D5F
:10FAF000C114D104E104F10469F445895689678988
:10FB0000708D41D7882379F3F501158A168A178AF3
:10FB1000108E37C0F50144815581668177819E0141
:10FB20002F5F3F4FB3D48823F1F249815A816B8113
:10FB30007C81F501818D928DFC012789203139F47A
:10FB4000483FFFEF5F0761057105D8F407C0483FE4
:10FB50002FEF520762072FE0720798F414D788231B
:10FB600009F4C1CFF50144815581668177810FEF9A
:10FB70001FEF2FEF3FE0818D928D6DD5882309F423
:10FB8000B2CFF501C18AD28AE38AF48A8181806882
:10FB90008183C5011BDF882309F4A5CFB701A60126
:10FBA0004C145D046E047F0410F4B301A201C5017E
:10FBB00074DE01C081E00F900F900F900F90DF91E5
:10FBC000CF911F910F91FF90EF90DF90CF90BF905A
:10FBD000AF907F906F905F904F900895FF920F933A
:10FBE0001F93CF93DF93EC01F42E80E2689FF00126
:10FBF0001124E45BF04F8385817121F0842F8271A1
:10FC000009F04EC080914C1190914D11A0914E1170
:10FC1000B0914F118C879D87AE87BF87688B4489D1
:10FC2000558960E070E0BA0155274427028D138D95
:10FC300020E030E0402B512B622B732B4D8B5E8BE1
:10FC40006F8B788F8385887151F4048D158D268D87
:10FC5000378D098B1A8B2B8B3C8B81E00BC080314D
:10FC6000F9F49E012F5E3F4F898D9A8D8ED48823A3
:10FC7000B9F084E08B838F2D8F7089831C821D8265
:10FC80001E821F82188619861A861B86F4FE0BC0F8
:10FC900040E050E0BA01CE01F0DE811104C011C095
:10FCA0001B8280E00EC0F5FE0BC049895A896B8922
:10FCB0007C89CE01DF91CF911F910F91FF90EDCD07
:10FCC00081E0DF91CF911F910F91FF900895AF9246
:10FCD000BF92CF92DF92EF92FF920F931F93CF9339
:10FCE000DF937C01EB016A01B22E898D9A8DF701B9
:10FCF000928F818F40E050E0BA01CE01CEDDA12C81
:10FD0000088519852A853B8589899A89AB89BC89AB
:10FD1000081719072A073B07A0F585E036952795B0
:10FD2000179507958A95D1F70F70CE0185DD00975D
:10FD300009F481C0FC012081222311F0253EB9F491
:10FD4000A1100EC040914C1150914D1160914E1177
:10FD500070914F11F7014487558766877787008B2D
:10FD6000FC018081AA24A3948111CACF0AC04BE070
:10FD700050E0BC01C6010E9488E3892B09F0C0CF86
:10FD800058C08B2D8274823409F055C0AA2049F0E6
:10FD9000F701008961E0C701DEDAEC01009769F440
:10FDA0004AC08B81823009F446C0CE014DDA8823E7
:10FDB00009F441C0CCE4DFE000E080E2FE011192F2
:10FDC0008A95E9F78BE0F601DE0101900D928A95A4
:10FDD000E1F7E091430FF091440F309739F0BE0105
:10FDE000625F7F4FCE014096199508C081E298E28C
:10FDF000998B888B80E098E09F878E878889998986
:10FE00009B8B8A8B998F888F8E859F859F8B8E8BFE
:10FE1000C5D2882381F04B2D602FC701DF91CF9190
:10FE20001F910F91FF90EF90DF90CF90BF90AF9018
:10FE3000D5CEB7FEF0CF80E0DF91CF911F910F912B
:10FE4000FF90EF90DF90CF90BF90AF9008953F92DA
:10FE50004F925F926F927F928F929F92AF92BF92DA
:10FE6000CF92DF92EF92FF920F931F93CF93DF9386
:10FE7000CDB7DEB7C354D1090FB6F894DEBF0FBEBD
:10FE8000CDBF5C016B0124965FAF4EAF2497522E1D
:10FE90001C8E1F8E19821C826115710511F410E0F1
:10FEA00073C0FC0183818111FACF2496EEADFFADC2
:10FEB000249780818F3211F076011DC02496EEAD1B
:10FEC000FFAD249780818F3231F431962496FFAFB5
:10FED000EEAF2497F3CFF60183818250823060F336
:10FEE000F601618D728DCE010196C8DA8823B9F2D0
:10FEF000CE0101967C018E01045E1F4F3801FE0188
:10FF000031964F01402E312E19C08823A9F121E0EE
:10FF1000AE01495C5F4FB701C801D9DE882309F4FF
:10FF2000BECFEC14FD0411F0C7019ADD06151705CC
:10FF300001F1942D832D7801092F182FAE014E5B0E
:10FF40005F4FBE01695C7F4F24968EAD9FAD2497B5
:10FF500056DA882309F4A3CF2496EEADFFAD24979B
:10FF600080818F3291F631962496FFAFEEAF2497C1
:10FF7000F3CF982D892DDFCF252DAE01495C5F4F42
:10FF8000B701C501A4DE182FCE01019671DDCE01A7
:10FF90004C966EDD812FCD5BDF4F0FB6F894DEBF40
:10FFA0000FBECDBFDF91CF911F910F91FF90EF90CA
:10FFB000DF90CF90BF90AF909F908F907F906F9089
:10FFC0005F904F903F900895CF93DF93EC0140E016
:10FFD00050E0BA0152DD882361F061E0CE01BBD967
:10FFE000009739F025EEFC0120831B82DF91CF9131
:10FFF000D5C180E0DF91CF9108951F93CF93DF9318
:020000021000EC
:10000000CDB7DEB76B970FB6F894DEBF0FBECDBF8E
:10001000AB0119821C8222E0BC01CE01019617DFE0
:10002000182F882321F0CE010196CEDF182FCE01A4
:1000300001961EDD812F6B960FB6F894DEBF0FBEC2
:10004000CDBFDF91CF911F9108952F923F924F9294
:100050005F926F927F928F929F92AF92BF92CF9258
:10006000DF92EF92FF920F931F93CF93DF9300D015
:100070001F921F92CDB7DEB78C015B013A01DC0104
:1000800013968C9113978130C1F411968C9181FF56
:1000900014C082FF18C0F8014189528963897489AC
:1000A00080859185A285B38584179507A607B70734
:1000B00051F0C801F2DB811106C081E0F8018083B4
:1000C0008FEF9FEF37C1630183C0D80159968D919F
:1000D0009C915A97FC01F481F1501A012B0169E0BF
:1000E00056944794379427946A95D1F7F221FD836B
:1000F0004A0121E09222FF2309F476C080E092E0D9
:100100008819990976018C159D0508F47C01D801A0
:100110005996ED91FC915A9714962D903D904D90E3
:100120005C901797B2E02B1A3108410851080584FA
:1001300004C0220C331C441C551C0A94D2F786853B
:100140009785A089B189280E391E4A1E5B1EED8154
:100150002E0E311C411C511CE114F2E0FF0609F087
:1001600089C080914C1190914D11A0914E11B09188
:100170004F1182159305A405B50569F41092490F36
:100180008FEF9FEFDC0180934C1190934D11A09362
:100190004E11B0934F119501B201A10180914A0F08
:1001A00090914B0F0E94BD78882309F486CFF80107
:1001B00080859185A285B3858E0D9F1DA11DB11DE2
:1001C00080879187A287B387AE0CBF1CCE18DF084B
:1001D000D80118964D915D916D917C911B97C1143A
:1001E000D10409F072CF7AC08114910409F086CF4E
:1001F00014964D915D916D917C9117974115510524
:100200006105710559F455968D919D910D90BC91A4
:10021000A02D0097A105B10539F520C09E012F5FE3
:100220003F4F34D1882309F448CF89819A81AB812B
:10023000BC81F801218D328DF9012789203139F4F3
:10024000883FFFEF9F07A105B10540F40DC0883F2F
:100250002FEF9207A2072FE0B20730F0C8010E94EB
:10026000FE7881114BCF29CFF80184839583A68333
:10027000B78344CF8114910411F5D80118964D919C
:100280005D916D917C911B9751968D919D910D90F3
:10029000BC91A02D481759076A077B0780F07ED0D4
:1002A000882309F40ACF81E08093490F20924C11F2
:1002B00030924D1140924E1150924F1107C041E0C3
:1002C000C201B101ABD0882309F4F7CEA701B50173
:1002D000C401845B904F0E9495E369CF51968D9144
:1002E0009D910D90BC91A02DF80121818417950757
:1002F000A607B70738F4418B528B638B748B206849
:1003000021830CC08091430F9091440F892B31F0D1
:100310006114710419F02068F8012183D801119645
:100320008C9183FD02C0C30105C0C8014FDB811160
:10033000FACFC3CE0F900F900F900F900F90DF91D8
:10034000CF911F910F91FF90EF90DF90CF90BF90D2
:10035000AF909F908F907F906F905F904F903F9065
:100360002F900895CF93DF931F92CDB7DEB76983A7
:1003700041E050E0BE016F5F7F4F049666DE0F9054
:10038000DF91CF910895FB0101900020E9F7AF01C3
:1003900041505109461B570B049657CECF9380917D
:1003A000490F8823B9F140914C1150914D11609142
:1003B0004E1170914F112CE43FE080914A0F9091C3
:1003C0004B0F0E94BD78C82F811102C0C0E023C02E
:1003D0004091450F5091460F6091470F7091480F23
:1003E000411551056105710591F02CE43FE08091C4
:1003F0004A0F90914B0F0E94BD78882339F31092D9
:10040000450F1092460F1092470F1092480F10920E
:10041000490F01C0C1E08C2FCF910895CF92DF9298
:10042000EF92FF92CF936B017C01C42F80914C110E
:1004300090914D11A0914E11B0914F118C159D05C9
:10044000AE05BF05C9F0AADF811102C080E018C067
:100450002CE43FE0B701A60180914A0F90914B0F29
:100460000E946478882391F3C0924C11D0924D1170
:10047000E0924E11F0924F1181E0C1118093490F2B
:10048000CF91FF90EF90DF90CF9008958F929F9241
:10049000AF92BF92CF92DF92EF92FF920F931F9392
:1004A000CF93DF93EC016A017B01890189859A85ED
:1004B000AB85BC850196A11DB11D84179507A607C4
:1004C000B70710F480E054C08F89803129F4992750
:1004D000872F762F652F0BC08032A1F7CB01BA0191
:1004E00027E096958795779567952A95D1F78B881C
:1004F0009C88AD88BE88680D791D8A1D9B1D8090E3
:100500004C1190904D11A0904E11B0904F11681564
:1005100079058A059B0581F48F89803191F4DD246A
:10052000EE24FF24F601EE0FFF1FE45BF04F808105
:100530009181A0E0B0E016C040E070DF8111ECCF07
:10054000C1CFE894C7F8DD24EE24FF24F601EE0FB6
:10055000FF1FEE0FFF1FE45BF04F80819181A281AE
:10056000B381BF70F80180839183A283B38381E05C
:10057000DF91CF911F910F91FF90EF90DF90CF907F
:10058000BF90AF909F908F9008954F925F926F921F
:100590007F92AF92BF92CF92DF92EF92FF920F9332
:1005A0001F93CF93DF9300D01F92CDB7DEB78C019E
:1005B00049835A836B837C835901C12CD12C7601EA
:1005C000412C42E0542E612C712C49815A816B815F
:1005D0007C819E012F5F3F4FC80158DF882341F186
:1005E000D301C201F801058404C0880F991FAA1F16
:1005F000BB1F0A94D2F7C80ED91EEA1EFB1E498102
:100600005A816B817C818789803139F481E0483F50
:100610005F4F6105710538F4D8CF81E0483F5F4FE7
:100620006F4F7F4090F2F501C082D182E282F38267
:100630000F900F900F900F90DF91CF911F910F911E
:10064000FF90EF90DF90CF90BF90AF907F906F9032
:100650005F904F9008954F925F926F927F928F922A
:100660009F92AF92BF92CF92DF92EF92FF920F9341
:100670001F93CF93DF93EC014A015B0128013901FD
:10068000423051056105710508F462C049855A85FB
:100690006B857C854F5F5F4F6F4F7F4F48155905C6
:1006A0006A057B0508F454C08F89803129F4FF2442
:1006B000EB2CDA2CC92C0CC0803209F049C0750132
:1006C000640177E0F694E794D794C7947A95D1F7CC
:1006D0004B895C896D897E89C40ED51EE61EF71E86
:1006E00041E0C701B6019ADE882391F19F899031DC
:1006F00059F49924AA24BB24F401EE0FFF1FE45BF4
:10070000F04F5182408210C0E89487F89924AA24BF
:10071000BB24F401EE0FFF1FEE0FFF1FE45BF04F51
:1007200040825182628273829A89923090F04D8128
:100730005E816F8178854C0D5D1D6E1D7F1D409320
:10074000450F5093460F6093470F7093480F01C0B9
:1007500080E0DF91CF911F910F91FF90EF90DF909C
:10076000CF90BF90AF909F908F907F906F905F9051
:100770004F9008952F923F924F925F926F927F9287
:100780008F929F92AF92BF92CF92DF92EF92FF92A1
:100790000F931F93CF93DF93CDB7DEB72F970FB68D
:1007A000F894DEBF0FBECDBF1C014C875D876E87FE
:1007B0007F873B872A87DC0119960D911D912D912A
:1007C0003C911C970F5F1F4F2F4F3F4F0D831E8390
:1007D0002F833887EA85FB8580809180A280B38053
:1007E00081149104A104B10431F0FFEF8F1A9F0A24
:1007F000AF0ABF0A10C0DC018D909D90AD90BC90F7
:10080000B1E0B9870C851D852E853F850130110526
:100810002105310509F0198675016401412C512C1F
:100820003201F10181859285A385B4854816590668
:100830006A067B0608F04EC00D811E812F81388527
:100840000C151D052E053F0550F4F2E0CF2ED12CDE
:10085000E12CF12CA2E08A2E912CA12CB12C9E012E
:100860002F5F3F4FB701A601C10110DE882391F130
:1008700049815A816B817C81D701C6010196A11DF6
:10088000B11D452B462B472B19F04C015D010FC0C4
:10089000AC01BD01481959096A097B090C851D8500
:1008A0002E853F85401751076207730741F01FEF00
:1008B000411A510A610A710A6C017D01B2CF0FEF32
:1008C0001FEF2FEF3FE0B701A601C101C4DE8D830A
:1008D000811113C01D823DC02601370121E0421A5B
:1008E00051086108710897018601B301A201C10195
:1008F000B2DE882379F3730162018C149D04AE0487
:10090000BF0450F3AA85BB854D915D916D917C919B
:100910004115510561057105A9F4EA85FB858082C1
:100920009182A282B382F985FF2399F00FEF801A9A
:10093000900AA00AB00AD1018D929D92AD92BC920C
:10094000139707C095018401C10185DE8111E5CFB0
:10095000C1CF8D812F960FB6F894DEBF0FBECDBFED
:10096000DF91CF911F910F91FF90EF90DF90CF908B
:10097000BF90AF909F908F907F906F905F904F90BF
:100980003F902F900895AF92BF92CF92DF92EF9257
:10099000FF920F931F93CF93DF9300D01F92CDB799
:1009A000DEB75C016A017B0182E090E0A0E0B0E08C
:1009B000F50180839183A283B3839E012F5F3F4F14
:1009C000B701A601C50162DD811102C080E023C02C
:1009D00000E010E09801B701A601C5013CDE8823C4
:1009E000A9F3C980DA80EB80FC80F501878980312A
:1009F00049F481E0F8EFCF16FFEFDF06E104F104E0
:100A000050F4DBCF81E098EFC9169FEFD906E906D5
:100A10009FE0F90690F20F900F900F900F90DF91EA
:100A2000CF911F910F91FF90EF90DF90CF90BF90EB
:100A3000AF9008957F928F929F92AF92BF92CF9284
:100A4000DF92EF92FF920F931F93CF93DF93EC010E
:100A5000142F70934B0F60934A0F1F8A82E090E02F
:100A6000A0E0B0E088839983AA83BB831092490FEA
:100A70001092450F1092460F1092470F1092480F98
:100A80008FEF9FEFDC0180934C1190934D11A09359
:100A90004E11B0934F11442349F1453008F0DEC0A8
:100AA00040E060E070E0CB01B9DC882309F4D6C0F7
:100AB00020E1129FF0011124E650FF4E80818F77D4
:100AC00009F0CCC084859585A685B78584369105C7
:100AD000A105B10508F4C2C0C084D184E284F384C6
:100AE000C114D104E104F10421F4B8C0C12CD12C0B
:100AF000760140E0C701B60191DC782E882309F425
:100B0000ADC08091570F9091580F8115924009F018
:100B1000A5C030915C0F332309F4A0C080915A0F17
:100B200090915B0F892B09F499C02091590F2223D2
:100B300009F494C03A8B2C831D8630E041E050E0EC
:100B40006D85062FCA01062E02C0880F991F0A94D0
:100B5000E2F72817390731F081E0860F8D8768307A
:100B600078F37CC02091620F3091630F211531051D
:100B700019F040E050E008C02091700F3091710FE3
:100B80004091720F5091730F2D833E834F8358878E
:100B900080915A0F90915B0F46015701880E991E64
:100BA000A11CB11C8B8A9C8AAD8ABE8AE0915D0F24
:100BB000F0915E0FF98FE88FA0915C0FB0E00E947A
:100BC00044DF680D791D8A1D9B1D6A8F7B8F8C8F7A
:100BD0009D8FB5E0EE0FFF1FBA95E1F7E150FE4F94
:100BE000EF2FFF27E695DC01CB018E0F9F1FA11D84
:100BF000B11D8E879F87A88BB98B80905F0F9090D7
:100C0000600F8114910419F0A12CB12C08C08090C0
:100C10006C0F90906D0FA0906E0FB0906F0FA701AA
:100C20009601281B390B4A0B5B0BDA01C901880DB1
:100C3000991DAA1DBB1D04C0B695A79597958795CC
:100C40000A95D2F789879A87AB87BC87853F3FE0B3
:100C50009307A105B10520F48CE08F8B712C15C092
:100C6000853F9F4FA105B10510F480E10DC0809133
:100C7000780F9091790FA0917A0FB0917B0F8A8FA6
:100C80009B8FAC8FBD8F80E28F8B872DDF91CF91B3
:100C90001F910F91FF90EF90DF90CF90BF90AF909A
:100CA0009F908F907F90089580916511811109C068
:100CB00080916411811105C080916311811101C07F
:100CC0000895E2EEF4E18491882341F09091C00010
:100CD00095FFFCCF8093C6003196F5CFE3EDFCE0A5
:100CE0008491882341F09091C00095FFFCCF8093C0
:100CF000C6003196F5CF809165118823F1F060919F
:100D000066117091671180916811909169110E942C
:100D1000D1DB20911F0F3091200F4091210F509176
:100D2000220F0E9436DBAB01BC018FEC9CE00E94DD
:100D30002B278FEB9CE00E94BFAA8091641188232F
:100D4000F1F060916A1170916B1180916C1190912A
:100D50006D110E94D1DB2091230F3091240F40911F
:100D6000250F5091260F0E9436DBAB01BC018BEBA7
:100D70009CE00E942B278BEA9CE00E94BFAA8091F6
:100D800063118823F1F060916E1170916F11809161
:100D90007011909171110E94D1DB2091270F309139
:100DA000280F4091290F50912A0F0E9436DBAB018A
:100DB000BC0187EA9CE00E942B2787E99CE00E9407
:100DC000BFAA8091C00085FFFCCF8AE08093C60057
:100DD000109265111092641110926311089510928F
:100DE00065111092641110926311089580936D0241
:100DF0000895EFE6F0E080818260808308951F927D
:100E00000F920FB60F9211240BB60F920F931F93F0
:100E10002F933F934F935F936F937F938F939F9302
:100E2000AF93BF93EF93FF93809196119091971199
:100E3000892B09F086C19091ED098091EC099817F2
:100E400071F0E091EC098DE4E89FF0011124E2518A
:100E5000F64FDF01A45BBF4F81E08C9302C0E0E05E
:100E6000F0E0F0939711E0939611309709F463C185
:100E7000DF01A45BBF4F81E08C9310927911109237
:100E80007A1110927B1110927C1160AD71AD6134BA
:100E90009CE9790728F461329EE4790748F002C0A2
:100EA00060E47CE9769567957695679584E007C060
:100EB000613197E2790730F07695679582E080930B
:100EC000761107C0809376116032710510F460E2EC
:100ED00070E060527109611588E07807D0F0872FC3
:100EE0009927880F991F880F991F8E519F4EFC01DB
:100EF000329645915491AA27659F9001649F210DD8
:100F00003A1F06942A1F3A1F1124FC0185919491DF
:100F10001DC0CB01969587958C7F8E51934FFC0118
:100F2000459154910296FC0185919491FB01E770E3
:100F3000FF278E9F90018F9F300D9E9F300D1124B3
:100F4000E3E036952795EA95E1F7CA01821B930BFA
:100F500084369105A0F4ECE5F4E08191882339F022
:100F60009091C00095FFFCCF8093C600F6CF4AE079
:100F700050E086EC94E00E94FF2284E690E090939B
:100F800075118093741180917611992787FD909542
:100F90009093731180937211E0919611F0919711D3
:100FA00064AD75AD709378116093771161349CE9ED
:100FB000790728F461328EE4780748F002C060E4D3
:100FC0007CE9769567957695679584E007C06131F1
:100FD00097E2790730F07695679582E080937611F5
:100FE00008C081E0809376116032710510F460E2F0
:100FF00070E060527109611588E07807E0F0872F92
:101000009927880F991F880F991F8E519F4EFC01B9
:10101000329625913491AA27639FA001629F410DCA
:101020005A1F06944A1F5A1F1124FC01259134911E
:10103000241B350B1EC0CB01969587958C7F8E5156
:10104000934FFC01259134910296FC0145915491F6
:10105000FB01E770FF274E9FC0014F9F900D5E9FE1
:10106000900D1124F3E096958795FA95E1F7281BEA
:10107000390B24363105A0F4ECE5F4E081918823A6
:1010800039F09091C00095FFFCCF8093C600F6CF59
:101090004AE050E086EC94E00E94FF2224E630E033
:1010A000C901A0E0B0E080937D1190937E11A093E0
:1010B0007F11B09380113093890020938800E091D4
:1010C0009611F091971180899189A289B389B6957B
:1010D000A79597958795B095A095909581959F4FE9
:1010E000AF4FBF4F8093911190939211A0939311A2
:1010F000B093941180938D1190938E11A0938F11C2
:10110000B09390118093891190938A11A0938B11C1
:10111000B0938C118093851190938611A0938711C1
:10112000B093881110928111109282111092831144
:101130001092841106C080ED97E09093890080930F
:101140008800E0919611F0919711309709F4C3C48B
:1011500080A18093951180FF03C0899A8FEF02C010
:10116000899881E0809369028091951181FF03C085
:101170008F988FEF02C08F9A81E080936A0220914E
:10118000951120FF3BC080916D028823B9F16599CC
:1011900002C080E031C080916211882361F1E0914A
:1011A0009611F091971180819181A281B3811816D7
:1011B00019061A061B06FCF48091501190915111EA
:1011C000A0915211B09153118093661190936711C1
:1011D000A0936811B093691181E0809365118089B3
:1011E0009189A289B3898093811190938211A093F0
:1011F0008311B093841181E08093621121FF3DC07F
:1012000080916D028823C9F18091030181FD02C0A4
:1012100080E031C080916111882361F1E0919611E5
:10122000F091971184819581A681B78118161906CE
:101230001A061B06FCF48091541190915511A0914F
:101240005611B091571180936A1190936B11A0932E
:101250006C11B0936D1181E0809364118089918944
:10126000A289B3898093811190938211A0938311F5
:10127000B093841181E0809361119FB722FF48C031
:10128000F89480910B01826080930B019FBF8FEFD8
:1012900080936B0280916D02882309F443C029B1C9
:1012A00031E023FB222720F9232779F18091601177
:1012B000882359F1E0919611F091971180859185DD
:1012C000A285B385181619061A061B06F4F4809138
:1012D000581190915911A0915A11B0915B118093BE
:1012E0006E1190936F11A0937011B09371113093A0
:1012F000631180899189A289B38980938111909328
:101300008211A0938311B0938411209360110AC0BD
:10131000F89480910B018D7F80930B019FBF81E03A
:1013200080936B028091951183FF03C016988FEF15
:1013300002C0169A81E080936C0220E080917611C1
:1013400028170CF0BCC18091C00087FF19C03091F4
:10135000C6004091470550914805CA0101968F7714
:1013600099276091490570914A058617970741F0C2
:10137000FA01E953FB4F308390934805809347056A
:10138000E0919611F09197118091911190919211A5
:10139000A0919311B0919411408151816281738128
:1013A000840F951FA61FB71F8093911190939211E0
:1013B000A0939311B0939411181619061A061B06E0
:1013C000CCF5889AE0919611F09197118091911146
:1013D00090919211A0919311B091941140895189EB
:1013E00062897389841B950BA60BB70B80939111AF
:1013F00090939211A0939311B0939411409169022C
:101400008091501190915111A0915211B0915311AE
:10141000552747FD5095652F752F840F951FA61FE3
:10142000B71F8093501190935111A0935211B09314
:1014300053118898E0919611F091971180918D1138
:1014400090918E11A0918F11B0919011448155818E
:1014500066817781840F951FA61FB71F80938D111A
:1014600090938E11A0938F11B093901118161906B6
:101470001A061B06CCF58E9AE0919611F091971101
:1014800080918D1190918E11A0918F11B09190113A
:101490004089518962897389841B950BA60BB70B10
:1014A00080938D1190938E11A0938F11B093901112
:1014B00040916A028091541190915511A09156115A
:1014C000B0915711552747FD5095652F752F840F03
:1014D000951FA61FB71F8093541190935511A09389
:1014E0005611B09357118E98E0919611F091971183
:1014F0008091891190918A11A0918B11B0918C11DA
:101500004085518562857385840F951FA61FB71F7F
:101510008093891190938A11A0938B11B0938C11B1
:10152000181619061A061B060CF047C09FB7F89448
:1015300080910B01886080930B019FBFE091961111
:10154000F09197118091891190918A11A0918B113E
:10155000B0918C114089518962897389841B950BE4
:10156000A60BB70B8093891190938A11A0938B11CE
:10157000B0938C1140916B02809158119091591148
:10158000A0915A11B0915B11552747FD5095652FD9
:10159000752F840F951FA61FB71F80935811909326
:1015A0005911A0935A11B0935B119FB7F894809191
:1015B0000B01877F80930B019FBFE0919611F09103
:1015C00097118091851190918611A0918711B0910A
:1015D00088114485558566857785840F951FA61FDC
:1015E000B71F8093851190938611A0938711B093B4
:1015F0008811181619061A061B06CCF5149AE091E4
:101600009611F09197118091851190918611A0917A
:101610008711B09188114089518962897389841B2F
:10162000950BA60BB70B8093851190938611A09311
:101630008711B093881140916C0280915C11909158
:101640005D11A0915E11B0915F11552747FD509536
:10165000652F752F840F951FA61FB71F80935C11F0
:1016600090935D11A0935E11B0935F1114988091D7
:10167000811190918211A0918311B09184110196F2
:10168000A11DB11D8093811190938211A0938311AC
:10169000B093841140918111509182116091831116
:1016A00070918411E0919611F09197118089918940
:1016B000A289B389481759076A077B07B0F04091A0
:1016C0008111509182116091831170918411E09188
:1016D0009611F091971184899589A689B789841705
:1016E0009507A607B70718F4DAC02F5F27CE4091F9
:1016F0007D1150917E1160917F1170918011048D48
:10170000158D268D378DAA27419FB12D529FC0017F
:10171000629F900D619F800D911D429FB00D811DB4
:101720009A1F519FB00D811D9A1F609FB00D811DA2
:101730009A1F509FB10D8A1F9A1FB6958A1F9A1F34
:10174000112444AD55AD480F591F50937811409363
:10175000771180AD91ADA2ADB3AD60E070E08417BC
:101760009507A607B70720F4909378118093771117
:10177000609177117091781161349CE9790728F4B0
:1017800061328EE4780748F002C060E47CE9769527
:1017900067957695679584E007C0613197E2790790
:1017A00030F07695679582E08093761108C081E0ED
:1017B000809376116032710510F460E270E060523F
:1017C0007109611588E07807E0F0872F9927880F65
:1017D000991F880F991F8E519F4EFC0132962591BB
:1017E0003491AA27639FA001629F410D5A1F06945E
:1017F0004A1F5A1F1124FC0125913491241B350BDB
:101800001EC0CB01969587958C7F8E51934FFC011E
:10181000259134910296FC0145915491FB01E770AA
:10182000FF274E9FC0014F9F900D5E9F900D11248A
:1018300013E0969587951A95E1F7281B390B243606
:101840003105A0F4ECE5F4E08191882339F0909122
:10185000C00095FFFCCF8093C600F6CF4AE050E071
:1018600086EC94E00E94FF2224E630E03093890069
:101870002093880080917D1190917E11A0917F111D
:10188000B0918011820F931FA11DB11D80937D1116
:1018900090937E11A0937F11B0938011F7C0409177
:1018A0008111509182116091831170918411808D0A
:1018B000918DA28DB38D84179507A607B70708F001
:1018C000D9C04091791150917A1160917B1170913A
:1018D0007C11048D158D268D378DAA27419FB12D42
:1018E000529FC001629F900D619F800D911D429F8C
:1018F000B00D811D9A1F519FB00D811D9A1F609FD1
:10190000B00D811D9A1F509FB10D8A1F9A1FB69569
:101910008A1F9A1F11242091771130917811E05C71
:10192000FF4F2817390718F42081318102C0281B86
:10193000390B80819181A281B381A90160E070E0BF
:10194000481759076A077B0708F49C0121349CE972
:10195000390728F421328EE4380748F002C020E429
:101960003CE9369527953695279584E007C02131C7
:1019700097E2390730F03695279582E0809376110B
:1019800008C081E0809376112032310510F420E206
:1019900030E0B90160527109611588E07807E0F024
:1019A000872F9927880F991F880F991F8E519F4E57
:1019B000FC01329625913491AA27639FA001629F72
:1019C000410D5A1F06944A1F5A1F1124FC012591EC
:1019D0003491241B350B1EC0CB01969587958C7FC7
:1019E0008E51934FFC01259134910296FC01459153
:1019F0005491FB01E770FF274E9FC0014F9F900D50
:101A00005E9F900D112443E0969587954A95E1F7E6
:101A1000281B390B24363105A0F4ECE5F4E0819164
:101A2000882339F09091C00095FFFCCF8093C600C9
:101A3000F6CF4AE050E086EC94E00E94FF2224E6D4
:101A400030E0309389002093880080917911909143
:101A50007A11A0917B11B0917C11820F931FA11D6F
:101A6000B11D8093791190937A11A0937B11B0935B
:101A70007C110CC080917411909175119093890024
:101A8000809388008091721180937611409181112A
:101A9000509182116091831170918411E09196119F
:101AA000F091971180899189A289B38948175907C4
:101AB0006A077B0780F0109297111092961190910F
:101AC000ED098091EC09981731F08091EC098F5F56
:101AD0008F708093EC09FF91EF91BF91AF919F912F
:101AE0008F917F916F915F914F913F912F911F91B6
:101AF0000F910F900BBE0F900FBE0F901F90189577
:101B0000819A879AEAE0F1E08081826080830E9A70
:101B10003B9A579A5F9A829A8A9AE7E0F1E080812D
:101B2000816080839FB7F894E8E0F1E08081816074
:101B300080839FBF0A9A129A3F9A479A6D98759A26
:101B4000E4E0F1E080818D7F80839FB7F894E5E049
:101B5000F1E08081826080839FBF53985B9A809A76
:101B600088985F9A10922707869A8E988A9A109280
:101B70002807EAE0F1E08081886080839FB7F894CD
:101B8000EBE0F1E08081877F80839FBF9FB7F8946F
:101B9000E8E0F1E08081816080839FBF1092290797
:101BA0000C9A1498129A399A4198A1E8B0E08C9155
:101BB0008F7E8C938C9188608C93E0E8F0E080813C
:101BC0008D7F808380818E7F808380818F738083EF
:101BD00080818F7C80838C91887F82608C9380E071
:101BE00090E4909389008093880010928500109271
:101BF0008400EFE6F0E080818260808381E0809362
:101C00006D02789408959091ED098091EC099817F0
